:1000000086C70000B5C70000B3C70000B1C7000035
:10001000AFC70000ADC70000ABC70000A9C7000014
:10002000A7C70000A5C70000A3C70000A1C7000024
:100030009FC700000C9486459BC7000099C700002D
:1000400097C7000095C7000093C7000091C7000044
:100050008FC700008DC700008BC700000C941E5195
:1000600087C700000C94B04F0C94874F81C70000E5
:100070007FC700007DC700007BC7000079C7000074
:1000800077C7000075C7000073C7000071C7000084
:100090006FC700006DC700006BC700000C94AC4632
:1000A00067C7000065C7000063C7000061C70000A4
:1000B0005FC700005DC700005BC7000059C70000B4
:1000C00057C7000055C7000053C700000C945E4F8F
:1000D0000C94354F4DC700000C940C4F0C94E34E1C
:1000E00047C7000042342434493449344934493440
:1000F0004934493449344934493449349C1FB22184
:100100001424E7259E26BA2779297D2AF52A0A2B69
:100110000E2B4934212B252B192CD62D4D2F7E301B
:10012000DE30B73133323A3240334934493449341E
:1001300049344934493449344934493449347B33A6
:100140004934493449344934493449347734CC4A00
:10015000CF4ABE4AC24AC84A064BD34AD74ADD4AAA
:10016000E14AE54AEB4AEF4AF34A064BF94AFD4AAF
:10017000014B084AD73B3BCE016E84BCBFFDC12F6B
:100180003D6C74319ABD56833DDA3D00C77F11BE88
:10019000D9E4BB4C3E916BAAAABE000000803F0789
:1001A000634236B79BD8A71A39685618AEBAAB5512
:1001B0008C1D3CB7CC5763BD6DEDFD753EF61772D7
:1001C00031BF000000803F08000000BE92244912A9
:1001D0003EABAAAA2ABECDCCCC4C3E00000080BECD
:1001E000ABAAAAAA3E00000000BF000000803F00AA
:1001F00000000000084178D3BB4387D1133D190E9E
:100200003CC3BD4282AD2B3E68EC8276BED98FE105
:10021000A93E4C80EFFFBE01C4FF7F3F00000000FD
:1002200000004E414E494E495459494E46CDCCCC22
:100230003D0AD7233C17B7D13877CC2B329595E6BA
:10024000241FB14F0A000020410000C84200401C9A
:100250004620BCBE4CCA1B0E5AAEC59D7400407AE7
:1002600010F35A00A0724E18090010A5D4E800003F
:10027000E87648170000E40B54020000CA9A3B00DD
:100280000000E1F505000080969800000040420F54
:10029000000000A08601000000102700000000E818
:1002A00003000000006400000000000A00000000DD
:1002B000000100000000002C76D888DC674F08237E
:1002C000DFC1DFAE59E1B1B796E5E3E453C63AE6E4
:1002D00051997696E8E6C28426EB898C9B62ED40C4
:1002E0007C6FFCEFBC9C9F40F2BAA56FA5F4900513
:1002F0005A2AF75C936B6CF9676DC11BFCE0E40D47
:1003000047FEF520E6B500D0ED902E03009435773A
:10031000050080841E080000204E0A000000C80C62
:10032000333333330F986E12831141EF8D211489CB
:100330003BE65516CFFEE6DB18D1844B381BF77C25
:100340001D901DA4BBE424203284725E228100C96A
:10035000F124ECA1E53D2723616E6F74686572207E
:10036000495220696E7075743D0023696E70757412
:100370002044535463616C6962726174653A002071
:10038000766F6C746167653D0023547572626964B1
:10039000697479205570706572204C696D69743A82
:1003A000200020766F6C746167653D0023434F32F7
:1003B000207A65726F20766F6C74202800234F328C
:1003C0002063616C6962726174696F6E3A20002308
:1003D000547572626964697479204C6F7765722014
:1003E0004C696D69742056313A2000235061726166
:1003F0006D6574657273003E4D6F74696F6E206237
:100400007920756C747261736F6E632073656E739F
:100410006F723A0A004E6F20445320546865726D23
:100420006F6D6574657221004F3220436F6E6300FB
:10043000434F3220436F6E630053656E736F7220BB
:100440006572726F722100234E6F2073656E736F39
:10045000722100434F3220436F6E63004D6561731C
:100460007572696E6700234E6F2073656E736F72CD
:1004700020666F7220504D21004E6F2073656E73A1
:100480006F722100504D313A322E353A3130004DE5
:100490006561737572696E672E2E0054757262699C
:1004A0006469747900234E6F2073656E736F7220D8
:1004B000666F722074656D7020262068756D6964A2
:1004C00069747921004E6F2053656E736F7221003D
:1004D00020666F722074656D7020262068756D69C6
:1004E0006469747921002353656E736F72204572BD
:1004F000726F72200053656E736F72204572726F57
:100500007221002357726F6E672073656E736F726E
:1005100020666F722074656D7020262068756D6985
:1005200064697479210057726F6E672053656E732A
:100530006F72210054656D702048756D696469742F
:1005400079004C6967687420496E74656E736974CC
:100550007900466C616D65204952007048207661D3
:100560006C756500496E76616C6964206B657921F4
:1005700000237265706C6965733D0067657453652F
:100580006C665465737442697428293A2000697353
:10059000496E74657272757074456E61626C6564E3
:1005A0002831293A2000676574496E746572727546
:1005B00070744D617070696E672831293A20006748
:1005C0006574496E74657272757074536F75726379
:1005D000652831293A2000676574496E7465727226
:1005E000757074536F7572636528293A20006765CA
:1005F000745261746528293A20332E3134313539EB
:100600003F00616363656C2E69734C6F77506F7741
:10061000657228293A2000616363656C2E69734115
:10062000736C65657028293A2000616363656C2EE0
:100630006973546170536F757263654F6E5A2829E0
:100640003A2000616363656C2E6973546170536F67
:10065000757263654F6E5928293A2000616363659E
:100660006C2E6973546170536F757263654F6E5869
:1006700028293A2000616363656C2E6973416374B5
:100680006976697479536F757263654F6E5A28295C
:100690003A2000616363656C2E6973416374697607
:1006A000697479536F757263654F6E5928293A20C2
:1006B0000069734163746976697479536F75726305
:1006C000654F6E5828293A2000697354617044655B
:1006D00074656374696F6E4F6E5A28293B2066619A
:1006E0006C73653F20006973546170446574656381
:1006F00074696F6E4F6E5A28293B20747275653F7E
:1007000020006973546170446574656374696F6E29
:100710004F6E5928293B2066616C73653F20006944
:1007200073546170446574656374696F6E4F6E597C
:1007300028293B20747275653F20006973546170ED
:10074000446574656374696F6E4F6E5828293B2049
:1007500066616C73653F2000697354617044657411
:10076000656374696F6E4F6E5828293B20747275EB
:10077000653F2000676574537570707265737342CE
:10078000697428293B2066616C73653F20006765AA
:1007900074537570707265737342697428293B20B5
:1007A000747275653F20006973416374697669747A
:1007B00079416328293A20006973496E616374693D
:1007C000766974795A456E61626C656428293A20AD
:1007D000006973496E616374697669747959456E0D
:1007E00061626C656428293A20006973496E61630F
:1007F00074697669747958456E61626C65642829FC
:100800003A2000697341637469766974795A456E58
:1008100061626C656428293A2000697341637469D8
:100820007669747959456E61626C656428293A204D
:10083000006973416374697669747958456E6162C1
:100840006C656428293A20006765744672656546C0
:10085000616C6C4475726174696F6E28293A20006E
:100860006765744672656546616C6C546872657341
:10087000686F6C6428293A200067657454696D6557
:10088000496E616374697669747928293A20006732
:100890006574496E616374697669747954687265C8
:1008A00073686F6C642829200067657441637469FC
:1008B000766974795468726573686F6C642829204E
:1008C00000676574446F75626C6554617057696E3A
:1008D000646F7728292000676574446F75626C65C2
:1008E0005461704C6174656E637928293A20006701
:1008F00065745461704475726174696F6E28293A29
:100900002000676574417869734F66667365742863
:1009100026782C2026792C20267A293A2000676513
:10092000745461705468726573686F6C6428293AF6
:10093000200058595A2047733A200058595A2043EA
:100940004F554E54533A2000736574206761696EA9
:10095000735B5D3A006761696E735F6F7269675BB5
:100960005D3A00005EBCE2613FDD83C29C7E20A355
:10097000FD1F41009D23BE46DB65F88C11AF32CAD6
:1009800057E97443616C6962726174696F6E2050DB
:10099000726573737572653D00536561206C657691
:1009A000656C20502863616C63293D002345727299
:1009B0006F723A707265737375726520424D503074
:1009C00038352C20636865636B20776972696E67C0
:1009D000210049522054656D702073656E736F72EB
:1009E00020666F756E6400504D322E352073656E33
:1009F000736F72206C696B656C7920666F756E64BD
:100A000000536F756E64204C6576656C2073656E5F
:100A1000736F7220666F756E640053656E736F72CC
:100A200020736C6F7420616E6420747970653A0075
:100A300057656C636F6D6520746F20456455484B36
:100A40000000002100240027002A002D0030003380
:100A50000001010000040107010A01000022002535
:100A60000028002B002E0031003400020100000598
:100A70000108010B01000020002300260029002CA2
:100A8000002F0032000001000003010601090105EA
:100A9000050505070508080808020202020A0A08F7
:100AA000080404040401010101010101010303031D
:100AB0000303030303040707070C0C0C0C0C0C0CBA
:100AC0000C0202020206060606060606060B0B0BC1
:100AD0000B0B0B0B0B0102102020080810204010FC
:100AE00020408002010201080402010102040810F2
:100AF0002040808040201008040201800402018010
:100B00004020100804020108040201010204081038
:100B1000204080010204081020408000000A0B02DF
:100B2000090C0D0E0807030401000000000000007E
:100B300000000000000000000000000000000000B5
:100B40000000000000000012111000000000000072
:100B50000000000000000000000000000000000095
:100B6000004E6F2073656E736F72210049522054DE
:100B7000656D7065726174757265004D6561737540
:100B800072696E672E2E004572726F72206E756DDF
:100B900062657220666F722074686520617272618E
:100BA0007920746F206176726167696E67212F6E9C
:100BB00000236B6579323D00236B6579323D004F30
:100BC0006666206169722D636F6E64210049742727
:100BD0007320746F6F20636F6F6C210054656D70AC
:100BE0002069732066696E6521004973206169720E
:100BF0002D636F6E64206F6E3F0049742773207100
:100C00007569746520686F742100497427732076B4
:100C100065727920686F742120004F6666206169D3
:100C2000722D636F6E6421004974277320746F6F97
:100C300020636F6F6C210054656D702069732066AE
:100C4000696E6521004973206169722D636F6E645E
:100C5000206F6E3F00497427732071756974652099
:100C6000686F742100497427732076657279206853
:100C70006F74210054656D702048756D69646974E6
:100C8000790020202020202020202020202020202B
:100C90002020002020202020202020202020202074
:100CA0002020200020202020202020202020202064
:100CB0002020202000202020202020202020202054
:100CC0002020202020002020202020202020202044
:100CD0002020202020002020202020202020202034
:100CE000202020202000233A53686F772F48696422
:100CF00065204C4344002A3A546869732048656C67
:100D0000700044433A436C656172204C4344004494
:100D1000423A5265736574204C6F67676572004490
:100D2000373A4D6F74696F6E0044363A445320541D
:100D3000656D700044353A555620496E74656E7382
:100D40006974790044343A4F3220636F6E632E0029
:100D500044333A434F3220636F6E632E0044323A7D
:100D6000504D28313A322E353A3130290044323A4A
:100D7000504D28313A322E353A3130292A0044314B
:100D80003A5475726269646974790044303A566FF6
:100D90006C7461676500393A6F7220334420616377
:100DA00063656C2E00393A496E636C2E20616E6764
:100DB0002E00383A70482076616C756500373A49E4
:100DC000522054656D7000373A49522054656D7059
:100DD0002A00363A4D61676E6574696320666965FD
:100DE0006C6400353A476173204C6576656C00345D
:100DF0003A495220466C616D6500333A4C69676828
:100E00007420496E742E00323A616E642048656920
:100E100067687400323A54656D7020507265737360
:100E200075726500313A54656D702048756D69645E
:100E300069747900303A536F756E64204C6576653D
:100E40006C00303A536F756E64204C6576656C2A81
:100E500000232D2D2D2D2D2D2D2D2D2D2D2D2D2DF9
:100E60002D2D2D2D2D2D2D2D2D2D2D2D2D2D2D2DB2
:100E70002D2D2D2D2D2D00235265736F6C757469EA
:100E80006F6E3A20202000234D696E2056616C75EC
:100E9000653A2020202000234D61782056616C7532
:100EA000653A202020200023556E69717565204920
:100EB000443A20202020002344726976657220562F
:100EC00065723A202020002353656E736F723A20BA
:100ED00020202020202000232D2D2D2D204D616746
:100EE0006E657469632053656E736F72202D2D2DAE
:100EF0002D2D2D2D2D2D2D2D2D2D2D2D2D2D2D2D22
:100F00002D00416E676C65732F003084C9831124F6
:100F10001FBECFEFD1E2DEBFCDBF00E00CBF1BE0B4
:100F2000A0E0B2E0E2E9F5E201E00BBF02C0079009
:100F30000D92AA3AB107D9F721E1AAEABBE001C0B4
:100F40001D92A33CB207E1F717E0C6E8D7E000E046
:100F500006C021970109802FFE010E941D90C5380F
:100F6000D10780E00807A9F70E94A27C0C94B892F0
:100F700047C82F923F924F925F926F927F928F92CB
:100F80009F92AF92BF92CF92DF92EF92FF920F9318
:100F90001F93CF93DF93CDB7DEB7EA970FB6F894E0
:100FA000DEBF0FBECDBF84EC9BE00E941935892BBC
:100FB00009F468C20E94D95B0E94586C64E07BE02F
:100FC000CE0101960E94C84D4AE050E060E070E01A
:100FD000CE0101960E94ED6DCE0101960E94FE4C5D
:100FE00080914E0C8823B9F06EE97AE08DEF9EE097
:100FF0000E94E24E4091C80B5091C90B6091CA0B00
:101000007091CB0B20E18DEF9EE00E942A4E8DEF78
:101010009EE00E94BF4E8091C80B9091C90BA09199
:10102000CA0BB091CB0B883025E09207A105B10522
:1010300009F405C208F08DC0893461E09607A10566
:10104000B10509F4FFC1E0F58434E1E09E07A10594
:10105000B10509F4E8C1E8F4813421E09207A10563
:10106000B10509F4D1C138F480349140A105B1052E
:1010700009F4BBC1EAC1823471E09707A105B1054B
:1010800009F4CBC183349140A105B10509F4C8C16D
:10109000DCC18634F1E09F07A105B10509F4C9C19F
:1010A00008F4C4C1873441E09407A105B10509F4EF
:1010B000C3C188349140A105B10509F4C0C1C5C1BF
:1010C000823075E09707A105B10509F4A6C1E8F4DF
:1010D0008437F1E09F07A105B10509F451C138F447
:1010E00082379140A105B10509F455C1AEC1811502
:1010F00065E09607A105B10509F477C181309540F7
:10110000A105B10509F480C1A0C18530E5E09E07C5
:10111000A105B10509F48AC170F4833025E0920776
:10112000A105B10509F47CC184309540A105B10544
:1011300009F479C18AC1863065E09607A105B10539
:1011400009F477C187309540A105B10509F474C150
:101150007CC18D3BE2E49E07EFEFAE07B10509F4D9
:1011600035C108F04BC08F3E20E192072FEFA20758
:10117000B10509F461C118F5823365E09607A10550
:10118000B10509F408C138F489309540A105B105CD
:1011900009F458C15AC18433F5E09F07A105B10590
:1011A00009F4EEC08D3F9240AF4FB10509F04DC13B
:1011B0006EE775E08DE990E10E94D44CE9C08D3D69
:1011C00042E294074FEFA407B10509F4D9C038F4FF
:1011D000873E9841AF4FB10509F428C136C18F3C15
:1011E000E0E39E07EFEFAE07B10509F41CC1873CB1
:1011F0009843AF4FB10509F422C127C1873928E6CA
:1012000092072FEFA207B10509F4FEC048F58D3A09
:1012100062E596076FEFA607B10509F4C8C038F478
:10122000853B9A44AF4FB10509F4DFC00EC1853A42
:10123000FAE59F07FFEFAF07B10509F403C18D3948
:101240009246AF4FB10509F000C16BE775E08DE93B
:1012500090E10E94D44C1092820C8CEF9FEF8DC0D5
:10126000873548EA94074FEFA407B105F9F078F401
:1012700085387AE797077FEFA707B10509F4D9C04A
:1012800087369849AF4FB10509F4C7C0DEC08F3427
:10129000F0EB9F07FFEFAF07B10509F4C1C08D3335
:1012A000924CAF4FB10509F476C0CFC082E0809375
:1012B000A60F1092AA0F00E010E08AEA9BE00E94BD
:1012C0001935892B69F40F5F1F4F093E43E014075E
:1012D00039F06EE170E080E090E00E94DA50EDCFEE
:1012E00080914E0C8823B9F067E573E08DEF9EE0A6
:1012F0000E94F14D4091AE0B5091AF0B6091B00B3D
:101300007091B10B2AE08DEF9EE00E942A4E8DEF86
:101310009EE00E94BF4E8091AE0B9091AF0BA091CA
:10132000B00BB091B10B853065E09607A105B10512
:1013300009F44EC308F0CEC28734E1E09E07A10550
:10134000B10509F451C308F0A5C2833421E0920726
:10135000A105B10509F42AC308F092C2813461E005
:101360009607A105B10509F084C26AE675E081E936
:1013700090E10E94D44C89EF9FEF0E94221F7CC015
:101380006EE775E08DE990E10E94D44C1092820CDA
:101390008BEF9FEFF2CF61E875E08DE990E10E945D
:1013A000D44C81E08093820C8DEF9FEFE6CF64E810
:1013B00075E081E990E10E94D44C64E875E08DE924
:1013C00090E10E94D44C8EEF9FEFD7CF67E875E095
:1013D00081E990E10E94D44C67E875E08DE990E1E5
:1013E0000E94D44C8FEF9FEFC8CF65E775E081E98D
:1013F00090E10E94D44C65E775E08DE990E10E9490
:10140000D44C80E090E0B9CF68E875E081E990E1E4
:101410000E94D44C81E090E0B0CF82E090E0ADCF6C
:1014200083E090E0AACF84E090E0A7CF85E090E051
:10143000A4CF86E090E0A1CF87E090E09ECF88E047
:1014400090E09BCF89E090E098CF60E070E0CE0123
:1014500001960E94CC64BE016F5F7F4F81E990E1ED
:101460000E94434CCE0101960E94FE4C64E670E05F
:1014700080E090E00E94DA5082E08093A60F109204
:10148000AA0F09C16CED7AE08DE990E10E94D44C7D
:101490001092BB0B6CED7AE08DE990E10E94D44C88
:1014A00001E08DEF9EE00E94D4492091BB0B1816FD
:1014B00019060CF0DEC22111DCC29FC28091210D01
:1014C0009091220D892B71F46FE776E0CE010196A1
:1014D0000E94C84DCE0101960E94F06ACE0101968D
:1014E0000E94FE4C8091210D9091220D019771F484
:1014F0006EE876E0CE0101960E94C84DCE010196BD
:101500000E94F06ACE0101960E94FE4C6091230277
:10151000709124024AE0CE0145960E948D4D68E903
:1015200076E0CE0101960E94C84DBE016B5E7F4FF2
:10153000CE0101960E941349BC01CE0183960E9400
:10154000C04DCE0183960E94F06ACE0183960E9420
:10155000FE4CCE0101960E94FE4CCE0145960E94A3
:10156000FE4C409100025091010260910202709184
:10157000030222E0CE0145960E94324D64EB76E0F4
:10158000CE0101960E94C84DBE016B5E7F4FCE0119
:1015900001960E94134964EB78E00E94FC48BC016C
:1015A000CE0183960E94C04DCE0183960E94F06AC0
:1015B000CE0183960E94FE4CCE0101960E94FE4C05
:1015C000CE0145960E94FE4C40910C0250910D02B6
:1015D00060910E0270910F0222E0CE0145960E94AA
:1015E000324D64EC76E0CE0101960E94C84DBE01FA
:1015F0006B5E7F4FCE0101960E94134964EB78E049
:101600000E94FC48BC01CE0183960E94C04DCE01D1
:1016100083960E94F06ACE0183960E94FE4CCE0112
:1016200001960E94FE4CCE0145960E94FE4CB12CC4
:101630008091A1109091A210039708F0E7C50E9435
:10164000D95B0E94586C64E07BE0CE0101960E9459
:10165000C84D4AE050E060E070E0CE0101960E9483
:101660003B6DCE0101960E94FE4C8091A11090919D
:10167000A2108130910509F057C5E0919D10F091BD
:101680009E10309711F40C94FC1E1081812F0E9443
:10169000076B0E9412510E9412516093C00B70930D
:1016A000C10B8093C20B9093C30BD5C083EC9DE01C
:1016B0000E94B2498093BA0B8A3009F4E6C18D309A
:1016C00009F4E3C19091BB0B9111DFC189831A82A8
:1016D00041E050E0BE016F5F7F4F8DE990E10E94D5
:1016E000CF488FEFE81AF80A6FE070E080E090E0F2
:1016F0000E94DA5083EC9DE00E94D4491816190626
:10170000ACF262E370E080E090E00E94DA50EF28F3
:1017100039F163E975E0CE0145960E94C84D6DE947
:1017200070E1CE0145960E941349BC01CE0101969D
:101730000E94C04DCE0101960E94BD70CE0101965F
:101740000E94FE4CCE0145960E94FE4C83EC9DE02B
:101750000E94624A64E670E080E090E00E94DA5005
:101760002091BB0B8091A1109091A210222309F42B
:1017700083C10197D1F564EB78E0CE0101960E9418
:10178000C84DCE0101960E940658811198C169E9A1
:1017900075E0CE0145960E94C84DCE0145960E9447
:1017A000065801E0811100E0CE0145960E94FE4CF2
:1017B000CE0101960E94FE4C002389F060E070E0AB
:1017C000CE0101960E94CC64BE016F5F7F4F81E91C
:1017D00090E10E94434CCE0101960E94FE4C64E1D0
:1017E00070E080E090E00E94DA506AE070E080E013
:1017F00090E00E94DA508091A1109091A210009781
:1018000009F05FC10E94377A182F81110C946C1E69
:101810008091820C81110C948A1E0E9412510091B9
:10182000C00B1091C10B2091C20B3091C30BDC0196
:10183000CB01801B910BA20BB30B88349E4EA105EC
:10184000B10548F01092961160E08BE891E10E949A
:101850004045109280048091820C882311F40C94EE
:10186000091F64E670E080E090E00E94DA500C947A
:10187000091F82349140A105B10509F48EC0F6CD4F
:101880008534E1E09E07A105B10509F4A1C008F483
:1018900096C0A7C0813025E09207A105B10509F4E3
:1018A00064CD70F4883461E09607A105B10509F4B0
:1018B0009EC089349140A105B10509F49BC0D6CDE5
:1018C0008330E5E09E07A105B10509F46FC008F477
:1018D00064C075C08F3C20E392072FEFA207B105CB
:1018E00009F46DC068F5883065E09607A105B1057B
:1018F00009F47DC070F48630E5E09E07A105B105CE
:1019000009F46FC087309540A105B10509F46CC09A
:10191000ADCD8F3E20E192072FEFA207B10509F46C
:1019200063C0873E48E194074FEFA407B10509F46F
:101930004FC089309540A105B10509F097CD5AC037
:10194000873978E697077FEFA707B10509F40DCD32
:1019500078F4873CF8E39F07FFEFAF07B10509F480
:1019600046C0853A9A45AF4FB10509F443C07ECDD4
:10197000873648E994074FEFA407B10571F08F341B
:1019800060EB96076FEFA607B10581F085389A479F
:10199000AF4FB10509F06ACD24C06DE675E081E96D
:1019A00090E10E94D44C88EF9FEFE7CC60E775E0B0
:1019B00081E990E10E94D44C87EF9FEFDECC63E792
:1019C00075E081E990E10E94D44C86EF9FEFD5CC81
:1019D00067E775E081E990E10E94D44C85EF9FEFC5
:1019E000CCCC84EF9FEFC9CC83EF9FEFC6CC82EFC6
:1019F0009FEFC3CC81EF9FEFC0CC8DEF9EE00E94A4
:101A0000B2498093BA0B8A3071F08D3061F08983CE
:101A10001A8241E050E0BE016F5F7F4F8DE990E197
:101A20000E94CF481FC00093BB0B6AE875E0CE014F
:101A300045960E94C84D6DE970E1CE0145960E9421
:101A40001349BC01CE0101960E94C04DCE01019602
:101A50000E94BD70CE0101960E94FE4CCE014596BB
:101A60000E94FE4C6AE070E080E090E00E94DA5054
:101A700018CD211175CE05C0009709F07ACE0C94CF
:101A8000D11EE12CF12C01E035CE8091A110909176
:101A9000A210892B09F428CE0093BB0B83EC9DE0A8
:101AA0000E94D449181619060CF01ECE6CED7AE08F
:101AB0008DE990E10E94D44C1092BB0B15CE00E052
:101AC00077CE0197E1F56BE975E0CE0183960E9430
:101AD000C84DCE0183960E94065881110C94031FB5
:101AE0006FE779E0CE0145960E94C84DCE0145963C
:101AF0000E940658811112C060E17BE0CE01019680
:101B00000E94C84DCE0101960E94065801E0811145
:101B100000E0CE0101960E94FE4C01C000E0CE0123
:101B200045960E94FE4CCE0183960E94FE4C0023F7
:101B300031F06DE970E181E990E10E94E94C80911A
:101B4000A1109091A2100497E8F56DE975E0CE011F
:101B500001960E94C84DCE0101960E940658082F9A
:101B6000CE0101960E94FE4C002361F161E070E01D
:101B7000CE0101960E94CC64CE0101960E94654878
:101B80002AEFC22EDD24DA94ED2CFD2C46015701FC
:101B9000861A970AA80AB90AB501A4012AE0CE015B
:101BA00045960E94614DBE016B5E7F4F81E990E1D9
:101BB0000E94434CCE0145960E94FE4CCE010196F8
:101BC0000E94FE4C6FE975E0CE0145960E94C84D1B
:101BD000CE0145960E940658811113C063EA75E054
:101BE000CE0101960E94C84DCE0101960E94065872
:101BF00001E0811101C000E0CE0101960E94FE4C7F
:101C000001C001E0CE0145960E94FE4C002309F47C
:101C100088C26BEE73E0CE0101960E94B84DCE01F2
:101C200001960E94F06ACE0101960E94FE4C67EA7E
:101C300075E0CE0101960E94C84D65E871E1CE01C4
:101C400001960E941349BC01CE0145960E94C04DE9
:101C5000CE0145960E94F06ACE0145960E94FE4C48
:101C6000CE0101960E94FE4C6091450270914602A1
:101C700080914702909148020E943F8B20E030E023
:101C800048EC52E40E948F8DAB01BC0122E0CE01F2
:101C900045960E94324D6DEB75E0CE0101960E9493
:101CA000C84DBE016B5E7F4FCE0101960E94134965
:101CB0006BE077E00E94FC48BC01CE0183960E9455
:101CC000C04DCE0183960E94F06ACE0183960E9499
:101CD000FE4CCE0101960E94FE4CCE0145960E941C
:101CE000FE4C40914102509142026091430270913A
:101CF000440224E0CE0145960E94324D62ED75E02B
:101D0000CE0101960E94C84DBE016B5E7F4FCE0191
:101D100001960E941349BC01CE0183960E94C04DDA
:101D2000CE0183960E94F06ACE0183960E94FE4CFB
:101D3000CE0101960E94FE4CCE0145960E94FE4CBB
:101D4000409135025091360260913702709138020D
:101D500022E0CE018F960E94324D40912D0250918B
:101D60002E0260912F027091300223E0CE018996FD
:101D70000E94324D4091390250913A0260913B02EB
:101D800070913C0222E0CE0183960E94324D409138
:101D9000310250913202609133027091340223E09B
:101DA000CE0145960E94324D6FEE75E0CE01019650
:101DB0000E94C84DBE016B5E7F4FCE0101960E940E
:101DC000134964E076E00E94FC48BE016D5D7F4FE0
:101DD0000E94134967E076E00E94FC48BE01675DFF
:101DE0007F4F0E94134964E076E00E94FC48BE01E8
:101DF000615D7F4F0E9413496DE076E00E94FC48D0
:101E0000BC01CE01C5960E94C04DCE01C5960E9470
:101E1000F06ACE01C5960E94FE4CCE0101960E944A
:101E2000FE4CCE0145960E94FE4CCE0183960E9448
:101E3000FE4CCE0189960E94FE4CCE018F960E94E8
:101E4000FE4C4091C2045091C3046091C40470914F
:101E5000C50423E0CE0183960E94324D2091BA043E
:101E60003091BB044091BC045091BD0460E070E02F
:101E700080E291E40E943D8FAB01BC0121E0CE01E4
:101E800045960E94034D62E176E0CE0101960E94E4
:101E9000C84DBE016B5E7F4FCE0101960E94134973
:101EA00065E276E00E94FC48BE016D5D7F4F0E94B6
:101EB00013496BE276E00E94FC48BC01CE01899692
:101EC0000E94C04DCE0189960E94F06ACE0189968B
:101ED0000E94FE4CCE0101960E94FE4CCE0145961A
:101EE0000E94FE4CCE0183960E94FE4C4091BE049F
:101EF0005091BF046091C0047091C10423E0CE01F1
:101F000083960E94324D2091B6043091B7044091DF
:101F1000B8045091B90460E070E080E291E40E945E
:101F20003D8FAB01BC0121E0CE0145960E94034DDF
:101F30006EE276E0CE0101960E94C84DBE016B5E56
:101F40007F4FCE0101960E94134965E276E00E9420
:101F5000FC48BE016D5D7F4F0E9413496BE276E045
:101F60000E94FC48BC01CE0189960E94C04DCE0162
:101F700089960E94F06ACE0189960E94FE4CCE019D
:101F800001960E94FE4CCE0145960E94FE4CCE0169
:101F900083960E94FE4C4091290250912A02609142
:101FA0002B0270912C0222E0CE0145960E94324D08
:101FB00061E476E0CE0101960E94C84DBE016B5EE1
:101FC0007F4FCE0101960E94134967E576E00E949B
:101FD000FC48BC01CE0183960E94C04DCE01839681
:101FE0000E94F06ACE0183960E94FE4CCE010196BB
:101FF0000E94FE4CCE0145960E94FE4C4091250267
:1020000050912602609127027091280222E0CE01B1
:1020100045960E94324D6EE576E0CE0101960E9413
:10202000C84DBE016B5E7F4FCE0101960E941349E1
:102030006BE276E00E94FC48BC01CE0183960E94D0
:10204000C04DCE0183960E94F06ACE0183960E9415
:10205000FE4CCE0101960E94FE4CCE0145960E9498
:10206000FE4C03E1C02E02E0D02EEE24E394F12CCE
:1020700007E180911102909112028E159F050CF4D8
:102080001DCAF601A190B1906F014AE0B501CE01E1
:1020900083960E948D4D4AE0B701CE0145960E947D
:1020A0008D4D61E776E0CE0101960E94C84DBE01DC
:1020B0006B5E7F4FCE0101960E9413496DE47BE079
:1020C0000E94FC48BE016D5D7F4F0E94134969E785
:1020D00076E00E94FC480A9DB0010B9D700D112412
:1020E000655A7D4F0E94FC48BC01CE0189960E9432
:1020F000C04DCE0189960E94F06ACE0189960E9459
:10210000FE4CCE0101960E94FE4CCE0145960E94E7
:10211000FE4CCE0183960E94FE4CFFEFEF1AFF0AA1
:10212000A8CFBB24B39484CA029709F0AFCA6DE963
:1021300075E0CE0101960E94C84DCE0101960E9425
:102140000658082FCE0101960E94FE4C002309F488
:102150009DCA8091A1109091A210029740F0E09149
:102160009D10F0919E10309711F0818101C080E0A8
:102170001A8219821C821B821E821D828D8B1E8AEE
:10218000BE016B5E7F4FCE0101960E94D44CBE0112
:102190006F5F7F4F81E990E10E94434CCE01019631
:1021A0000E94FE4C8091A1109091A210892B41F0C9
:1021B000E0919D10F0919E10309711F0108101C0B8
:1021C00010E080914E0C882309F460CA64ED76E03B
:1021D000CE0101960E94C84D6DE970E1CE010196D5
:1021E0000E94134964E07BE00E94FC48BC018DEF33
:1021F0009EE00E94E34DCE0101960E94FE4C61E9F3
:1022000070E18DEF9EE00E94D24E40CA41E050E066
:1022100060E070E0CE0101960E948A64BE016F5FAB
:102220007F4F8FE790E10E94434CCE0101960E94C0
:10223000FE4C67E077E0CE0145960E94C84DCE0186
:1022400045960E940658811113C06CE07BE0CE01D8
:1022500001960E94C84DCE0101960E94065811E0D9
:10226000811101C010E0CE0101960E94FE4C01C018
:1022700011E0CE0145960E94FE4C112309F4B2C034
:1022800062E070E0CE0101960E94CC64BE016F5FF7
:102290007F4F8FE790E10E94434CCE0101960E9450
:1022A000FE4C6FE770E1CE0101960E94C04DCE0159
:1022B00001960E94BD70CE0101960E94FE4C0E94C4
:1022C000074820E030E048EC52E40E949E8B0E94D8
:1022D000288EAB01BC0140934502509346026093A7
:1022E0004702709348022AE0CE0101960E94614D98
:1022F000CE0101960E94BD70CE0101960E94FE4C57
:102300006091450270914602809147029091480287
:102310008B019C0100591F452140310901341C49A2
:102320002105310588F06AED76E0CE0101960E9424
:10233000C84D6FE770E1CE0101960E9413496DEE22
:1023400076E00E94FC4852C119821A821B821C82CC
:102350001D821E821F8218860E943F8B20E030E083
:1023600048EC52E40E948F8D8E010F5F1F4F22E0D8
:1023700047E00E946B86BC0185E890E10E94D44C46
:102380006DEF76E0CE0145960E94C84D65E870E19C
:10239000CE0145960E9413496AE077E00E94FC480E
:1023A000BC0185E890E10E94E94CCE0145960E946F
:1023B000FE4C1092780C1092770C8091450290910F
:1023C0004602A0914702B09148028093AB0C9093D3
:1023D000AC0CA093AD0CB093AE0C80E090E00E94EA
:1023E00039650DC16FE077E0CE0145960E94C84D7A
:1023F000CE0145960E940658811113C065E177E031
:10240000CE0101960E94C84DCE0101960E94065849
:1024100011E0811101C010E0CE0101960E94FE4C36
:1024200001C011E0CE0145960E94FE4C112309F433
:1024300067C046E050E065E070E0CE0101960E9482
:102440008A64BE016F5F7F4F8FE790E10E94434C2B
:10245000CE0101960E94FE4C8FE790E10E946548F4
:102460006B017C0165E576E0CE0101960E94C84DC6
:10247000CE0101960E941348BC016F5F7F4FCE01D1
:1024800045960E94CC64BE016B5E7F4F8FE790E162
:102490000E94434CCE0145960E94FE4CCE0101960F
:1024A0000E94FE4C8FE790E10E946548DB01E1E16C
:1024B000F2E041E050E02091110230911202241725
:1024C00035075CF0228133812A173B0711F4138210
:1024D00012824F5F5F4F3296EECF9601220F331F6D
:1024E000F901EF5EFD4F7183608382E090E00E940E
:1024F000305D6DE970E18DEF9EE00E94D24ECDC25D
:102500006BE177E0CE0145960E94C84DCE0145961D
:102510000E940658811113C061E277E0CE01019656
:102520000E94C84DCE0101960E94065811E081110B
:1025300001C010E0CE0101960E94FE4C01C011E0E6
:10254000CE0145960E94FE4C1123F1F0E1E1F2E04C
:1025500081E090E020911102309112022817390792
:1025600074F0863091051CF49383828305C09C012E
:102570002E5F3F4F3383228301963296EBCF82E06A
:1025800090E00E94305D89C267E277E0CE01459617
:102590000E94C84DCE0145960E940658811113C075
:1025A0006FE277E0CE0101960E94C84DCE01019600
:1025B0000E94065811E0811101C010E0CE01019681
:1025C0000E94FE4C01C011E0CE0145960E94FE4CD7
:1025D000112359F167E377E0CE0101960E94C84DBF
:1025E0006FE771E1CE0101960E941349BC0185E8B5
:1025F00090E10E94E94CCE0101960E94FE4C6EE9EA
:102600007AE0CE0101960E94C84D65E870E1CE01E6
:1026100001960E941349BC01CE0145960E94C04D0F
:10262000CE0145960E94F06A9DC161E477E0CE013B
:1026300045960E94C84DCE0145960E9406588111CC
:1026400013C068E477E0CE0101960E94C84DCE0128
:1026500001960E94065811E0811101C010E0CE01E0
:1026600001960E94FE4C01C011E0CE0145960E94E9
:10267000FE4C1123A9F06FE477E0CE0101960E9491
:10268000C84D65E871E1CE0101960E941349BC0175
:1026900085E890E10E94E94CCE0101960C942D1D35
:1026A0006EE577E0CE0145960E94C84DCE01459675
:1026B0000E940658811113C063E677E0CE010196AF
:1026C0000E94C84DCE0101960E94065811E081116A
:1026D00001C010E0CE0101960E94FE4C01C011E045
:1026E000CE0145960E94FE4C112309F43FC065E5DA
:1026F00076E0CE0101960E94C84DCE0101960E945F
:102700001348BC016F5F7F4FCE0145960E94CC6499
:10271000BE016B5E7F4F8FE790E10E94434CCE017C
:1027200045960E94FE4CCE0101960E94FE4C8FE71A
:1027300090E10E9465486115710521F481E0809364
:10274000810410C06130710519F4109281040AC02F
:102750006230710511F00C944B0B81E08093810481
:10276000109280040E94E95B0C944B0B68E677E0C2
:10277000CE0145960E94C84DCE0145960E9406584E
:10278000811113C06CE677E0CE0101960E94C84D1E
:10279000CE0101960E94065811E0811101C010E09F
:1027A000CE0101960E94FE4C01C011E0CE0145967B
:1027B0000E94FE4C112309F470C063E070E0CE016A
:1027C00001960E94CC64BE016F5F7F4F8FE790E15E
:1027D0000E94434CCE0101960E94FE4C6FE770E1CF
:1027E0008DEF9EE00E94D24E1092780C1092770CE2
:1027F0006FE770E185E891E10E94E94C87EC9CE08D
:10280000892BE1F00091891110918A1101151105B0
:1028100019F41092C70C12C00730110510F007E030
:1028200010E06091851170918611A80187EC9CE001
:102830000E948F92F801E953F34F10828091770C38
:102840009091780C0E94396560E777E0CE0145965B
:102850000E94C84D65E871E1CE0145960E9413497A
:10286000BC01CE0101960E94C04DCE0145960E944A
:10287000FE4CBE016F5F7F4F83EC9DE00E94E34DF5
:1028800068EB7BE080E090E00E94DA5067EC7CE04F
:10289000CE0145960E94C84D61C068E777E0CE0141
:1028A00045960E94C84DCE0145960E94065881115A
:1028B00013C06DE777E0CE0101960E94C84DCE01AE
:1028C00001960E94065811E0811101C010E0CE016E
:1028D00001960E94FE4C01C011E0CE0145960E9477
:1028E000FE4C112309F444C064E070E0CE0101966F
:1028F0000E94CC64BE016F5F7F4F8FE790E10E9422
:10290000434CCE0101960E94FE4C62E877E0CE0176
:1029100045960E94C84D6FE770E1CE0145960E9432
:102920001349BC01CE0101960E94C04DCE014596CF
:102930000E94FE4CBE016F5F7F4F83EC9DE00E94C2
:10294000E34D68EB7BE080E090E00E94DA50BE014E
:102950006F5F7F4FCE0145960E94C04DCE014596D8
:102960000E94BD70CE0145960E94FE4C0C94661EDE
:1029700069E877E0CE0145960E94C84DCE014596A4
:102980000E940658811113C06EE877E0CE010196CF
:102990000E94C84DCE0101960E94065811E0811197
:1029A00001C010E0CE0101960E94FE4C01C011E072
:1029B000CE0145960E94FE4C1123E1F045E050E027
:1029C00064E070E0CE0101960E948A64BE016F5FF0
:1029D0007F4F8FE790E10E94434CCE0101960E9409
:1029E000FE4C8FE790E10E9465487093220D609342
:1029F000210D45C063E977E0CE0145960E94C84DA0
:102A0000CE0145960E940658811113C068E977E00F
:102A1000CE0101960E94C84DCE0101960E94065833
:102A200011E0811101C010E0CE0101960E94FE4C20
:102A300001C011E0CE0145960E94FE4C1123B9F170
:102A400046E050E064E070E0CE0101960E948A64A6
:102A5000BE016F5F7F4F8FE790E10E94434CCE0134
:102A600001960E94FE4C8FE790E10E9465487093AA
:102A7000240D6093230D70932402609323026DE96B
:102A800070E1CE0101960E94C04DCE0101960E94D8
:102A9000BD70CE0101960E94FE4C1092780C1092EF
:102AA000770C80E090E00E9439650C944B0B6DE947
:102AB00077E0CE0145960E94C84DCE0145960E9412
:102AC0000658811113C064EA77E0CE0101960E9496
:102AD000C84DCE0101960E94065811E0811101C037
:102AE00010E0CE0101960E94FE4C01C011E0CE0123
:102AF00045960E94FE4C112311F147E050E066E03C
:102B000070E0CE0101960E948A64BE016F5F7F4F24
:102B10008FE790E10E94434CCE0101960E94FE4C4B
:102B20008FE790E10E946548672B21F410924E0CCC
:102B30000C945C1E81E080934E0C0C945C1E6BEA3E
:102B400077E0CE0183960E94C84DCE0183960E9405
:102B5000065881118FC76EEA77E0CE0145960E9434
:102B6000C84DCE0145960E940658811113C061EBF5
:102B700077E0CE0101960E94C84DCE0101960E94D9
:102B8000065811E0811101C010E0CE0101960E94AB
:102B9000FE4C01C011E0CE0145960E94FE4CCE01D4
:102BA00083960E94FE4C111169C765EE77E0CE0155
:102BB00001960E94C84DCE0101960E940658182F1A
:102BC000CE0101960E94FE4C112309F46CC0809145
:102BD000A1109091A210079710F40C94581E66E073
:102BE00070E0CE0101960E94CC64BE016F5F7F4F02
:102BF0008FE790E10E94434CCE0101960E94FE4C6B
:102C00000E940748AB01BC014093000250930102AF
:102C1000609302027093030221E0CE0145960E9468
:102C2000324D64EB76E0CE0101960E94C84DBE01A4
:102C30006B5E7F4FCE0101960E94134964EB78E0F2
:102C40000E94FC48BC0185E890E10E94E94CCE015D
:102C500001960E94FE4CCE0145960E94FE4C65E80E
:102C600070E1CE0101960E94C04DCE0101960E94F6
:102C7000F06ACE0101960E94FE4C0E94125128EE8D
:102C800033E040E050E00E94978CCA01B9010E94F5
:102C90003D8B6093BC0B7093BD0B8093BE0B9093E8
:102CA000BF0B0C94581E6CEE77E0CE0101960E948B
:102CB000C84DCE0101960E940658182FCE010196EC
:102CC0000E94FE4C112309F446C08091A1109091FE
:102CD000A210079708F4ECC766E070E0CE010196F9
:102CE0000E94CC64BE016F5F7F4F8FE790E10E942E
:102CF000434CCE0101960E94FE4C0E940748AB0156
:102D0000BC0140930C0250930D0260930E0270932D
:102D10000F0221E0CE0145960E94324D64EC76E030
:102D2000CE0101960E94C84DBE016B5E7F4FCE0161
:102D300001960E94134964EB78E00E94FC48BC01B4
:102D400085E890E10E94E94CCE0101960E94FE4C7C
:102D5000CE01459682C663EF77E0CE0145960E948C
:102D6000C84DCE0145960E940658811114C067EFE8
:102D700077E0CE0101960E94C84DCE0101960E94D7
:102D80000658FF24F394811101C0F12CCE01019665
:102D90000E94FE4C02C0FF24F3948E010B5E1F4F75
:102DA000C8010E94FE4CFF2009F455C080917404B4
:102DB000909175040E94695F6093310270933202B2
:102DC00080933302909334026093BF0C7093C00CD5
:102DD0008093C10C9093C20C80E090E0A0E8BFE328
:102DE0008093390290933A02A0933B02B0933C0245
:102DF0008093B70C9093B80CA093B90CB093BA0C15
:102E000080914E0C882381F06FEC73E08DEF9EE093
:102E10000E94F14D60913102709132028091330233
:102E2000909134020E94F9541092780C1092770C11
:102E300080E090E00E943965409131025091320269
:102E4000609133027091340222E0C8010E94324D39
:102E50006BEF77E0EFC564E078E0C8010E94C84DF1
:102E6000C8010E940658811114C06AE078E0CE01C2
:102E700001960E94C84DCE0101960E940658FF247B
:102E8000F394811101C0F12CCE0101960E94FE4CF9
:102E900002C0FF24F394C8010E94FE4CFF2009F4F5
:102EA000B6C08091A1109091A2100797D8F066E06B
:102EB00070E0CE0101960E94CC64BE016F5F7F4F2F
:102EC0008FE790E10E94434CCE0101960E94FE4C98
:102ED0000E9407486093290270932A0280932B0274
:102EE00090932C02809172049091730499270E9410
:102EF0006B5EBC01990F880B990B0E943F8B2DE0F4
:102F000038E643E55BE30E949E8B6B017C012091D8
:102F10009E0430919F044091A0045091A1040E940E
:102F2000398B18164CF0609186047091870480915B
:102F30008804909189041BC02091B2043091B3049D
:102F40004091B4045091B504C701B6010E947E8E31
:102F500087FF05C0C701B6010E94F36308C06091F6
:102F60009A0470919B0480919C0490919D0420E0B0
:102F700030E048EC52E40E949E8B6B017C0120E023
:102F800030E0A9010E94398B181634F0C12CD12CE5
:102F9000A8EAEA2EA1E4FA2EC0922902D0922A02CF
:102FA000E0922B02F0922C02C092DF0CD092E00C47
:102FB000E092E10CF092E20C80914E0C882381F0BB
:102FC0006DEB73E08DEF9EE00E94F14D6091290260
:102FD00070912A0280912B0290912C020E94F95448
:102FE0001092780C1092770C80E090E00E94396586
:102FF0004091290250912A0260912B0270912C027B
:1030000022E0C8010E94324D60E178E013C56AE118
:1030100078E0C8010E94C84DC8010E94065881117D
:1030200014C06FE178E0CE0101960E94C84DCE0138
:1030300001960E940658FF24F394811101C0F12CDF
:10304000CE0101960E94FE4C02C0FF24F394C801F9
:103050000E94FE4CFF2009F492C08091A110909133
:10306000A2100697E8F065E070E0CE0101960E949C
:10307000CC64BE016F5F7F4F8FE790E10E94434CAD
:10308000CE0101960E94FE4C0E9407480E94BF8E0E
:103090006093BA047093BB048093BC049093BD0406
:1030A0008091C6049091C7040E94F18320E030E033
:1030B00048E051E40E948F8D6093C2047093C30472
:1030C0008093C4049093C5046093CF0C7093D00C8C
:1030D0008093D10C9093D20C8091BA049091BB0450
:1030E000A091BC04B091BD048093D70C9093D80CF0
:1030F000A093D90CB093DA0C80914E0C882341F147
:103100006CEA73E08DEF9EE00E94F14D2091BA04CD
:103110003091BB044091BC045091BD0460E070E06C
:1031200080E291E40E943D8F41E050E00E94AC6259
:1031300064E278E08DEF9EE00E94E24E6091C2046E
:103140007091C3048091C4049091C5040E94F95405
:103150001092780C1092770C80E090E00E94396514
:103160004091C2045091C3046091C4047091C5049D
:1031700023E0C8010E94324D6BE278E0A9C066E30B
:1031800078E0C8010E94C84DC8010E94065881110C
:1031900014C06BE378E0CE0101960E94C84DCE01C9
:1031A00001960E940658FF24F394811101C0F12C6E
:1031B000CE0101960E94FE4C02C0FF24F394C80188
:1031C0000E94FE4CFF2009F491C08091A1109091C3
:1031D000A2100697E8F065E070E0CE0101960E942B
:1031E000CC64BE016F5F7F4F8FE790E10E94434C3C
:1031F000CE0101960E94FE4C0E9407480E94BF8E9D
:103200006093B6047093B7048093B8049093B904A4
:103210008091C6049091C7040E94F18320E030E0C1
:1032200048E051E40E948F8D6093BE047093BF0408
:103230008093C0049093C1046093D30C7093D40C1A
:103240008093D50C9093D60C2091B6043091B7049E
:103250004091B8045091B9042093DB0C3093DC0CFE
:103260004093DD0C5093DE0C80914E0C8823D1F0FE
:1032700060E070E080E291E40E943D8F41E050E028
:103280000E94AC6264E278E08DEF9EE00E94E24E24
:103290006091BE047091BF048091C0049091C104FC
:1032A0000E94F9541092780C1092770C80E090E014
:1032B0000E9439654091BE045091BF046091C004E2
:1032C0007091C10423E0C8010E94324D60E478E0AF
:1032D000CE0101960E94C84DB801CE0101960E9410
:1032E000134964E378E00E94FC48ADC369E478E0E8
:1032F000C8010E94C84DC8010E940658811114C01F
:103300006DE478E0CE0101960E94C84DCE01019691
:103310000E940658FF24F394811101C0F12CCE01C4
:1033200001960E94FE4C02C0FF24F394C8010E9443
:10333000FE4CFF2009F46DC060E080916E040E9495
:103340005450F9E1AF2EB12CC12CD12C76018091D3
:103350006E040E949050BC01990F880B990B0E943B
:103360003F8B9B01AC01C701B6010E94C98C6B0168
:103370007C016AE070E080E090E00E94DA5061E059
:10338000A61AB10821F720E030E040EA50E4C70176
:10339000B6010E949E8B20E030E040E85AE30E9494
:1033A0009E8B20E030E048EC51E40E948F8D6093CA
:1033B000250270932602809327029093280260933F
:1033C000F50C7093F60C8093F70C9093F80C109218
:1033D000780C1092770C80E090E00E943965409163
:1033E000250250912602609127027091280222E066
:1033F000C8010E94324D6EE576E0CE0101960E9432
:10340000C84DB801CE0101960E9413496BE276E0E7
:103410006ACF61E578E0C8010E94C84DC8010E94EA
:103420000658811114C065E578E0CE0101960E942E
:10343000C84DCE0101960E940658FF24F3948111D5
:1034400001C0F12CCE0101960E94FE4C02C0FF2467
:10345000F394C8010E94FE4CFF2009F435C146E0F8
:1034600050E064E070E0CE0101960E948A64BE01E3
:103470006F5F7F4F8FE790E10E94434CCE01019632
:103480000E94FE4C8FE790E10E9465484B015C0171
:103490001B0165E576E0CE0101960E94C84DCE0184
:1034A00001960E941348BC016F5F7F4FC8010E94C4
:1034B000CC64B8018FE790E10E94434CC8010E94A0
:1034C000FE4CCE0101960E94FE4CF0906C040E94CE
:1034D00007482B013C01640171E0C71AD1088091B3
:1034E0004E0C8823B9F06AE673E08DEF9EE00E94EF
:1034F000F14D4AE050E0B4018DEF9EE00E94B94EDC
:1035000064E07BE08DEF9EE00E94E24EC301B201D9
:103510000E94F9546F2DC8010E94114518870F832E
:103520001D821E82198289E08A8381E08B838C83CD
:103530001C8A1B8ACE0101960E946D44CE01019621
:103540000E94FD42CE0101960E94C456EE80F12CED
:103550008BE0E816F1041CF0EAE0EE2EF12CEBE52E
:103560008E16910408F44CC07FE4A72E7CE0B72EA1
:103570003501212C312C2101C12CD12CCE14DF049A
:10358000B9F06C2DCE0101960E94FF439B01AC0166
:10359000F30161937193819391933F01C201B10152
:1035A0000E94C98C1B012C01FFEFCF1ADF0AE6CF66
:1035B000B7010F2C000C880B990B0E943F8B9B01CD
:1035C000AC01C201B1010E948F8D2B013C01C12CC5
:1035D000D12CCE14DF0409F457C0F50120813181CC
:1035E00042815381C301B2010E94C88CF5016193ED
:1035F0007193819391935F01FFEFCF1ADF0AE9CFB7
:10360000121413040CF5E214F30424F4670121E00E
:10361000C21AD1086C2DCE0101960E94FF439B0176
:10362000AC01C601880F991F880F991FBC01615B0F
:10363000734F6B01C301B2010E94C88CF601608315
:1036400071838283938320C02328F1F44FE4A42E56
:103650004CE0B42EC12CD12CCE14DF04A9F06C2D7B
:10366000CE0101960E94FF439B01AC01C301B20150
:103670000E94C88CF50161937193819391935F01CE
:10368000FFEFCF1ADF0AE8CFEFE4FCE0A9EFBCE0E0
:1036900041915191619171914D935D936D937D93A2
:1036A0002CE0E737F207A1F71092780C1092770C14
:1036B00080E090E00E94396564E070E0C8010E94FB
:1036C000CC6469E578E0B6C16AE778E0C8010E9499
:1036D000C84DC8010E940658811114C06EE778E0F9
:1036E000CE0101960E94C84DCE0101960E94065857
:1036F000FF24F394811101C0F12CCE0101960E94A8
:10370000FE4C02C0FF24F394C8010E94FE4CFF202F
:1037100009F449C080917404909175040E94695F16
:1037200060932D0270932E0280932F0290933002AB
:103730006093C30C7093C40C8093C50C9093C60C1B
:10374000C12C30E5D32E33ECE32E37E4F32EC092B8
:103750003502D0923602E0923702F0923802C092DF
:10376000BB0CD092BC0CE092BD0CF092BE0C209130
:103770004E0C21110E94F9541092780C1092770C83
:1037800080E090E00E94396540912D0250912E0218
:1037900060912F027091300222E0C8010E94324DE8
:1037A00062E878E047C16DE878E0C8010E94C84D42
:1037B000C8010E940658811114C061E978E0CE0169
:1037C00001960E94C84DCE0101960E940658FF2422
:1037D000F394811101C0F12CCE0101960E94FE4CA0
:1037E00002C0FF24F394C8010E94FE4CFF2009F49C
:1037F00074C08091A1109091A2100497D8F064E059
:1038000070E0CE0101960E94CC64BE016F5F7F4FD5
:103810008FE790E10E94434CCE0101960E94FE4C3E
:103820000E9407486093390270933A0280933B02EA
:1038300090933C026091390270913A0280913B0270
:1038400090913C026093B70C7093B80C8093B90CC4
:103850009093BA0C20914E0C222321F042E050E0CC
:103860000E94AC6280917404909175040E94695F1B
:10387000609331027093320280933302909334024A
:103880006093BF0C7093C00C8093C10C9093C20CDA
:1038900080914E0C882381F062EA73E08DEF9EE008
:1038A0000E94F14D60913102709132028091330299
:1038B000909134020E94F9541092780C1092770C77
:1038C00080E090E00E9439654091310250913202CF
:1038D0006091330270913402A7C06DE978E0C801AD
:1038E0000E94C84DC8010E940658811114C061EAA7
:1038F00078E0CE0101960E94C84DCE0101960E944B
:103900000658FF24F394811101C0F12CCE010196D9
:103910000E94FE4C02C0FF24F394C8010E94FE4C9A
:10392000FF2009F4C5C18091A1109091A2100497C5
:10393000D8F064E070E0CE0101960E94CC64BE0134
:103940006F5F7F4F8FE790E10E94434CCE0101965D
:103950000E94FE4C0E940748609335027093360225
:10396000809337029093380280913502909136020D
:10397000A0913702B09138028093BB0C9093BC0C9D
:10398000A093BD0CB093BE0C80914E0C882391F097
:1039900069E873E08DEF9EE00E94F14D6091350281
:1039A00070913602809137029091380242E050E0E7
:1039B0000E94AC6280917404909175040E94695FCA
:1039C00060932D0270932E0280932F029093300209
:1039D0006093C30C7093C40C8093C50C9093C60C79
:1039E00080914E0C882381F06FE773E08DEF9EE0AD
:1039F0000E94F14D60912D0270912E0280912F0254
:103A0000909130020E94F9541092780C1092770C29
:103A100080E090E00E94396540912D0250912E0285
:103A200060912F027091300222E0C8010E94324D55
:103A300065E978E0CE0101960E94C84DB801CE013B
:103A400001960E941349BC0185E890E10E94E94C6F
:103A5000CE0101960E94FE4CC8010E94FE4C65E812
:103A600070E1CE0101960E94C04DCE0101960E94E8
:103A7000F06A2CC1CE0183960E94FE4C0AE010E051
:103A8000C12CD12C760166246A9483E0782E6EE1F5
:103A900070E080E090E00E94DA50809176040E940D
:103AA0009050B3010E940A90072E000C880B990BCE
:103AB0000E943F8B20E030E040EA50E40E949E8B61
:103AC0009B01AC01C701B6010E94C98C6B017C014E
:103AD00001501109E1F620E030E040E251E40E949B
:103AE0008F8D6B017C0164EB77E0CE0145960E94DF
:103AF000C84DCE0145960E940658811180C168EBE1
:103B000077E0CE0101960E94C84DCE0101960E9439
:103B1000065811E0811101C010E0CE0101960E940B
:103B2000FE4CCE0145960E94FE4C112309F43FC085
:103B300020E030E040E650E4C701B6010E949E8BD1
:103B40009B01AC0160E070E080E890E40E94C88CCA
:103B5000AB01BC014093040250930502609306023E
:103B60007093070222E0CE0101960E94324DBE0101
:103B70006F5F7F4F85E890E10E94434CCE01019634
:103B80000E94FE4C6CEB77E0CE0101960E94C84D7E
:103B900065E870E1CE0101960E941349BC0185E8F9
:103BA00090E10E94E94CCE0101960E94FE4C6BEC24
:103BB00077E0CE0145960E94C84DCE0145960E9401
:103BC000065881111EC160ED77E0CE0101960E947A
:103BD000C84DCE0101960E94065811E0811101C026
:103BE00010E0CE0101960E94FE4CCE0145960E9447
:103BF000FE4C112309F43FC020E030E040E650E4E1
:103C0000C701B6010E949E8B9B01AC0160E070E091
:103C100080E291E40E94C88CAB01BC014093080291
:103C20005093090260930A0270930B0222E0CE01C6
:103C300001960E94324DBE016F5F7F4F85E890E193
:103C40000E94434CCE0101960E94FE4C65ED77E048
:103C5000CE0101960E94C84D65E870E1CE01019643
:103C60000E941349BC0185E890E10E94E94CCE0115
:103C700001960E94FE4C6EE97AE0CE0101960E9408
:103C8000C84D65E870E1CE0101960E941349BC0160
:103C9000CE0145960E94C04DCE0145960E94F06A25
:103CA000CE0145960E94FE4CCE0101960E94FE4C2C
:103CB000BB2011F40C944B0B6DE970E1CE01019621
:103CC0000E94C04DCE0101960E94BD70CE010196AA
:103CD0000E94FE4C0C944B0B6CED7AE081E990E174
:103CE0000E94D44C80914E0C882379F065EA78E0EC
:103CF0008DEF9EE00E94E24E612F8DEF9EE00E94CC
:103D0000DC4D8DEF9EE00E94BF4E812F0E94076B1D
:103D10000C944B0B0E94125128EEC22E23E0D22E9F
:103D2000E12CF12CA70196010E94978CCA01B901E0
:103D30000E943D8B2091BC0B3091BD0B4091BE0B7E
:103D40005091BF0B0E94C88C20910002309101025B
:103D500040910202509103020E947E8E181614F0C8
:103D60000C940D0C0E941251A70196010E94978C91
:103D7000CA01B9010E943D8B6093BC0B7093BD0BCF
:103D80008093BE0B9093BF0B8091DC0B9091DD0B69
:103D900059D064E170E080E090E00E94DA500C9429
:103DA0002B0C64E670E080E090E00E94DA500E9404
:103DB0001251CB0168EE73E00E940A90CB0164E6D9
:103DC00070E00E940A908236910514F40C94F50B71
:103DD0008091820C81110C94F50B81E990E10E9495
:103DE0006548613071058105910511F00C94F50B62
:103DF0000E9452680C94F50B10E00C94460B11E0F5
:103E000090CE11E0F2CECE0183960E94FE4C0C942F
:103E10009F0DEA960FB6F894DEBF0FBECDBFDF91BF
:103E2000CF911F910F91FF90EF90DF90CF90BF90B7
:103E3000AF909F908F907F906F905F904F903F904A
:103E40002F9008952F923F924F925F926F927F92A0
:103E50008F929F92AF92BF92CF92DF92EF92FF929A
:103E60000F931F93CF93DF93CDB7DEB7CF55D10913
:103E70000FB6F894DEBF0FBECDBF1C0100914A0CF7
:103E800010914B0C80914E0C882349F061E775E04E
:103E90008DEF9EE00E94F14DC1010E948854C10146
:103EA0000596059708F180914A0C90914B0C82156C
:103EB000930519F10E94586C30924B0C20924A0CD9
:103EC0000E94D95B4AE0B101CE0101960E948D4D5E
:103ED000BE016F5F7F4F81E990E10E94434CCE01AC
:103EE00001960E94FE4C09C02EEF22162FEF3206DB
:103EF000B1F40E94E95B0C94FF3464E07BE0CE01F6
:103F000001960E94C84D4AE050E06FEF7FEFCE016E
:103F100001960E943B6DCE0101960E94FE4CF1017C
:103F20007996E533F10510F00C9449348827EE5862
:103F3000FF4F8F4F0C941D908091820C882321F0AD
:103F40000E94665A0C947734C0900C02D0900D02F7
:103F5000E0900E02F0900F020E9412512E966CAF6C
:103F60007DAF8EAF9FAF2E9761E0809184040E9459
:103F7000545060E0809182040E9454500E94655326
:103F80006093830C7093840C8093850C9093860CC3
:103F900023E333E948E853E40E948F8D20E030E0CA
:103FA00040E85FE30E94C98C0E948D8F26E636EAC6
:103FB00045EA53E40E949E8B6093870C7093880CB3
:103FC0008093890C90938A0C0E94245A62966CAF5D
:103FD0007DAF8EAF9FAF62970E94B5504B015C01E1
:103FE0006AE070E080E090E00E94DA5067EF73E0F2
:103FF00085E890E10E94384920E030E04AE754E447
:10400000C701B6010E949E8B66966CAF7DAF8EAFE6
:104010009FAF6697412C512C3201C12CD12C7601D7
:10402000C701B6010E943F8B66962CAD3DAD4EADEB
:104030005FAD66970E94398B87FF8DC10E94125138
:104040002E962CAD3DAD4EAD5FAD2E97621B730B22
:10405000840B950B0E943D8B20E030E04AE754E44E
:104060000E948F8DAB01BC0123E0CE0101960E941E
:10407000324DBE016F5F7F4F8FE790E10E94434C4E
:10408000CE0101960E94FE4C0E94245A6B017C01D5
:104090000E94B5509B01AC01281939094A095B09F6
:1040A00049015A0131ED831637E09306A104B104AA
:1040B0000CF443C020E030E0A901C701B6010E9422
:1040C0007E8E18165CF426EA3BE944EC5BE3C701FC
:1040D000B6010E94398B87FF0BC02FC026EA3BE94F
:1040E00044EC5BEBC701B6010E947E8E18162CF1E2
:1040F000C501B40128EE33E040E050E00E946B8C33
:10410000CA01B9010E943F8B4B015C0162962CAD44
:104110003DAD4EAD5FAD6297C701B6010E94C88C40
:1041200020E030E04AE754E40E949E8BA501940110
:104130000E948F8D4B015C0103C0812C912C540196
:104140006FE770E1CE0101960E94C04D64EB78E00C
:10415000CE0101960E94FC48BC018FE790E10E94CD
:10416000E94CCE0101960E94FE4C23E0B701A60166
:10417000CE0180960E94324DBE01605E7F4FCE011F
:1041800001960E94C04D6BEA78E0CE0101960E9434
:10419000FC48BC0189E790E10E94E94CCE01019600
:1041A0000E94FE4CCE0180960E94FE4C22E0B5019A
:1041B000A401CE0101960E94324D69E57BE0CE015B
:1041C00080960E94C84D6FE770E1CE0180960E94F4
:1041D00013496EEA78E00E94FC4869E770E10E94AA
:1041E00013496EED7AE00E94FC48BE016F5F7F4F7D
:1041F0000E94134962EB78E00E94FC48BC0185E80C
:1042000090E10E943249CE0180960E94FE4CCE0180
:1042100001960E94FE4C20E030E0A901C501B401E6
:104220000E947E8E87FD06C064E07BE089E790E116
:104230000E94244922E0B501A401CE0180960E948B
:10424000324DBE01605E7F4FCE0101960E94C04D8F
:1042500062EB78E0CE0101960E94FC48BC0189E740
:1042600090E10E943249CE0101960E94FE4CCE019F
:1042700080960E94FE4C65E870E1CE0101960E9496
:10428000C04DCE0101960E94F06ACE0101960E94B7
:10429000FE4CC301B20125E030E040E050E00E9456
:1042A0006B8C672B682B692B21F566EB78E0CE01D0
:1042B00001960E94C84D45E050E060E070E0CE01FC
:1042C00001960E94ED6DCE0101960E94FE4C69E7B9
:1042D00070E1CE0101960E94C04D45E050E06FEFC5
:1042E0007FEFCE0101960E94BC6CCE0101960E9428
:1042F000FE4C6CED7AE085E890E10E94D44C65E0DC
:1043000070E080E090E00E94DA500E9412516B0150
:104310007C012E962CAD3DAD4EAD5FAD2E97C21AF1
:10432000D30AE40AF50A0E94245A62966CAF7DAF64
:104330008EAF9FAF62970E94B5504B015C016AE05F
:1043400070E080E090E00E94DA503FEF431A530A99
:10435000630A730A65CE60E0809184040E94545021
:104360000C947734F0906C046CED7AE0CE01805CB4
:104370009F4F0E94C84D8E01005E1F4F6F2DC801D8
:104380000E94114518870F831D821E82198289E0C1
:104390008A8381E08B838C831C8A1B8ACE010196E1
:1043A0000E946D44CE0101960E94FD42CE0101960D
:1043B0000E94C4560E8110E00330110509F46FC14C
:1043C0006DEB78E0CE01805C9F4F0E94D44C6CED89
:1043D0007AE085E890E10E94D44CBE01605C7F4F9A
:1043E000CE018E960E94C04D4AE050E060E070E041
:1043F000CE018E960E94ED6DCE018E960E94FE4CEF
:1044000061E080E00E94A36161EE78E0CE01805C13
:104410009F4F0E94D44C5FE4A52E5CE0B52ECC24C7
:10442000C394D12CE12CF12CE016F1060CF0EEC077
:104430006E2DCE0101960E94FF43D5012D913D9135
:104440004D915D915D010E94C98C2B013C0120E0E2
:1044500030E04CEF52EC0E94398B87FF21C04AE0DC
:10446000B601CE018E960E948D4D65EA75E0CE01B3
:10447000C4960E94C84DBE01625D7F4FCE01C496B6
:104480000E94134967EC78E00E94FC48BC0185E873
:1044900090E10E943249CE01C4960E94FE4C45C074
:1044A00022E0B301A201CE018E960E94324D4AE075
:1044B000B601CE01C4960E948D4D65EA75E0CE012D
:1044C000CA960E94C84DBE016C5C7F4FCE01CA9651
:1044D0000E94134965E576E00E94FC48BE01625DDA
:1044E0007F4F0E941349BC0189E790E10E94E94C8B
:1044F000CE01CA960E94FE4CCE01C4960E94FE4C8C
:10450000CE018E960E94FE4C69E770E1CE018E9638
:104510000E94C04D64E07BE0CE018E960E94FC4874
:10452000BC0185E890E10E943249CE018E960E943E
:10453000FE4C0130110561F4E114F10409F05FC093
:1045400065E870E1CE01805C9F4F0E94E94C57C046
:104550000230110519F522E0B301A201CE01C49683
:104560000E94324DBE016C5C7F4FCE018E960E9440
:10457000C04D64E07BE0CE018E960E94FC48BC01F9
:10458000CE01805C9F4F0E943249CE018E960E94E0
:10459000FE4CCE01C4960E94FE4C31C00330110582
:1045A00071F169E770E1CE018E960E94C04D44E141
:1045B00050E06FEF7FEFCE018E960E94BC6CCE0173
:1045C0008E960E94FE4C60E17BE0CE018E960E94AA
:1045D000C84DCE018E960E947C6CCE018E960E94B4
:1045E000FE4C80918104882351F0809180048823BF
:1045F00031F060ED77E080E090E00E94DA50BFEFAC
:10460000EB1AFB0AEFEFCE1ADE0A0ECFCE01805C6A
:104610009F4F0E94704885E890E10E947048011504
:104620001105A9F465E174E085E890E10E9438493C
:1046300063ED78E0CE018E960E94C84D4AE050E0CE
:104640006FEF7FEFCE018E960E94BC6CE4C0043009
:10465000110514F00C949934BE01605C7F4FCE01BB
:104660008E960E94C04D4AE050E06FEF7FEFCE0182
:104670008E960E94BC6CCE018E960E94FE4C60E12C
:104680007BE0CE018E960E94C84DCE018E960E9490
:104690007C6CCE018E960E94FE4C0C9499346EED8B
:1046A00078E0CE01805C9F4F0E94D44CBE01605CDC
:1046B0007F4FCE018E960E94C04D4AE050E060E0F0
:1046C00070E0CE018E960E94ED6DCE018E960E9416
:1046D000FE4C6CED7AE085E890E10E94D44C65E8F0
:1046E00070E1CE01805C9F4F0E94E94C00E010E039
:1046F000602FCE0101960E94FF436B017C0122E0F6
:10470000AB01BC01CE010115110569F48E960E9422
:10471000324DBE01625D7F4F8BE891E10E94E34D17
:10472000CE018E961CC0C4960E94324DBE016C5CB8
:104730007F4FCE018E960E94C04D64E07BE0CE019B
:104740008E960E94FC48BC01CE01805C9F4F0E9467
:104750003249CE018E960E94FE4CCE01C4960E9434
:10476000FE4C22E0B701A601CE01C4960E94324D54
:10477000BE016C5C7F4FCE018E960E94C04D64E0FE
:104780007BE0CE018E960E94FC48BC0185E890E15A
:104790000E943249CE018E960E94FE4CCE01C496F4
:1047A0000E94FE4C0F5F1F4F0330110509F0A0CF90
:1047B000CE01805C9F4F0E947048BE01605C7F4FBD
:1047C000CE018E960E94C04D4AE050E06FEF7FEF21
:1047D000CE018E960E94BC6CCE018E960E94FE4C3D
:1047E0000E949A6C85E890E10E94704864EE78E03F
:1047F000CE018E960E94C84D65E870E1CE018E967E
:104800000E9413496EEE78E00E94FC48BC0185E8E6
:1048100090E10E94E94CCE018E960E94FE4CCE01A2
:10482000805C9F4F0C947534F0916E046896FFAFD6
:10483000689760E08F2F0E9454508091820C8823EB
:1048400059F022E030E040E050E06C962CAF3DAFF4
:104850004EAF5FAF6C970AC08FE090E0A0E0B0E091
:104860006C968CAF9DAFAEAFBFAF6C9761E079E057
:1048700085E890E10E94D44C65E870E1CE01019694
:104880000E94C04D4AE050E06FEF7FEFCE010196ED
:104890000E94ED6DCE0101960E94FE4CC12CD12CE0
:1048A00076012B961FAE2B972F961FAE2F976396F0
:1048B0001FAE639767961FAE679702E310E0412C27
:1048C000512C320168968FAD68970E949050092E46
:1048D000000CAA0BBB0B480E591E6A1E7B1E65E01E
:1048E00070E080E090E00E94DA500150110951F729
:1048F0008090250290902602A0902702B090280276
:10490000C301B2010E943F8B20E030E040EA50E456
:104910000E949E8B20E030E040E85AE30E949E8B8C
:1049200020E030E048E452E40E948F8DA50194011C
:104930000E94C88C20E030E040E751E40E949E8B4A
:104940002B013C01A50194016AE979E989E390E42E
:104950000E94C88C9B01AC01C301B2010E948F8DE3
:1049600020E030E0A9010E94C98C20E030E040E264
:1049700051E40E949E8B5B018C012B962FAD2B97EF
:104980002F963FAD2F9763964FAD639767965FADB8
:1049900067970E947E8E181664F42B96AFAE2B9705
:1049A0002F96BFAE2F9763960FAF639767961FAF93
:1049B000679720E030E0A901B501C8010E94398B5A
:1049C00087FF04C0A12CB12C00E010E022E0A5017B
:1049D000B801CE0180960E94324DBE01605E7F4FCD
:1049E000CE0101960E94C04D6EE079E0CE010196A5
:1049F0000E94FC48BC018FE790E10E94E94CCE0187
:104A000001960E94FE4CCE0180960E94FE4C6FE7FC
:104A100070E1CE0101960E94C04D4AE050E060E096
:104A200070E0CE0101960E94BC6CCE0101960E94FE
:104A3000FE4C0E9412514090D40B5090D50B6090C8
:104A4000D60B7090D70B930182010C591F4F2F4F3B
:104A50003F4F061717072807390710F40C94A134A5
:104A60000E9412510E943D8B4B015C01C301B201B7
:104A70000E943F8B20E030E048EC51E40E94C98C5A
:104A80009B01AC01C501B4010E94398B87FF02C0B4
:104A90000C94A1346CE370E080E090E00E94DA5066
:104AA0009FEFC91AD90AE90AF90A6C962CAD3DADF7
:104AB0004EAD5FAD6C972C153D054E055F050CF0B6
:104AC000FCCE64E670E080E090E00E94DA500E9444
:104AD000586C64E670E080E090E00E94DA5063E198
:104AE00079E08FE790E10E94D44C6FE770E1CE014E
:104AF00001960E94C04D44E150E060E070E0CE01BC
:104B000001960E94ED6DCE0101960E94FE4C22E0BE
:104B10002B964FAD2B972F965FAD2F9763966FAD6A
:104B2000639767967FAD6797CE0180960E94324D5E
:104B3000BE01605E7F4FCE0101960E94C04D6EE0C7
:104B400079E0CE0101960E94FC48BC018FE790E11C
:104B50000E94E94CCE0101960E94FE4CCE01809647
:104B60000E94FE4C6FE770E1CE0101960E94C04D9D
:104B700042E350E06FEF7FEFCE0101960E94BC6CE4
:104B8000CE0101960E94FE4C0E94AE6C62E370E082
:104B900080E090E00E94DA506BE179E0CE0101966E
:104BA0000E94C84D6FE770E1CE0101960E94134943
:104BB0006FE179E00E94FC4865E870E10E941349CA
:104BC000BC0185E890E10E94E94C0C94733480911B
:104BD00072049091730499270E946B5EBC01990F37
:104BE000880B990B0E943F8B2DE038E643E55BE391
:104BF0000E949E8B6B017C0120919E0430919F044A
:104C00004091A0045091A1040E94398B18164CF0D9
:104C10006091860470918704809188049091890442
:104C20001BC02091B2043091B3044091B404509160
:104C3000B504C701B6010E947E8E87FF05C0C7017B
:104C4000B6010E94F36308C060919A0470919B04BE
:104C500080919C0490919D0420E030E048EC52E467
:104C60000E949E8B20E030E048EA51E40E949E8B37
:104C70002091290230912A0240912B0250912C025E
:104C80000E948F8D6B017C0168E274E08FE790E1F8
:104C90000E9438496FE770E1CE0101960E94C04D35
:104CA00042E350E060E070E0CE0101960E94ED6DBD
:104CB000CE0101960E94FE4C22E0B701A601CE0172
:104CC00001960E94324D69E279E0CE0180960E9401
:104CD000C84DBE016F5F7F4FCE0180960E94134981
:104CE00063E279E00E94FC48BC0185E890E10E9403
:104CF000E94CCE0180960E94FE4CCE0101960E94A6
:104D0000FE4C65E870E1CE0101960E94C04D42E381
:104D100050E06FEF7FEFCE0101960E94BC6CCE0198
:104D200001960E94FE4C8091820C882311F40C9411
:104D3000773460E273E080E090E0D7C20E94586C64
:104D40006CE574E085E890E10E94384965E870E11F
:104D5000CE0101960E94C04D4AE050E060E070E054
:104D6000CE0101960E94ED6DCE0101960E94FE4C8F
:104D700063E574E08FE790E10E9438496FE770E1E6
:104D8000CE0101960E94C04D44E150E06FEF7FEFED
:104D9000CE0101960E94BC6CCE0101960E94FE4C91
:104DA00080914C0C90914D0C8430910549F40E94F7
:104DB000235881111AC010924D0C10924C0C15C042
:104DC000892B99F40E942358882339F084E090E0DD
:104DD00090934D0C80934C0C08C00E942358811175
:104DE000F5CF0E9423588111F1CF80914C0C909106
:104DF0004D0C049741F167E474E085E890E10E946E
:104E0000384965E870E1CE0101960E94C04D4AE044
:104E100050E060E070E0CE0101960E94ED6DCE01A1
:104E200001960E94FE4C65E870E1CE0101960E9459
:104E3000C04D64E07BE0CE0101960E94FC486FE724
:104E400070E10C94AE318AE090E00E94135C6B013B
:104E50007C0120E030E0A9010E94398B181634F063
:104E60008AE090E00E94135C6B017C010BE010E093
:104E700020E030E041EE53E4C701B6010E94398BD7
:104E8000181684F420E030E0A901C701B6010E94A1
:104E9000398B1816BCF069E374E085E890E10E9454
:104EA000384941C00150110969F368EC70E080E0B5
:104EB00090E00E94DA5083E090E00E94135C6B0166
:104EC0007C01D6CF20E030E048EC52E4C701B601C7
:104ED0000E94398B87FF02C021E001C020E0B701AA
:104EE000A601CE0101960E94324D68E279E0CE0122
:104EF00080960E94C84DBE016F5F7F4FCE018096A5
:104F00000E9413496DE279E00E94FC48BC0185E8EB
:104F100090E10E94E94CCE0180960E94FE4CCE01A9
:104F200001960E94FE4C65E870E1CE0101960E9458
:104F3000C04D42E350E06FEF7FEFCE0101960E943B
:104F4000BC6CCE0101960E94FE4C60E374E08FE7DA
:104F500090E10E9438496FE770E1CE0101960E940E
:104F6000C04D42E350E060E070E0CE0101960E9447
:104F7000ED6DD5CE0E9412512B013C0180E69EE0E2
:104F80000E94D94F64E670E080E090E00E94DA5021
:104F900040E855E260E070E080E69EE00E94F67B2B
:104FA00064E670E080E090E00E94DA506FE874E020
:104FB0008FE790E10E9438496FE770E1CE010196DA
:104FC0000E94C04D42E350E06FEF7FEFCE010196AB
:104FD0000E94ED6DCE0101960E94FE4C64E874E0E3
:104FE0008FE790E10E9438496FE770E1CE010196AA
:104FF0000E94C04D42E350E06FEF7FEFCE0101967B
:105000000E94BC6CCE0101960E94FE4C80914C0C1B
:1050100090914D0C8D7F2B961FAE2B97C12CD12CD0
:10502000E12CF12C00E010E0019709F477C09E011B
:10503000205E3F4F28963FAF2EAF2897AE01425ECD
:105040005F4F2A965FAF4EAF2A970E941251DC0144
:10505000CB0184199509A609B709883B9B40A10596
:10506000B10508F05BC080E69EE00E94D449892B20
:1050700009F44DC08CED95E0A0E0B0E08093640EA3
:105080009093650EA093660EB093670E0E94D8644D
:1050900097FD06C082349105C9F780E090E002C018
:1050A0008FEF9FEF892B99F5DE0111964D015D0180
:1050B0000E94D86497FF06C089818D3441F520E0B5
:1050C00030E00BC0D5018D935D0128962EAD3FAD2C
:1050D0002897A217B30761F7EFCFD4018D914D0147
:1050E000280F311D2A964EAD5FAD2A97A417B5073C
:1050F000A1F72E5B3F4F8E8D90E0982F88274F8D24
:10510000840F911D2817390711F40C94A53462E31C
:1051100070E080E090E00E94DA5097CF0E94125138
:10512000DC01CB0184199509A609B709883B9B408E
:10513000A105B10528F42B962FAD2B972111C7C0DF
:105140000E94586C6FE770E1CE0180960E94C04DBE
:1051500042E350E066E070E0CE0180960E94ED6D83
:10516000CE0180960E94FE4C2B963FAD2B973323A9
:1051700011F40C94C03482E090E090934D0C809335
:105180004C0C4AE0B601CE0180960E948D4D4AE05B
:10519000B701CE018E960E948D4D4AE0B801CE0136
:1051A000CA960E948D4DBE01665C7F4FCE01C496AB
:1051B0000E94C04D63EE77E0CE01C4960E94FC4889
:1051C000BE01625D7F4F0E94134963EE77E00E944B
:1051D000FC48BE01605E7F4F0E941349BC0185E818
:1051E00090E10E94E94CCE01C4960E94FE4CCE0193
:1051F000CA960E94FE4CCE018E960E94FE4CCE01B5
:1052000080960E94FE4C65E870E1CE0180960E9477
:10521000C04D4AE050E06FEF7FEFCE0180960E94D4
:10522000BC6CCE0180960E94FE4C61E379E08BE875
:1052300091E10E94E24E67E379E085E890E10E9407
:10524000D44C4AE0B601CE0180960E948D4D4AE0D2
:10525000B701CE018E960E948D4D4AE0B801CE0175
:10526000CA960E948D4DBE01665C7F4FCE01C496EA
:105270000E94C04D64E07BE0CE01C4960E94FC48D1
:10528000BE01625D7F4F0E94134964E07BE00E9493
:10529000FC48BE01605E7F4F0E94134961E379E0E4
:1052A0000E94FC48BC0185E890E10E943249CE0191
:1052B000C4960E94FE4CCE01CA960E94FE4CCE01BE
:1052C0008E960E94FE4CCE0180960E94FE4C62E3B8
:1052D00070E080E090E00E94DA5080E69EE00E945C
:1052E000D94F62E370E080E090E00E94DA500C94C5
:1052F000773400917404109175046BE974E08FE7C2
:1053000090E10E9438490E94586C6FE770E1CE012D
:1053100001960E94C04D4AE050E06FEF7FEFCE0152
:1053200001960E94ED6DCE0101960E94FE4CC801CF
:105330000E94695F62966CAF7DAF8EAF9FAF629740
:105340008090310290903202A0903302B0903402EB
:10535000A501940160912D0270912E0280912F027F
:10536000909130020E94C88C2B013C0120E030E07B
:10537000A9010E94398B882309F45BC0C0903902CF
:10538000D0903A02E0903B02F0903C0220E030E006
:10539000A901C701B6010E94398B18160CF049C04B
:1053A0008091350290913602A0913702B091380277
:1053B0002E968CAF9DAFAEAFBFAF2E979C01AD01C7
:1053C000C701B6010E94398B882399F1A701960184
:1053D0002E966CAD7DAD8EAD9FAD2E970E948F8DBC
:1053E0000E94CA8E2E966CAF7DAF8EAF9FAF2E9768
:1053F000A501940162966CAD7DAD8EAD9FAD6297B7
:105400000E94C88CA30192010E948F8D2E962CAD14
:105410003DAD4EAD5FAD2E970E949E8B0E94FC8DE0
:105420009B01AC01C701B6010E949E8B6B017C0100
:1054300003C0C12CD12C76016FE770E1CE0101963B
:105440000E94C04D4AE050E060E070E0CE0101965D
:105450000E94ED6DCE0101960E94FE4C20E030E6E8
:105460004AEE56E4C701B6010E947E8E18163CF43F
:1054700067E479E085E890E10E94D44C25C021E002
:10548000B701A601CE0180960E94324D66E579E013
:10549000CE0101960E94C84DBE01605E7F4FCE01D5
:1054A00001960E9413496AE579E00E94FC48BC011C
:1054B00085E890E10E94E94CCE0101960E94FE4CE5
:1054C000CE0180960E94FE4C65E870E1CE01019607
:1054D0000E94C04D4AE050E06FEF7FEFCE01019691
:1054E0000E94BC6CCE0101960E94FE4C64E670E006
:1054F00080E090E00E94DA5016CC00917E0410917A
:105500007F040E94586CC8010E946B5E8C0162E3AC
:1055100070E080E090E00E94DA50B801110F880B33
:10552000990B0E943F8B20E030E040EA50E40E945B
:105530009E8B20E030EC4FE754E40E948F8DAB014E
:10554000BC0123E0CE0101960E94324D6CE179E06E
:10555000CE0180960E94C84DBE016F5F7F4FCE0185
:1055600080960E9413496BE276E00E94FC48BC01E1
:1055700085E890E10E94E94CCE0180960E94FE4CA5
:10558000CE0101960E94FE4C6EE579E08FE790E136
:105590000E94D44C6FE770E1CE0101960E94C04D8D
:1055A0004AE050E068E070E0CE0101960E94ED6DA7
:1055B000CE0101960E94FE4C65E870E1CE01019695
:1055C0000E94C04D4AE050E06FEF7FEFCE010196A0
:1055D0000E94BC6CCE0101960E94FE4C6FE770E108
:1055E00085E890E10E9432499ECB9091020C81E0C7
:1055F00089278093020C8091820C882331F065E822
:1056000070E183EC9DE00E94D24E68EC70E080E097
:1056100090E06BCE1092820C0C94773481E08093F2
:10562000820C61E970E187E990E10E94E94C809188
:105630004A0C90914B0C9093DD0B8093DC0B0C94F7
:1056400077340E948B6E0C94773480E69EE00E9443
:10565000D94F40E052EC61E070E080E69EE00E94AD
:10566000F67B8CED95E0A0E0B0E08093640E909323
:10567000650EA093660EB093670E64E670E080E05E
:1056800090E00E94DA5066E679E085E890E10E94B9
:10569000D44C65E870E1CE0101960E94C04DCE0168
:1056A00001960E94BD70CE0101960E94FE4C62E3FD
:1056B00070E080E090E00E94DA5065E870E1CE0191
:1056C00001960E94C04D42E350E06FEF7FEFCE01A4
:1056D00001960E94ED6DCE0101960E94FE4C62E79C
:1056E00079E08FE790E10E94D44C6FE770E1CE0142
:1056F00001960E94C04D44E150E06FEF7FEFCE0174
:1057000001960E94BC6CCE0101960E94FE4C8091D5
:105710004C0C90914D0C019739F484E090E00E947C
:105720008F5E6B017C0103C0C12CD12C760180916E
:105730004C0C90914D0C892B31F481E090E00E944B
:105740008F5E6B017C0120E030E040EA51E4C7014C
:10575000B6010E947E8E181664F521E0B701A601FD
:10576000CE0101960E94324D68EA77E0CE01809624
:105770000E94C84DBE016F5F7F4FCE0180960E9490
:1057800013496EE779E00E94FC48BC0185E890E18E
:105790000E94E94CCE0180960E94FE4CCE010196FB
:1057A0000E94FE4C81E090E090934D0C80934C0C55
:1057B00010C061E879E085E890E10E94D44C8091C6
:1057C0004C0C90914D0C019721F410924D0C1092BD
:1057D0004C0C65E870E1CE0101960E94C04D4AE094
:1057E00050E060E070E0CE0101960E94ED6DCE01C8
:1057F00001960E94FE4C65E870E1CE0101960E9480
:10580000C04D64E07BE0CE0101960E94FC486FE74A
:1058100070E10E941349BC0185E890E10E94E94CC7
:10582000CE0101960E94FE4C80E69EE00E94D94F78
:105830007ACA64E375E0CE0101960E94B84D4AE051
:1058400050E06FEF7FEFCE0101960E94BC6CCE015D
:1058500001960E94FE4C60917C0470917D048091C1
:105860002302909124020E941C66B4E18B2E912C9D
:10587000A12CB12CE12CF12CAFEFEA1AFA0AC501E8
:10588000B4010E94DA5060917C0470917D04809193
:105890002302909124020E941C668C01B3E0EB1657
:1058A000F10434F494E1890E911CA11CB11CE4CFE5
:1058B000EAE0EE16F1041CF4892BA1F703C000976F
:1058C00009F0F5C080912302909124028B3091055C
:1058D000C9F48091EF109091F010A091F110B09167
:1058E000F2108093A9119093AA11A093AB11B093D9
:1058F000AC118091EB109091EC10A091ED10B09153
:10590000EE101DC08631910521F30C9701F58091B1
:105910009C1190919D11A0919E11B0919F11809327
:10592000A9119093AA11A093AB11B093AC118091DF
:10593000981190919911A0919A11B0919B11809317
:10594000A5119093A611A093A711B093A81140910F
:10595000A9115091AA116091AB117091AC1121E085
:10596000CE0101960E94324D61EE78E0CE01809624
:105970000E94C84DBE016F5F7F4FCE0180960E948E
:105980001349BC0185E890E10E94E94CCE01809664
:105990000E94FE4CCE0101960E94FE4C4091A51142
:1059A0005091A6116091A7117091A81121E0CE012C
:1059B00001960E94324D6DE879E0CE0180960E94FA
:1059C000C84DBE016F5F7F4FCE0180960E94134984
:1059D000BC0185E890E10E943249CE0180960E9488
:1059E000FE4CCE0101960E94FE4C66E279E085E80D
:1059F00090E10E9424496CED7AE0CE0101960E946C
:105A0000C84D44E150E060E070E0CE0101960E9494
:105A1000ED6DCE0101960E94FE4C6091A91170912E
:105A2000AA118091AB119091AC110E94288E4AE08E
:105A3000CE0101960E948D4DBE016F5F7F4F8FE7B3
:105A400090E10E94434CCE0101960E94FE4C60E022
:105A500086E00E94A3616FE770E18BE891E10E940C
:105A6000E34D6FED8BE891E10E94DC4D63E979E055
:105A70008BE891E10E94E24E6091A5117091A61110
:105A80008091A7119091A8110E94288E4AE050E0C1
:105A90008BE891E10E94B94E66E279E08BE891E1F2
:105AA0000E94E24E64E670E080E090E01ECC8F3F02
:105AB000FFEF9F07ACF066E275E0CE0101960E9411
:105AC000B84D4AE050E060E070E0CE0101960E94DF
:105AD000ED6DCE0101960E94FE4C63E075E061C061
:105AE000029609F44AC065EF74E0CE0101960E9467
:105AF000B84D4AE050E060E070E0CE0101960E94AF
:105B0000ED6DCE0101960E94FE4C66EE74E085E8D4
:105B100090E10E9438494AE0B801CE0101960E9406
:105B20008D4DBE016F5F7F4F85E890E10E94324945
:105B3000CE0101960E94FE4C0091891010918A10AE
:105B40000B5E1F4FB80185E890E10E947C4C8823D2
:105B500009F4CDC62091851030918610809189106E
:105B600090918A1060ED74E0820F931F0E94B386BB
:105B700010938A1000938910BAC665EC74E0CE01C8
:105B800001960E94B84D4AE050E060E070E0CE011E
:105B900001960E94ED6DCE0101960E94FE4C65EAD1
:105BA00074E085E890E10E943849A1C68091100216
:105BB000882309F49CC66CED7AE0CE0101960E9420
:105BC000C84D4AE050E061E070E0CE0101960E94CD
:105BD000ED6DCE0101960E94FE4C0E94586C0E9411
:105BE0008B512B013C010E9465534B015C0160917C
:105BF00045027091460280914702909148020E94AE
:105C00003F8B9B01AC016D966FAF6D976E963FAF6A
:105C10006E976F964FAF6F97A0965FAFA0970E9459
:105C20008B510E943F8B6D962FAD6D976E963FAD59
:105C30006E976F964FAD6F97A0965FADA0970E943D
:105C40008F8D21E03EED42E45EE30E943D8F9B019B
:105C5000AC0160E070E080E89FE30E94C88C20E027
:105C60003AE24DE257E40E949E8B6B017C01C30136
:105C7000B2010E943F8B20E030E048EC52E40E94E9
:105C80008F8DAB01BC0122E0CE0101960E94324D06
:105C9000BE016F5F7F4F89E790E10E94434CCE01C8
:105CA00001960E94FE4C6BE077E089E790E10E944C
:105CB000244969E770E18FE790E10E94E94C67E0D1
:105CC00077E0CE0101960E94C84D69E770E1CE01F0
:105CD00001960E941349BC0189E790E10E94E94CBA
:105CE000CE0101960E94FE4C61EE78E085E890E1DD
:105CF0000E94D44C21E0B501A401CE0101960E947E
:105D0000324DBE016F5F7F4F85E890E10E943249BE
:105D1000CE0101960E94FE4C66E979E085E890E1AB
:105D20000E94244921E0B701A601CE0180960E947D
:105D3000324DBE01605E7F4FCE0101960E94C04D84
:105D400061E179E0CE0101960E94FC48BC0185E842
:105D500090E10E943249CE0101960E94FE4CCE0194
:105D600080960E94FE4C69E770E1CE0101960E9488
:105D7000C04D64E07BE0CE0101960E94FC4865E8DE
:105D800070E10E941349BC0185E890E10E94E94C52
:105D9000CE0101960E94FE4C6FE770E1CE010196A4
:105DA0000E94C04D4AE050E060E070E0CE010196F4
:105DB0000E94ED6DCE0101960E94FE4C21E0B501DE
:105DC000A401CE0101960E94324DBE016F5F7F4F4C
:105DD0008BE890E10E94434CCE0101960E94FE4C5C
:105DE0006BE870E1CE0101960E94C04D4AE050E0A0
:105DF0006FEF7FEFCE0101960E94BC6CCE01019641
:105E00000E94FE4C63E979E0CE0101960E94C84DE4
:105E1000CE0101960E947C6CCE0101960E94FE4C40
:105E200021E0B701A601CE0180960E94324DBE014D
:105E3000605E7F4FCE0101960E94C04D61E179E026
:105E4000CE0101960E94FC48BC018BE890E10E94C3
:105E5000E94CCE0101960E94FE4CCE0180960E9434
:105E6000FE4C6BE870E1CE0101960E94C04D4AE005
:105E700050E068EF7FEFCE0101960E94BC6CCE012E
:105E800001960E94FE4C8091820C882309F42FC554
:105E900068E572E080E090E028CA8091820C882357
:105EA00031F0A2E04A2E512C612C712C05C0FEE18C
:105EB0004F2E512C612C712C62E475E085E890E145
:105EC0000E94384965E870E1CE0101960E94C04DFC
:105ED0004AE050E06FEF7FEFCE0101960E94BC6C6C
:105EE000CE0101960E94FE4C812C912C5401C12CB4
:105EF000D12C760183E20E94886187E090E00E94C5
:105F000084610E94276166E970E080E090E00E9471
:105F1000DA5083E20E94886180E290E00E9484610E
:105F20000E94276166E970E080E090E00E94DA500C
:105F300062E070E083E290E00E94AE6540E050E0F5
:105F4000BA018091770D90E02091780D821B910924
:105F5000181619062CF58AE99FE06F964FAF6F97D8
:105F6000A0965FAFA0976D966FAF6D976E967FAF5F
:105F70006E970E943B596F964FAD6F97A0965FAD9D
:105F8000A0976D966FAD6D976E967FAD6E97762FDD
:105F9000652F542F4427480F511D611D711DD1CF0E
:105FA000CB01BA010E943F8B2AE939E949E95FE355
:105FB0000E948F8D0E94288EAB01BC01C416D506AD
:105FC000E606F70614F46A017B012AE0CE0180960A
:105FD0000E94614DBE01605E7F4FCE0101960E941E
:105FE000C04D6CE979E0CE0101960E94FC48BC01ED
:105FF0008FE790E10E94E94CCE0101960E94FE4C91
:10600000CE0180960E94FE4C6FE770E1CE010196B2
:106010000E94C04D4EE150E060E070E0CE0101967C
:106020000E943B6DCE0101960E94FE4C3FEF831A09
:10603000930AA30AB30A481459046A047B040CF0B7
:1060400059CF2AE0B701A601CE0180960E94614D8A
:10605000BE01605E7F4FCE0101960E94C04D6CE98B
:1060600079E0CE0101960E94FC48BC018FE790E1E7
:106070000E94E94CCE0101960E94FE4CCE01809612
:106080000E94FE4C6FE770E1CE0101960E94C04D68
:106090004AE050E060E070E0CE0101960E94ED6DB4
:1060A000CE0101960E94FE4C2AE0B701A601CE0166
:1060B00001960E94614D60EA79E0CE0180960E94CF
:1060C000C84DBE016F5F7F4FCE0180960E9413497D
:1060D00063EA79E00E94FC4865E870E10E94134998
:1060E000BC0185E890E10E94E94CCE0180960E94B7
:1060F000FE4CCE0101960E94FE4CF3C800917A043A
:1061000010917B0481E080935A0264E670E080E0A5
:1061100090E00E94DA500E94586CC8010E946B5EA9
:1061200060E074E0681B790B4AE0CE0101960E94A2
:106130008D4D68EA79E0CE0180960E94C84DBE017F
:106140006F5F7F4FCE0180960E941349BC0185E8A6
:1061500090E10E94E94CCE0180960E94FE4CCE0157
:1061600001960E94FE4C60E086E00E94A36162E519
:1061700075E0CE0101960E94B84D42E350E068E020
:1061800070E0CE0101960E94ED6DCE0101960E9455
:10619000FE4C65E870E1CE0101960E94C04D42E3DD
:1061A00050E06FEF7FEFCE0101960E94BC6CCE01F4
:1061B00001960E94FE4C6FEA79E0C8C08091780495
:1061C000909179040E946B5E8C019093DF0B809319
:1061D000DE0B62E370E080E090E00E94DA504AE07B
:1061E000B801CE0101960E948D4DBE016F5F7F4FB9
:1061F00085E890E10E94434CCE0101960E94FE4C3E
:106200008091E9109091EA10892B09F45EC065EE47
:1062100070E1CE0180960E94C04DBE01605E7F4F4E
:10622000CE0101960E94C04D44E150E060E070E074
:10623000CE0101960E94ED6DCE0101960E94FE4CAA
:1062400069EB79E0CE0101960E94C84D65E870E1E6
:10625000CE0101960E941349BC018FE790E10E9494
:10626000E94CCE0101960E94FE4C6FE770E1CE0131
:1062700001960E94C04D44E150E06FEF7FEFCE01E8
:1062800001960E94BC6CCE0101960E94FE4CBE019C
:10629000605E7F4FCE0101960E94C04D64E07BE0BE
:1062A000CE0101960E94FC486FE770E10E941349FD
:1062B000BC0185E890E10E94E94CCE0101960E9464
:1062C000FE4CCE0180960C94912664EC79E08FE729
:1062D00090E10E94D44C6FE770E1CE0101960E94DC
:1062E000C04D44E150E060E070E0CE0101960E94B4
:1062F000ED6DCE0101960E94FE4C68EA79E0CE0178
:1063000001960E94C84D65E870E1CE0101960E9499
:106310001349BC018FE790E10E94E94CCE01019640
:106320000E94FE4C6FE770E1CE0101960E94C04DC5
:1063300044E150E06FEF7FEFCE0101960E94BC6C0C
:10634000CE0101960E94FE4C69EB79E0CE010196E8
:106350000E94C84D65E870E1CE0101960E94134984
:10636000BC0185E890E10E94E94C0C948F26809155
:106370001002882309F4BBC28091820C882329F083
:1063800082E090E00E94E970B2C2C0900C02D0900E
:106390000D02E0900E02F0900F0220E030E040E4A9
:1063A00050E4C701B6010E947E8E18166CF420E0FE
:1063B00030E04AE754E4C701B6010E949E8B0E9478
:1063C000288E6B017C0106C040E3C42E45E7D42E25
:1063D000E12CF12C0E94586C60E080E00E94A361E7
:1063E00068EC79E08BE891E10E94E24E61E080E0A8
:1063F0000E94A36169ED79E08BE891E10E94E24E91
:1064000064E670E080E090E00E94DA500E94125151
:106410006093D80B7093D90B8093DA0B9093DB0BBE
:106420000E9412510091D80B1091D90B2091DA0BD8
:106430003091DB0BDC01CB01801B910BA20BB30B6A
:106440008C159D05AE05BF050CF051C283E090E0B0
:106450000E94E9700E94125164E170E080E090E0D7
:106460000E94DA50DDCF0E948F5F83EC9DE00E9496
:10647000624A3DC26BE575E08FE790E10E943849C2
:106480006FE770E1CE0101960E94C04D4AE050E0F6
:1064900060E070E0CE0101960E94ED6DCE010196A4
:1064A0000E94FE4C409176042B964FAF2B97809123
:1064B000FA0B81110DC00E9412516093F60B70937C
:1064C000F70B8093F80B9093F90B81E08093FA0B14
:1064D0008091EE0B81110DC00E9412516093EA0B66
:1064E0007093EB0B8093EC0B9093ED0B81E080931A
:1064F000EE0B1092E90B1092E80B0091E80B109153
:10650000E90B083211050CF085C02B968FAD2B9747
:106510000E949050F801EE0FFF1FE95DF24F91834A
:1065200080830E94D36220E030E040EA50E40E9481
:106530009E8B20E030E040E85AE30E949E8B6B0186
:106540007C016093E40B7093E50B8093E60B9093D2
:10655000E70B409004025090050260900602709094
:106560000702A301920160910802709109028091D3
:106570000A0290910B020E94C88C9B01AC0160E062
:1065800070E080EC90E40E94C88C4B015C0120E03C
:1065900030E0A9010E94398B20E030E040E650E471
:1065A000811105C0C701B6010E949E8B1EC0C701A4
:1065B000B6010E949E8BA30192010E94C98C20E02B
:1065C00030E040E850E40E94C88CA50194010E948C
:1065D0008F8D20E030E040EC50E40E949E8B20E064
:1065E00030E040E850E40E94C98C6093E00B709367
:1065F000E10B8093E20B9093E30B64E170E080E0A9
:1066000090E00E94DA500F5F1F4F1093E90B009348
:10661000E80B73CFC090E00BD090E10BE090E20B61
:10662000F090E30B20E030E0A901C701B6010E9421
:106630007E8E87FD1EC022E0B701A601CE01019625
:106640000E94324D61EE79E0CE0180960E94C84DE5
:10665000BE016F5F7F4FCE0180960E941349BC013F
:1066600085E890E10E94E94CCE0180960E94FE4CA4
:1066700028C165EE79E085E890E10E94D44C25C1FF
:1066800080911002882309F432C18091820C81111B
:1066900027C0C0900C02D0900D02E0900E02F09046
:1066A0000F0220E030E04AE754E4C701B6010E943F
:1066B0009E8B0E94288E4B015C0120E030E040EA76
:1066C00050E4C701B6010E949E8B20E030E040EA12
:1066D00050E40E94C98C0E94288EA501940108C034
:1066E00021E030E040E050E06AE070E080E090E0DF
:1066F0000E94F275FCC08091210D9091220D892B92
:10670000F1F581E090E09093220D8093210D64EFEC
:1067100079E0CE0101960E94C84DCE0101960E94FB
:10672000BD70CE0101960E94FE4C6DEF79E0CE0166
:1067300001960E94C84D65E871E1CE0101960E9464
:106740001349BC01CE0180960E94C04D48EC50E038
:106750006FEF7FEFCE0180960E94ED6DCE018096A7
:106760000E94FE4CCE0101960E94FE4C83EC9DE0FF
:106770000E94D94F40E052EC61E070E03BC01092C3
:10678000220D1092210D63E07AE0CE0101960E9465
:10679000C84DCE0101960E94BD70CE0101960E94A7
:1067A000FE4C61E17AE0CE0101960E94C84D65E899
:1067B00071E1CE0101960E941349BC01CE01809681
:1067C0000E94C04D48EC50E06FEF7FEFCE01809605
:1067D0000E94ED6DCE0180960E94FE4CCE01019686
:1067E0000E94FE4C83EC9DE00E94D94F40E855E2A8
:1067F00060E070E083EC9DE00E94F67B1092780CE4
:106800001092770C80E090E00E94396565E17AE0B3
:10681000CE0101960E94C84D6FE771E1CE0101964D
:106820000E941349BC01CE0180960E94C04D40EDEC
:1068300057E06FEF7FEFCE0180960E94BC6CCE01D7
:1068400080960E94FE4C4FC08091250D9091260DA0
:10685000892BA1F481E090E09093260D8093250D83
:106860008EED93E09093780C8093770C0E941265E4
:1068700068EC70E080E090E00E94DA50E0E0F0E048
:10688000199535C00E949E570E94586C0E94D95B92
:106890002EC010934B0C00934A0C64E675E085E81B
:1068A00090E10E9438496CED7AE0CE0101960E9499
:1068B000C84D4AE050E060E070E0CE0101960E94D1
:1068C000ED6DCE0101960E94FE4C65E870E1CE01AF
:1068D00001960E94C04D4AE050E06FEF7FEFCE017D
:1068E00001960E94BC6CCE0101960E94FE4C8091E4
:1068F000891090918A100097A9F0419728F4F2E04E
:106900002F1631040CF068C065E870E1CE010196E5
:106910000E94C04DCE0101960E94F06ACE01019600
:106920000E94FE4C64E670E080E090E00E94DA5045
:1069300066C06EEE78E085E890E10E9424490C94F0
:106940000F240E94AE6C0C944A250C8110E0102F8D
:1069500000278D81080F111DEE80F12CFE2CEE24F6
:106960008F81E80EF11CC884D12CDC2CCC248985C5
:10697000C80ED11C21E02B962FAF2B970C948728A3
:1069800069E774E085E890E10E94384965E870E1C4
:10699000CE0180960E94C04D4AE050E060E070E079
:1069A000CE0180960E94BC6CCE0180960E94FE4C67
:1069B00066E674E085E890E10E94384980914C0CCD
:1069C00090914D0C029711F00C94672910924D0C88
:1069D00010924C0C0C94672965E870E1CE01019689
:1069E0000E94C04D4AE050E06FEF7FEFCE0101966C
:1069F0000E94BC6CCE0101960E94FE4C85CFC15A0C
:106A0000DF4F0FB6F894DEBF0FBECDBFDF91CF9141
:106A10001F910F91FF90EF90DF90CF90BF90AF90BC
:106A20009F908F907F906F905F904F903F902F90AE
:106A300008952F923F924F925F926F927F928F9222
:106A40009F92AF92BF92CF92DF92EF92FF920F93FD
:106A50001F93CF93DF93CDB7DEB728970FB6F89487
:106A6000DEBF0FBECDBFFC018DEA9FE0938782871A
:106A70008091AA0F90E0958784878091771090E0AD
:106A8000978786878091A60F853009F0B7C38091DC
:106A9000AF0F9091B00F885891098D35910588F40A
:106AA0008091AA0F843041F48091B10F9091B20F80
:106AB0008097479708F407C28091AA0F843408F0A2
:106AC000E8C18091AA0F8A3108F448C08091AD0FC7
:106AD0009091AE0F843F914050F4118610868FEF55
:106AE0009FEFDC0184839583A683B78351C0809197
:106AF000AF0F9091B00F85974B9780F513EBE12E78
:106B00001FE0F12E82E090E040E050E0BA018C01FD
:106B10000F5F1F4F2091AA0F30E0021713076CF48C
:106B2000970122503109D9012D913C91275031090B
:106B30002730310508F40AC2C80101979595879559
:106B4000918780870C971CF41186108607C04483B8
:106B500055836683778384E090E01CC18091AA0FFF
:106B60008A3108F448C08091AD0F9091AE0F803209
:106B7000934008F4B2CF8091AF0F9091B00FC697B9
:106B8000869708F403C237C04483558366837783AE
:106B90008BE090E0FFC0D7012D913C912552310947
:106BA0002B31310508F004C2440F551F661F771FB3
:106BB00041600296B4E0EB0EF11C8C010F5F1F4F99
:106BC0002091AA0F30E00217130764F497012250B6
:106BD0003109D9012D913C912C5031092B303105CF
:106BE000D0F2C801019795958795918780870C977A
:106BF0005CF6118610868091AA0F823208F44CC090
:106C00008091AF0F9091B00F0697079708F044C09E
:106C100043EBC42E4FE0D42E82E090E040E050E001
:106C2000BA018C010F5F1F4F2091AA0F30E00217AD
:106C300013070CF5D6011297ED90FC9011979D016A
:106C4000BEE1EB1AF108A7E1EA16F10408F0BEC1B3
:106C5000440F551F661F771F4160D6012D913C914F
:106C6000B4E0CB0ED11C235031092530310510F48E
:106C70000296D7CFC8010197959587959187808710
:106C800040971CF41186108607C0448355836683A1
:106C900077838CE090E07EC07F011C821B8281E0C4
:106CA00090E09A8389838091AA0F8D3008F475C093
:106CB00029E733E0AE014D5F5F4FBE016F5F7F4F4D
:106CC000CF010E94817B892B09F067C029E733E05F
:106CD000AE014D5F5F4FBE016F5F7F4FC7010E94E6
:106CE000817B019709F059C029E733E0AE014D5F80
:106CF0005F4FBE016F5F7F4FC7010E94817B892B71
:106D000009F04BC0812C912C540100E010E08091DF
:106D1000AA0F90E029813A81281739077CF529E7E5
:106D200033E0AE014D5F5F4FBE016F5F7F4FC70124
:106D30000E94817B6C0129E733E0AE014D5F5F4F1C
:106D4000BE016F5F7F4FC7010E94817BE1E0CE16DD
:106D5000D10449F4892B09F5880C991CAA1CBB1C89
:106D6000689480F808C0CD28C1F40197B1F4880C6C
:106D7000991CAA1CBB1C0F5F1F4FC9CFD7011996C6
:106D80001C930E931897F70184829582A682B7828E
:106D900081E090E09183808329C21C821B8281E084
:106DA00090E09A838983D7011C968D919C911D97C1
:106DB000181619060CF061C01A96ED91FC911B97FC
:106DC00082E090E09A8389838281938189974E97AC
:106DD00008F053C083E090E09A8389838481958191
:106DE0000B970A9708F049C02CEB31E0AE014D5FDC
:106DF0005F4FBE016F5F7F4FC7010E94817B892B70
:106E0000E1F52CEB31E0AE014D5F5F4FBE016F5FEE
:106E10007F4FC7010E94817B019779F5412C512C4E
:106E2000320100E010E029813A81D7011C968D9152
:106E30009C911D97281739070CF010C12CEB31E0FD
:106E4000AE014D5F5F4FBE016F5F7F4FC7010E9474
:106E5000817B5C010330110509F0C6C02CEB31E0E9
:106E6000AE014D5F5F4FBE016F5F7F4FC7010E9454
:106E7000817BA816B90609F4B7C0D7011A96ED911F
:106E8000FC911B9782819381C697869708F4F2C084
:106E90003EC18091B10F9091B20F825491098E97AB
:106EA00008F00FCE20E030E0C12CD12C7601A901F2
:106EB0004D54504FDA014D915C9149505109493080
:106EC000510598F0FECD8091B30F9091B40F0997C2
:106ED000099708F0F1CD118610868FEF9FEFDC0146
:106EE00084839583A683B7838CC1B9016B54704F9B
:106EF000DB014D915C914751510942315105C0F47C
:106F0000D701C601880F991FAA1FBB1F6C017D0105
:106F10006894C0F82C5F3F4F2038310541F620E2DD
:106F200030E031872087C482D582E682F78269C14A
:106F3000DB014D915C91465051094730510508F0F5
:106F4000C0CDCC0CDD1CEE1CFF1CE4CFD7012D9175
:106F50003C91235131092F30310550F4440F551F16
:106F6000661F771F41600296B4E0EB0EF11CCFCD97
:106F7000D7012D913C912A5031092930310508F073
:106F8000EDCD440F551F661F771FEDCF8091B10FD8
:106F90009091B20FC697869708F02DCE85EBE82E1C
:106FA0008FE0F82E83E090E040E050E0BA0105CE9B
:106FB000D7012D913C912C5031092A30310508F030
:106FC0001ACE440F551F661F771FF3CDD9012D919F
:106FD0003C912C5031092B30310508F05DCE440F27
:106FE000551F661F771F39CE2CEB31E0AE014D5F88
:106FF0005F4FBE016F5F7F4FC7010E94817B6C01B5
:107000000330110579F42CEB31E0AE014D5F5F4F99
:10701000BE016F5F7F4FC7010E94817BC816D906F2
:1070200009F02BCFA114B10459F4CA94CD2809F06A
:1070300024CF440C551C661C771C689440F80BC088
:10704000AA94AB2809F019CFCD2809F016CF440C2B
:10705000551C661C771C0F5F1F4FE5CE19961C93BD
:107060000E931897F701448255826682778282E0F8
:1070700090E090CE848195814B97459708F047C06A
:10708000DF0116966F0126ECC20ED11C20E030E025
:1070900040E050E060E070E080E090E00D911C91F5
:1070A0001197095011090830110588F512960D91B4
:1070B0001C911397015111090D301105D8F401E00D
:1070C0000E94259021601496AC15BD0539F7F70193
:1070D000248335834683578300E20E9440902283B5
:1070E000338385E090E09183808380E390E0918713
:1070F00080877CC012960D911C9113970450110942
:107100000530110520F401E00E942590DCCF80912C
:10711000AA0F893340F08281938189579109833581
:10712000910508F47CC18091AA0F823209F46CC0E9
:1071300082819381895791098335910508F4E6C1CD
:10714000828193818C549109C59708F064C0809125
:10715000AA0F843031F4848195818097479708F491
:1071600034C28091AA0F843408F455C0848195817B
:1071700089549109C39708F04EC09F012A5F3F4F81
:10718000AF014A575F4F812C912C5401D9016D9169
:107190007C916950710969307105E8F5D901129641
:1071A0006D917C911397665171096131710508F0F9
:1071B00022C2D501C401880F991FAA1FBB1F4C0111
:1071C0005D01689480F82C5F3F4F24173507F1F676
:1071D00020E230E0F70131872087D7018482958251
:1071E000A682B78287E090E08D939C9381E090E047
:1071F000BFC282E08093A60F1092AA0F80E090E0B9
:10720000B7C283E090E0C6CD828193810A97099747
:1072100008F460C18DCF8091AA0F863460F182811D
:1072200093810C970B9708F4F6C125C0D9011296EB
:107230006D917C9113976E5171096731710508F05A
:107240001EC2D501C401880F991FAA1FBB1F4C0184
:107250005D01689480F84E5F5F4F2C5F3F4F45346F
:10726000510509F4F3C1D9016D917C916C507109FC
:107270006B307105D8F28091AA0F883578F1828140
:107280009381855891098B35910508F408C226C071
:10729000BC016F5F7F4FD8012D913C912750310980
:1072A0002730310508F00AC2440F551F416002968D
:1072B0000C5F1F4F2091AA0F30E024503109821734
:1072C00093070CF004C2980122503109D9012D9185
:1072D0003C912950310928303105D0F28091AA0F14
:1072E0008032E1F48281938106970697B8F4848115
:1072F00095810997099790F49F012A5F3F4FAF014D
:10730000425C5F4F812C912C5401D9016D917C918D
:10731000665071096630710508F4F3C1D7011C96F7
:107320002D903C901D97B6E02B1631040CF461CFE4
:107330008F010A5F1F4F73E0C72ED12CE5EC8E2E14
:10734000EDE99E2EECE1AE2EE1E8BE2EF801608163
:10735000718134976080718080E090E00E943D8B65
:107360006D837E838F839887B30180E090E00E94D5
:107370003D8B2B013C012DEC3CEC4CE45FE30E9487
:107380009E8B9B01AC016D817E818F8198850E94CF
:10739000398B87FD19C02DEC3CEC4CE45FE36D812B
:1073A0007E818F8198850E949E8B9B01AC01C301D9
:1073B000B2010E94398BE82F880FFF0BEE27FF0FD9
:1073C000EE1FFF27319602C0E0E0F0E0A501940136
:1073D00063E971E080E091E00E94E78F4F01FF0FC9
:1073E000AA08BB0886269726A826B926FFEFCF1A3B
:1073F000DF0A0E5F1F4FC214D30409F0A7CFD701D5
:1074000014968D929D92AD92BC92179780E290E077
:1074100019969C938E9318978FEF9FEFE5CE8481FA
:107420009581CA97899708F07ECE9F012A5F3F4FCA
:10743000812C912C540143E050E0D9016D917C9155
:107440006A5071096930710508F06DCED901129644
:107450006D917C911397665171096131710550F5F9
:10746000D501C401880F991FAA1FBB1F4C015D01E4
:10747000689480F84E5F5F4F2C5F3F4F4B33510550
:10748000E1F69F012A583F4FD9012D913C912A5096
:1074900031092930310508F046CE2CE130E0F70102
:1074A00031872087D70184829582A682B7828AE0BD
:1074B00090E09ACED90112966D917C911397665007
:1074C00071096730710508F02ECE880C991CAA1C32
:1074D000BB1CD0CF2091AA0FCF01820F911D820F2C
:1074E000911DDC0112978D919C910A97099708F0E4
:1074F0001FCEF701118610868FEF9FEFDC0184838A
:107500009583A683B78386E090E044CC8091AA0F50
:10751000813208F415CE84819581CA97899708F045
:107520000FCE9F012A5F3F4F812C912C540143E0E5
:1075300050E0D9016D917C916A50710969307105F3
:1075400008F0FECDD90112966D917C91139766518A
:1075500071096131710570F112966D917C911397EB
:10756000665071096730710508F0EACD880C991CE6
:10757000AA1CBB1C4E5F5F4F2C5F3F4F433251052F
:10758000C1F69F012A5B3F4FD9012D913C912A50B2
:1075900031092930310508F0D3CD20E130E0F70181
:1075A00031872087D70184829582A682B78286E0C0
:1075B00090E01ACED501C401880F991FAA1FBB1FE6
:1075C0004C015D01689480F8D5CF86819781099739
:1075D000099708F0C6CDD70119961C921E921897EC
:1075E0008FEF9FEFDC01F70184839583A683B78338
:1075F00087E090E0CFCBD90112966D917C911397E3
:10760000665071096730710508F005CE880C991C29
:10761000AA1CBB1CD8CD848195810997099708F0D5
:107620002ACE868197818C974F9708F024CE80854B
:10763000918589974D9708F01ECE9F01265F3F4F99
:10764000812C912C540145E050E00DCE9F0126572E
:107650003F4FD9012D913C912C5031092B303105F0
:1076600008F009CE20E230E0F70131872087D7010A
:1076700084829582A682B78288E090E0B5CDD90158
:1076800012966D917C91139769507109693071055B
:1076900008F0F1CD880C991CAA1CBB1CDCCD8481A0
:1076A0009581825491098E9708F018CE8F01045C61
:1076B0001F4F8DE190E040E050E0FCCDD8012D91CE
:1076C0003C912851310922313105C0F0CB0101979D
:1076D00095958795D70119969C938E9318978A97BD
:1076E0000CF4FCCD052E000C660B770BF7014483E0
:1076F00055836683778389E090E04CCB440F551F18
:10770000D6CDD90112966D917C911397695171096B
:1077100063317105E8F4D501C401880F991FAA1FD0
:10772000BB1F4C015D01689480F82C5F3F4F24170C
:10773000350709F0EACD2EE030E0F70131872087E8
:10774000D70184829582A682B7828FE090E04CCDEB
:10775000D90112966D917C91139769507109693026
:10776000710508F0DBCD880C991CAA1CBB1CDDCF71
:1077700028960FB6F894DEBF0FBECDBFDF91CF9134
:107780001F910F91FF90EF90DF90CF90BF90AF903F
:107790009F908F907F906F905F904F903F902F9031
:1077A00008954F925F926F927F928F929F92AF92C5
:1077B000BF92DF92EF92FF920F931F93CF93DF93CD
:1077C000CDB7DEB7A9970FB6F894DEBF0FBECDBF19
:1077D000D82E882351F080914E0C882331F06CED27
:1077E0007AE08DEF9EE00E94C24E0E94AD6260E0A2
:1077F0008DE20E94B65460E18DE20E94B65468E0CA
:107800008DE20E94B6544090FB105090FC106090A6
:10781000FD107090FE1049825A826B827C828090AB
:10782000FF1090900011A0900111B09002118D8274
:107830009E82AF82B8868091031190910411A0912D
:107840000511B09106118EA39FA3A8A7B9A7898798
:107850009A87AB87BC87DD20A1F180914E0C8823ED
:1078600081F17E019DE0E90EF11C65E579E0C7013B
:107870000E94B84DC7010E94BD70C7010E94FE4C16
:107880008E010F5F1F4FD8016D917D918D919D915C
:107890008D0146E050E00E94AC6264E07BE08DEF39
:1078A0009EE00E94E24E0E151F0569F76CED7AE02E
:1078B000C8010E94C84DC8010E94BD70C8010E9445
:1078C000FE4C23E938E144E85FE3C301B2010E94C2
:1078D0009E8B2B013C016D877E878F87988B22E4DE
:1078E00030E645E85FE3C501B4010E949E8B4B0181
:1078F0005C01698B7A8B8B8B9C8B25E83BEE41E995
:107900005FE36EA17FA188A599A50E949E8B6D8BD8
:107910007E8B8F8B988F4092FB105092FC10609260
:10792000FD107092FE108092FF1090920011A092B4
:107930000111B092021160930311709304118093AE
:10794000051190930611DD2009F4A7C080914E0C1B
:10795000882309F4A2C07E01B9E1EB0EF11C68E4B2
:1079600079E0C7010E94B84DC7010E94BD70C701F0
:107970000E94FE4C8E01035F1F4FF80161917191CF
:10798000819191918F0142E050E00E94AC6264E0ED
:107990007BE08DEF9EE00E94E24E0E151F0569F719
:1079A0006CED7AE0C8010E94C84DC8010E94BD700C
:1079B000C8010E94FE4C47E051E166E070E082E3BE
:1079C0000E944F5480900811912C982C882480910B
:1079D0000711882AA0900A11B12CBA2CAA248091F0
:1079E0000911A82AE0900C11F12CFE2CEE248091B4
:1079F0000B11E82A6BE379E08DEF9EE00E94F14DD8
:107A00004AE050E0B4018DEF9EE00E94B94E64E080
:107A10007BE08DEF9EE00E94E24E4AE050E0B5012F
:107A20008DEF9EE00E94B94E64E07BE08DEF9EE01A
:107A30000E94E24E4AE050E0B7018DEF9EE00E94C6
:107A4000B94E6CED7AE08DEF9EE00E94C24EC80107
:107A50000E94075562E379E08DEF9EE00E94F14DB0
:107A60007E01F5E2EF0EF11CD8016D917D918D91B3
:107A70009D918D014AE050E00E94AC6264E07BE0A1
:107A80008DEF9EE00E94E24E0E151F0569F76CED2A
:107A90007AE08DEF9EE00E94C24E61E08DE10E948F
:107AA000B654DD20B1F080914E0C882391F06EE148
:107AB00079E08DEF9EE00E94F14DAE014B5D5F4F8E
:107AC00061E070E08DE10E944F548DA190E00E9432
:107AD000885462E08EE10E94B65463E08FE10E9418
:107AE000B65464E080E20E94B654DD2009F450C030
:107AF00080914E0C882309F44BC062E079E08DEF51
:107B00009EE00E94F14DAE014B5D5F4F61E070E081
:107B10008EE10E944F54ADA0B12CAE014B5D5F4F82
:107B200061E070E08FE10E944F54EDA0F12CAE01B6
:107B30004B5D5F4F61E070E080E20E944F540DA109
:107B400010E04AE050E0B5018DEF9EE00E94B94E92
:107B500064E07BE08DEF9EE00E94E24E4AE050E060
:107B6000B7018DEF9EE00E94B94E64E07BE08DEF9F
:107B70009EE00E94E24E4AE050E0B8018DEF9EE0A8
:107B80000E94B94E6CED7AE08DEF9EE00E94C24EED
:107B900065E081E20E94B654DD20B1F080914E0C88
:107BA000882391F06FEE78E08DEF9EE00E94F14D1A
:107BB000AE014B5D5F4F61E070E081E20E944F5487
:107BC0008DA190E00E94885466E082E20E94B65443
:107BD000DD20B1F080914E0C882391F067ED78E0C4
:107BE0008DEF9EE00E94F14DAE014B5D5F4F61E075
:107BF00070E082E20E944F548DA190E00E94885470
:107C000067E083E20E94B654DD20B1F080914E0C13
:107C1000882391F061EC78E08DEF9EE00E94F14DB9
:107C2000AE014B5D5F4F61E070E083E20E944F5414
:107C30008DA190E00E94885468E084E20E94B654CE
:107C4000DD20B1F080914E0C882391F069EA78E054
:107C50008DEF9EE00E94F14DAE014B5D5F4F61E004
:107C600070E084E20E944F548DA190E00E948854FD
:107C700069E085E20E94B654DD20B1F080914E0C9F
:107C8000882391F06FE878E08DEF9EE00E94F14D3F
:107C9000AE014B5D5F4F61E070E085E20E944F54A2
:107CA0008DA190E00E9488546AE086E20E94B6545A
:107CB000DD20B1F080914E0C882391F069E778E0E7
:107CC0008DEF9EE00E94F14DAE014B5D5F4F61E094
:107CD00070E086E20E944F548DA190E00E9488548B
:107CE0006BE088E20E94B654DD20B1F080914E0C2A
:107CF000882391F060E678E08DEF9EE00E94F14DE0
:107D0000AE014B5D5F4F61E070E088E20E944F542E
:107D10008DA190E00E9488546CE089E20E94B654E4
:107D2000DD2009F479C080914E0C882309F474C0D9
:107D300068E478E08DEF9EE00E94F14DAE014B5D6E
:107D40005F4F61E070E089E20E944F548DA190E0A6
:107D50000E94885461E378E08DEF9EE00E94F14D2F
:107D600066E070E087E20E949C5490E00E94885494
:107D70006AE178E08DEF9EE00E94F14D65E070E0F1
:107D800087E20E949C5490E00E94885463E078E06F
:107D90008DEF9EE00E94F14D64E070E087E20E946A
:107DA0009C5490E00E9488546AEE77E08DEF9EE04C
:107DB0000E94F14D62E070E087E20E949C5490E0E6
:107DC0000E94885461ED77E08DEF9EE00E94F14DB6
:107DD00061E070E087E20E949C5490E00E94885429
:107DE00068EB77E08DEF9EE00E94F14D60E070E07F
:107DF00087E20E949C5490E00E94885467EA77E0F2
:107E00008DEF9EE00E94F14D63E070E087E20E94FA
:107E10009C5490E00E94885441E067E070E087E263
:107E20000E94C95441E063E070E087E20E94C954B7
:107E300041E063E070E08AE20E94C954DD2091F0E5
:107E400080914E0C882371F06EE877E08DEF9EE014
:107E50000E94F14D63E070E08AE20E949C5490E041
:107E60000E94885440E063E070E08AE20E94C954B6
:107E7000DD2091F080914E0C882371F064E777E06B
:107E80008DEF9EE00E94F14D63E070E08AE20E9477
:107E90009C5490E00E94885441E062E070E08AE2E5
:107EA0000E94C954DD2091F080914E0C882371F01E
:107EB00068E577E08DEF9EE00E94F14D62E070E0B2
:107EC0008AE20E949C5490E00E94885440E062E064
:107ED00070E08AE20E94C954DD2091F080914E0C3E
:107EE000882371F06BE377E08DEF9EE00E94F14D07
:107EF00062E070E08AE20E949C5490E00E94885404
:107F000041E061E070E08AE20E94C954DD2091F016
:107F100080914E0C882371F06FE177E08DEF9EE049
:107F20000E94F14D61E070E08AE20E949C5490E072
:107F30000E94885440E061E070E08AE20E94C954E7
:107F4000DD2091F080914E0C882371F062E077E0A3
:107F50008DEF9EE00E94F14D61E070E08AE20E94A8
:107F60009C5490E00E94885441E060E070E08AE216
:107F70000E94C954DD2091F080914E0C882371F04D
:107F800066EE76E08DEF9EE00E94F14D60E070E0DD
:107F90008AE20E949C5490E00E94885440E060E095
:107FA00070E08AE20E94C954DD2091F080914E0C6D
:107FB000882371F069EC76E08DEF9EE00E94F14D30
:107FC00060E070E08AE20E949C5490E00E94885435
:107FD00041E066E070E087E20E94C95441E065E05C
:107FE00070E087E20E94C95441E064E070E087E2FB
:107FF0000E94C95440E062E070E087E20E94C954E8
:1080000040E061E070E087E20E94C95440E060E037
:1080100070E087E20E94C954DD2009F475C08091A8
:108020004E0C882309F470C061EB76E08DEF9EE082
:108030000E94F14D66E070E08BE20E949C5490E05B
:108040000E94885463E976E08DEF9EE00E94F14D36
:1080500065E070E08BE20E949C5490E00E9488549E
:1080600065E776E08DEF9EE00E94F14D64E070E000
:108070008BE20E949C5490E00E9488546CE576E06C
:108080008DEF9EE00E94F14D62E070E08BE20E9475
:108090009C5490E00E94885463E476E08DEF9EE06B
:1080A0000E94F14D61E070E08BE20E949C5490E0F0
:1080B0000E9488546AE276E08DEF9EE00E94F14DC6
:1080C00060E070E08BE20E949C5490E00E94885433
:1080D00067E176E08DEF9EE00E94F14D63E070E095
:1080E0008BE20E949C5490E00E94885462E076E00B
:1080F0008DEF9EE00E94F14D64E070E08CE20E9402
:108100009C5490E00E94885440E064E070E08CE26F
:108110000E94C954AE014B5D5F4F61E070E08CE29C
:108120000E944F546DA1607F66608CE20E94B6543D
:10813000DD2009F465C080914E0C882309F460C0ED
:108140006EEE75E08DEF9EE00E94F14DAE014B5D4D
:108150005F4F61E070E08CE20E944F546DA16F7040
:1081600070E066507109072E000C880B990B0E9475
:108170003F8B9B01AC0160E070E080E090E40E94E6
:108180003D8F20E030E048EC50E40E949E8B0E943E
:10819000F95467ED75E08DEF9EE00E94F14DAE0160
:1081A0004B5D5F4F61E070E080E30E944F544DA152
:1081B00050E060E070E02AE08DEF9EE00E942A4EE1
:1081C0008DEF9EE00E94BF4E6FEB75E08DEF9EE05D
:1081D0000E94F14D61E070E080E30E949C5490E0C9
:1081E0000E94885466EA75E08DEF9EE00E94F14D92
:1081F00061E070E08FE20E949C5490E00E948854FD
:1082000041E061E070E08FE20E94C954DD2091F00E
:1082100080914E0C882371F06EE875E08DEF9EE042
:108220000E94F14D61E070E08EE20E949C5490E06B
:108230000E94885441E061E070E08EE20E94C954DF
:1082400040E067E070E081E30E94C954DD2009F45A
:1082500053C080914E0C882309F44EC06BE775E043
:108260008DEF9EE00E94F14D67E070E081E30E9497
:108270009C5490E00E9488546AE17AE08DEF9EE081
:108280000E94E24EAE014B5D5F4F61E070E080E026
:108290000E944F548DA13CD56CED7AE08DEF9EE0AD
:1082A0000E94C24E0DE110E066E47AE08DEF9EE0A0
:1082B0000E94E24E40E150E0B8018DEF9EE00E9446
:1082C000B94E68E278E08DEF9EE00E94E24EAE018A
:1082D0004B5D5F4F61E070E0802F0E944F548DA195
:1082E00017D56CED7AE08DEF9EE00E94C24E0F5FD5
:1082F0001F4F0A331105C1F6A9960FB6F894DEBFD9
:108300000FBECDBFDF91CF911F910F91FF90EF90E6
:10831000DF90BF90AF909F908F907F906F905F9015
:108320004F900895DC0180E0615090F09D91982776
:10833000E92FEF70F0E0ED59F64F249192959F7080
:10834000E92FF0E0ED58F64FE4918E2F8227ECCF25
:10835000089585ED8093BC008091BC0084FDFCCF26
:1083600010929F0D08950895E091780D8091770DFA
:10837000E81730F4F0E0E557F34F808190E008957E
:108380008FEF9FEF0895862F642F0C942550862F32
:10839000642F0C945450DF92EF92FF920F931F932F
:1083A000CF93DF937C018B01D42EDC011696ED91E7
:1083B000FC911797138615861486DF011B9633965A
:1083C0001E92AE17BF07E1F7C0E0B801D7011696BD
:1083D0008D919C9117970E943456D82F811102C01D
:1083E000D0E00DC0CD1107C067E0C8019BDFF801E8
:1083F0009781891721F0CF5FDC1690F3E6CF8D2FA0
:10840000DF91CF911F910F91FF90EF90DF90089532
:10841000FC0190810180F281E02DF8948181892B0B
:1084200081832281892F809528232283A7E0B0E0D1
:108430001197F1F7218182238183A3E2B0E01197A4
:10844000F1F780817894EFECF0E03197F1F7982321
:1084500081E009F480E00895FC0190810180F281BF
:10846000E02D892F809560FF12C0F894228182232D
:1084700082838181892B8183A3E2B0E01197F1F798
:108480008281982B9283789487ED90E011C0F894C4
:108490002281822382838181892B8183AFEFB0E0A7
:1084A0001197F1F78281982B928378948FE090E076
:1084B0000197F1F70895CF92DF92EF92FF920F9319
:1084C0001F93CF93DF931F92CDB7DEB76C01E62EDB
:1084D00008E010E0FF24F39461E08F2D8E2109F471
:1084E00060E0C6014983B8DFFF0C015011094981E2
:1084F0000115110589F7411115C0F894D60111969F
:10850000ED91FC91129791818C91809589238183C3
:108510001196ED91FC91129792818C91809589230F
:10852000828378940F90DF91CF911F910F91FF90EC
:10853000EF90DF90CF900895CF92DF92EF92FF926D
:108540000F931F93CF93DF931F92CDB7DEB78C01AC
:10855000F62E40E065E57983AEDFCF2C7981D72E0A
:10856000760188E0E80EF11CF60161916F0140E0B0
:10857000C801A1DFCE14DF04B9F70F90DF91CF91CE
:108580001F910F91FF90EF90DF90CF900895FC0125
:1085900090810180F281E02DF8948181292F20952E
:1085A0008223818378948DE743E050E0815021F16C
:1085B000DA011197F1F730813923C1F3F894828100
:1085C000822382838181892B81837894ABE7B7E012
:1085D0001197F1F7F894818128232183A3E1B1E079
:1085E0001197F1F78081982381E009F080E0789479
:1085F000E3E6F6E03197F1F708958F929F92AF92FC
:10860000BF92CF92DF92EF92FF920F931F93CF937F
:10861000DF93EC018E819F81BADF40E06CEC8E81AC
:108620009F8149DF488164E48E819F8144DF8A8194
:10863000882309F441C0E981E950E33040F4F0E0D7
:10864000EE0FFF1FEA51FB4F0081118102C00EEEB9
:1086500012E08B818823F1F0888181111BC00E9478
:1086600012514B015C016801110FEE08FF088E8169
:108670009F81CEDE813001F10E941251DC01CB01DD
:108680008C199D09AE09BF0988159905AA05BB0576
:1086900070F312C0B801110F880B990BDF91CF91C5
:1086A0001F910F91FF90EF90DF90CF90BF90AF9010
:1086B0009F908F900C94DA50DF91CF911F910F9182
:1086C000FF90EF90DF90CF90BF90AF909F908F90F2
:1086D00008954F925F926F927F928F929F92AF9286
:1086E000BF92CF92DF92EF92FF920F931F93CF939F
:1086F000DF931F921F92CDB7DEB72C018A01FC01D8
:108700008681978169837A8342DF69817A818823B0
:10871000A1F1F201868197810FDF40E06EEBF2015B
:1087200086819781C8DE78014801F9E08F0E911C9F
:10873000F2016680778088E0A82EB12CCC24C39407
:10874000D12CC30165DE8111DC28CC0CF1E0AF1A1D
:10875000B108B9F7F701D1927F01E815F90541F7A2
:10876000F2018681978113DF813039F468E0C80116
:10877000D9DD91E0F8012085821390E0892F0F90D8
:108780000F90DF91CF911F910F91FF90EF90DF90AD
:10879000CF90BF90AF909F908F907F906F905F90A1
:1087A0004F900895CF93DF93CDB7DEB729970FB6DB
:1087B000F894DEBF0FBECDBFAE014F5F5F4F89DFC4
:1087C000882389F08D818F3361F020F48F3159F443
:1087D00089E00CC08F3519F08F3739F004C08BE079
:1087E00005C08AE003C080E001C08CE029960FB686
:1087F000F894DEBF0FBECDBFDF91CF9108950F93E8
:108800001F93CF93DF93CDB7DEB761970FB6F89480
:10881000DEBF0FBECDBF8C01462FBE01665F7F4F0E
:10882000BADD811105C060E070E08EEF92EC4AC0C5
:10883000AE014F5F5F4FBE01665F7F4FC80149DFEA
:10884000882359F1698148E0649FB00111248A812D
:10885000282F30E0322F2227330F330F330F262BF0
:10886000372B8A858031E1F4688570E08F81AB0118
:10887000481B5109CA019695982F88279795879587
:108880000E940A9060517109207F53E0220F331F2C
:108890005A95E1F7620F731F04C060E874EE01C0DF
:1088A000B901613854EE75070CF4BDCF072E000CEA
:1088B000880B990B0E943F8B20E030E040E05CE3A6
:1088C0000E949E8B61960FB6F894DEBF0FBECDBF9F
:1088D000DF91CF911F910F910895EF92FF920F9327
:1088E0001F93CF93DF93CDB7DEB728970FB6F894D9
:1088F000DEBF0FBECDBF8C01DC011696ED91FC9161
:108900001797138615861486DF011B9633961E92E1
:10891000AE17BF07E1F7F80114821582EE24E39445
:10892000BE016F5F7F4FF801868197810E943456A8
:10893000882309F469C067E0CE010196F3DC9885CD
:108940008913EECFD8018C91811121C016968D919B
:108950009C9117971CDEBE016F5F7F4FF8018681E7
:108960009781EADD40E064EBD80116968D919C91E9
:108970001797A1DDF801868197814ADDF82ED8018D
:1089800016968D919C91179702DEFF20B1F1F801A8
:10899000F18089818031A1F1BE016F5F7F4FC801F5
:1089A00001DF8F1520F4D80111968C910AC08981BE
:1089B000803111F48CE005C0BE016F5F7F4FC801AC
:1089C000F1DEF801818384818F5F8483898188321D
:1089D00061F030F4803149F0823209F0A1CF05C056
:1089E0008B3319F0823409F09BCFD80115968C9106
:1089F00015978F5F15968C9393CFD801EC92C7CFC4
:108A0000BCE0BF1580F2D6CF28960FB6F894DEBF33
:108A10000FBECDBFDF91CF911F910F91FF90EF90CF
:108A200008950F931F93CF93DF93EC01162F60E00F
:108A3000812F0E945450612F70E0FB01EB52F54FE3
:108A4000E491E883FB01E157F54FE491F0E0EE0F8C
:108A5000FF1FEB58F54F859194919A8389831B866C
:108A60001D861C86FE013B968E010D5F1F4F1292E4
:108A7000E017F107E1F7DF91CF911F910F91089572
:108A80000F931F93CF93DF931F92CDB7DEB78C0167
:108A9000FC01848169830E948861F8018385698172
:108AA000862B90E00E9484610F90DF91CF911F91FF
:108AB0000F910C9427610F931F93CF938C01C62FB6
:108AC000DFDF6C2F6460C801DBDF6C2F6B7FC801B8
:108AD000D7DF83EC90E00197F1F7CF911F910F91D1
:108AE00008950F931F93CF938C01C62F607F616011
:108AF000E2DF80E1C89FB00111246160C801DBDFC3
:108B000081E090E0CF911F910F9108951F920F92F5
:108B10000FB60F9211240BB60F922F933F934F93E2
:108B20005F936F937F938F939F93AF93BF93EF93D5
:108B3000FF938091A70F0E94FB4F2091AB0F3091C4
:108B4000AC0F2F5F3F4F3093AC0F2093AB0F909142
:108B5000AA0F953618F096E09093A60F9091A60F65
:108B60009430C9F128F4923069F09330D1F05EC0AE
:108B7000953009F451C0963009F058C091E09093B7
:108B8000771051C0811152C02091AB0F3091AC0FC2
:108B90002436310508F442C0109277101092AA0FC3
:108BA0001CC0813009F042C0E091AA0F91E09E0FF5
:108BB0009093AA0FF0E02091AB0F3091AC0FEE0F25
:108BC000FF1FEA55F04F308727831092AC0F1092A9
:108BD000AB0F94E029C0811117C0E091AA0F91E07A
:108BE0009E0F9093AA0FF0E02091AB0F3091AC0F45
:108BF000EE0FFF1FEA55F04F308727831092AC0F1E
:108C00001092AB0F93E010C02091AB0F3091AC0FDE
:108C10002536310558F007C0811108C01092AC0FFD
:108C20001092AB0F03C095E09093A60F9091A90FFF
:108C30009923B9F081110AC08091A80F882321F0EF
:108C40008091A80F61E009C02F9A0BC08091A80FF6
:108C5000882331F08091A80F60E00E94255001C068
:108C60002F98FF91EF91BF91AF919F918F917F913D
:108C70006F915F914F913F912F910F900BBE0F908D
:108C80000FBE0F901F901895CF92DF92EF92FF9238
:108C9000CF93DF93EC01072E000C880B990B0E94F9
:108CA0003F8B6B017C0120E030E040E45FE30E94F9
:108CB0009E8B20E030E048E452E40E948F8D0E94B9
:108CC000288EC617D707D4F020E030E040EA5FE3F3
:108CD000C701B6010E949E8B20E030E048E452E4D8
:108CE0000E948F8D20E030E040E85FE30E94C98C55
:108CF0000E94288E21E06C177D070CF420E0822F63
:108D000090E0DF91CF91FF90EF90DF90CF900895AA
:108D10000F931F93CF93DF93082F6FE779E08DEFC9
:108D20009EE00E94E24EC7E0D0E010E0B8010C2EB9
:108D300002C0759567950A94E2F76170772742E063
:108D400050E08DEF9EE00E94B94E219778F7DF91B9
:108D5000CF911F910F9108951F920F920FB60F920E
:108D600011240BB60F922F933F934F935F936F9302
:108D70007F938F939F93AF93BF93EF93FF938091D4
:108D8000B900887F803609F49CC068F5883209F400
:108D90005BC090F4803109F454C038F4882309F49E
:108DA000F6C0883009F44DC0F5C0883109F44CC0D4
:108DB000803209F45DC0EEC0803409F468C048F424
:108DC000803309F455C0883309F0E4C080939D0DC9
:108DD000D8C0803509F44FC0883509F45DC08834A7
:108DE00009F0D8C0D6C0883909F4C7C0A8F48837BC
:108DF00009F467C038F4883609F463C0803709F491
:108E000060C0C8C0883809F4B8C0803909F45FC0B0
:108E1000803809F0BFC05BC0803B09F486C038F4DD
:108E2000803A09F466C0883A09F47FC0B3C0803C38
:108E300009F4A7C0883C09F4A4C0883B09F48AC09F
:108E4000A9C080917A0D10C090919C0D80919B0DCE
:108E5000981770F5E0919C0D81E08E0F80939C0D2A
:108E6000F0E0E558F24F80818093BB0085EC86C02E
:108E700080939D0D8EC0E0919C0D81E08E0F8093BC
:108E80009C0D8091BB00F0E0E558F24F80839091FB
:108E90009C0D80919B0D6EC0E0919C0D81E08E0F2A
:108EA00080939C0D8091BB00F0E0E558F24F8083E9
:108EB00080919E0D81116DC081E08093790D84EACF
:108EC00061C083E080939F0D1092490CCFCF8091B9
:108ED000490C803208F051C0E091490C81E08E0FBE
:108EE0008093490C8091BB00F0E0E75DF34F8083F5
:108EF000BDCF85EC8093BC0010929F0D8091490CF2
:108F0000803230F4E091490CF0E0E75DF34F1082DD
:108F10006091490C70E0E091270CF091280C89E2F7
:108F20009CE019951092490C35C084E080939F0D08
:108F30001092260C1092250CE091230CF091240C39
:108F400019958091250C811105C081E08093250C35
:108F50001092030CE091260C81E08E0F8093260C7A
:108F6000F0E0ED5FF34F80818093BB009091260C81
:108F70008091250C981708F479CF85E88093BC0080
:108F800009C085EC8093BC0010929F0D03C0109225
:108F90009D0DDFD9FF91EF91BF91AF919F918F917F
:108FA0007F916F915F914F913F912F910F900BBEE9
:108FB0000F900FBE0F901F9018954091250C262FF3
:108FC00030E0240F311D21323105DCF420919F0D5A
:108FD0002430C9F4FC0180E090E0861758F4309109
:108FE000250C2191DC01AD5FB34FA30FB11D2C9374
:108FF0000196F3CF8091250C680F6093250C80E0DB
:10900000089581E0089582E008950E946D92809114
:109010007F1090918010009711F00C948A8660E088
:1090200070E0CB010895AF92BF92CF92DF92EF92A2
:10903000FF920F931F93CF93DF932091A110309154
:10904000A210FC01448155818901041B150B4115B7
:10905000510559F12115310541F12417350728F142
:109060000217130718F08901015011097C01A09023
:109070009D10B0909E10C501DFEFCFEF6501C00ECF
:10908000D11EC816D906A0F0F701608171810E9437
:109090009E92009769F09C012A193B090217130759
:1090A00010F0D22FC32F0196ECCF8FEF9FEF02C0AD
:1090B0008D2F9C2FDF91CF911F910F91FF90EF90FB
:1090C000DF90CF90BF90AF900895FC018081918197
:1090D000009711F00C948D8660E070E0CB0108954C
:1090E000AF92BF92CF92DF92EF92FF920F931F93B6
:1090F000CF93DF93DC01CD90DC901197C114D104A4
:1091000009F442C01496CD91DC9115972097E1F1B6
:109110008C0156017501BFEFAB1ABB0AF7018081C4
:10912000082E000C990B0E94098B892B99F7219727
:10913000CC0DDD1D8881082E000C990B0E94098B37
:10914000892B91F4AE014F5F5F4F4E195F09D80133
:1091500015965C934E931497CE14DF0450F4B70128
:10916000C6010E94719205C0CE15DF0558F3219704
:10917000E1CFD801ED91FC91119714968D919C91BE
:109180001597E80FF91F1082DF91CF911F910F9172
:10919000FF90EF90DF90CF90BF90AF900895EF9247
:1091A000FF920F931F93CF93DF93FC0124813581AE
:1091B0006115710511F480E018C041155105A1F049
:1091C0007B01EC018A01020F131FB80195D388239C
:1091D00091F3288139818C819D81B701820F931F82
:1091E0000E947A921D830C8381E0DF91CF911F91C1
:1091F0000F91FF90EF900895CF93DF93EC016115ED
:10920000710559F0FB0101900020E9F73197AF019A
:10921000461B570BC4DF811102C0CE0194D3CE018F
:10922000DF91CF910895CF93DF93EC01FB0144814F
:10923000558160817181B3DF811102C0CE0183D37A
:10924000CE01DF91CF9108956115710549F0FB01C1
:1092500001900020E9F73197AF01461B570B9FCFD4
:1092600080E00895FB01448155816081718197CF31
:10927000EF92FF920F931F93CF93DF93EC018B013B
:109280006115710549F0CB010E94BA867C01BC01D1
:10929000CE0132D3811103C0CE0155D307C0FD8268
:1092A000EC82B801888199810E94B386CE01DF915A
:1092B000CF911F910F91FF90EF9008950895CF9255
:1092C000DF92EF92FF920F931F93CF93DF936C0186
:1092D0007A018B01C0E0D0E0CE15DF0589F0D8011E
:1092E0006D918D01D601ED91FC910190F081E02D01
:1092F000C6011995892B11F47E0102C02196ECCF8D
:10930000C701DF91CF911F910F91FF90EF90DF90F8
:10931000CF900895FC01A089B1898C91A689B78965
:1093200082FD0FC09C91818D8F5F8F73228D82177C
:1093300049F0218DDF01A20FB11D5D969C93818FB5
:1093400008958C910895FC01538D448D252F30E0B4
:10935000842F90E0821B930B541710F0CF96089542
:1093600001970895FC01918D828D981761F0828D8F
:10937000DF01A80FB11D5D968C91928D9F5F9F7349
:10938000928F90E008958FEF9FEF0895FC01918DEB
:10939000828D981731F0828DE80FF11D858D90E058
:1093A00008958FEF9FEF0895FC01918D228D892FF5
:1093B00090E0805C9F4F821B91098F7399270895DD
:1093C00083EC9DE0F1DF21E0892B09F420E0822F7E
:1093D000089580E69EE0E8DF21E0892B09F420E093
:1093E000822F08958DEF9EE0DFDF21E0892B09F4C5
:1093F00020E0822F0895FC01848DDF01A80FB11DAC
:10940000A35ABF4F2C91848D90E001968F739927BA
:10941000848FA689B7892C93A089B1898C918064A7
:109420008C93938D848D981306C00288F389E02D68
:1094300080818F7D80830895EF92FF920F931F9319
:10944000CF93DF93EC0181E0888F9B8D8C8D9813F7
:1094500005C0E889F989808185FD23C0F62E0B8D32
:1094600010E00F5F1F4F0F731127E02E8C8DE81255
:109470000BC00FB607FCFACFE889F989808185FF18
:10948000F5CFCE01B8DFF2CF8B8DFE01E80FF11DD5
:10949000E35AFF4FF0820B8FEA89FB89808180625B
:1094A00007C0EE89FF896083E889F989808180643B
:1094B000808381E090E0DF91CF911F910F91FF9029
:1094C000EF900895CF93DF93EC01888D8823C1F04E
:1094D000EA89FB89808185FD05C0A889B9898C91BD
:1094E00086FD0EC00FB607FCF5CF808185FFF2CF59
:1094F000A889B9898C9185FFEDCFCE017CDFE8CFBB
:10950000DF91CF91089580E090E0892B19F06ADF18
:1095100081111BC080E090E0892B41F080E090E059
:10952000892B21F00E940000811112C080E090E0A0
:10953000892B19F04EDF81110EC080E090E0892B5D
:1095400079F03EDF81110AC008950E940000E2CF49
:109550000E940000EBCF0E940000EFCF0C940000AF
:10956000089590E0FC013197E231F10508F04EC01A
:109570008827E955FF4F8F4F0C941D9080918000F4
:109580008F7703C0809180008F7D80938000089545
:1095900080918000877FF9CF84B58F7702C084B532
:1095A0008F7D84BD08958091B0008F7703C0809136
:1095B000B0008F7D8093B0000895809190008F77E8
:1095C00007C0809190008F7D03C080919000877FBD
:1095D0008093900008958091A0008F7707C08091BC
:1095E000A0008F7D03C08091A000877F8093A000A2
:1095F0000895809120018F7707C0809120018F7D91
:1096000003C080912001877F8093200108950F93EC
:109610001F93CF93DF938C01EB0188E2FB01119242
:109620008A95E9F74BE050E062ED7AE0CE010E94C6
:109630008F921B8681E090E0A0E0B0E08C879D8750
:10964000AE87BF87F80185899689A789B08D888BF9
:10965000998BAA8BBB8B82E090E0A0E0B0E08C8B72
:109660009D8BAE8BBF8B1CA21DA21EA21FA280E0F1
:1096700090E0A8E4B4E4888F998FAA8FBB8F80E034
:1096800090E0A8E4B4EC8C8F9D8FAE8FBF8F8DECF3
:109690009CECACE4BEE388A399A3AAA3BBA3DF918F
:1096A000CF911F910F9108954F925F926F927F9289
:1096B0008F929F92AF92BF92CF92DF92EF92FF92E2
:1096C0000F931F93CF93DF938C01EB0184E2FB0197
:1096D00011928A95E9F78EE10E94886183E090E01B
:1096E0000E9484610E94276166E08EE10E946A65A3
:1096F0001092780D8093770D90E086309105ECF311
:109700008AE99FE00E943B59882E8AE99FE00E94E7
:109710003B59982E8AE99FE00E943B59682E8AE9BE
:109720009FE00E943B59782E8AE99FE00E943B59B6
:10973000482E8AE99FE00E943B59582EB82CA12C54
:10974000B5016929072E000C880B990B0E943F8BED
:109750004B015C01F8016583768387839087D42C65
:10976000C12CB6016529072E000C880B990B0E94AD
:109770003F8BF8016187728783879487F62CE12CF1
:10978000B7016729072E000C880B990B0E943F8BAD
:10979000F801658776878787908B118A128A138AEA
:1097A000148A84E290E0A0E0B0E088839983AA83E1
:1097B000BB8385899689A789B08D8C839D83AE8371
:1097C000BF8382E090E0A0E0B0E088879987AA8715
:1097D000BB87188A198A1A8A1B8AC0905602D090B1
:1097E0005702E0905802F0905902A7019601C50176
:1097F000B4010E948F8D20E030E048EC52E40E94DA
:109800009E8B6C8B7D8B8E8B9F8BA7019601F801B5
:1098100061857285838594850E948F8D20E030E07C
:1098200048EC52E40E949E8B688F798F8A8F9B8FC1
:1098300020915202309153024091540250915502AE
:10984000F80165857685878590890E948F8D20E057
:1098500030E048EC52E40E949E8B6C8F7D8F8E8F9F
:109860009F8F81E0DF91CF911F910F91FF90EF903B
:10987000DF90CF90BF90AF909F908F907F906F9030
:109880005F904F9008950F931F93CF93DF938C01B8
:10989000EB01FC01808191810097B1F068817981B1
:1098A0006115710579F0428153812C813D81421708
:1098B000530740F00E947A928C819D81F801958334
:1098C000848313C00E94F19088819981F80191836B
:1098D00080838A819B81938382838C819D81958300
:1098E0008483198218821B821A821D821C82DF9156
:1098F000CF911F910F9108950F931F93CF93DF93F3
:10990000EC0188819981009729F02A813B812617F3
:10991000370788F48B016F5F7F4F0E948991009712
:1099200061F0998388831B830A832C813D81232BDB
:1099300011F4FC01108281E001C080E0DF91CF9141
:109940001F910F910895CF93DF93EC018881998146
:10995000009711F00E94F190198218821D821C82DA
:109960001B821A82DF91CF910895EF92FF920F939D
:109970001F93CF93DF93EC017B018A01BA01BCDF17
:10998000811103C0CE01DFDF07C01D830C83B70147
:10999000888199810E947A92CE01DF91CF911F91A7
:1099A0000F91FF90EF900895CF93DF93EC01611535
:1099B000710551F0FB0101900020E9F73197AF01EB
:1099C000461B570BD2DF01C0BEDFCE01DF91CF9126
:1099D0000895CF93DF93EC01FB018617970751F0B1
:1099E000608171816115710521F044815581BDDF70
:1099F00001C0A9DFCE01DF91CF910895FC018081E4
:109A000091810C94F190EF92FF920F931F93CF935B
:109A1000DF93CDB7DEB7A1970FB6F894DEBF0FBEC8
:109A2000CDBF7C01CB01BA01F701118210821382F4
:109A300012821582148242E0420F8E010F5F1F4F87
:109A40000E946B86BC01C701AFDFA1960FB6F894E8
:109A5000DEBF0FBECDBFDF91CF911F910F91FF9061
:109A6000EF900895EF92FF920F931F93CF93DF93A0
:109A7000CDB7DEB7A1970FB6F894DEBF0FBECDBF4E
:109A80007C01CB01BA01F70111821082138212828C
:109A90001582148242E0420F8E010F5F1F4F0E9419
:109AA0006B86BC01C70180DFA1960FB6F894DEBFBC
:109AB0000FBECDBFDF91CF911F910F91FF90EF901F
:109AC00008950F931F93CF93DF93CDB7DEB7A2977F
:109AD0000FB6F894DEBF0FBECDBF8C01CB01BA012B
:109AE000F80111821082138212821582148230E0F2
:109AF000AE014F5F5F4F0E94D786BE016F5F7F4F01
:109B0000C80152DFA2960FB6F894DEBF0FBECDBFDC
:109B1000DF91CF911F910F9108950F931F93CF93D2
:109B2000DF93CDB7DEB762970FB6F894DEBF0FBEF6
:109B3000CDBF8C01CB01F8011182108213821282F9
:109B40001582148250E0BE016F5F7F4F0E94C38672
:109B5000BE016F5F7F4FC80127DF62960FB6F89492
:109B6000DEBF0FBECDBFDF91CF911F910F91089542
:109B7000FC0111821082138212821582148278CB2A
:109B8000FC0111821082138212821582148221CF6D
:109B9000FC011182108213821282158214826115D7
:109BA000710549F0FB0101900020E9F73197AF0101
:109BB000461B570BDACE0895DC01ED91FC91019024
:109BC000F081E02D1994DC01ED91FC91DB011496FC
:109BD0004D915C9115976D917C910280F381E02D00
:109BE0001994EF92FF920F931F93CF93DF938C0101
:109BF0007B01C0E0D0E0F701EC0FFD1F649166230C
:109C000061F0D801ED91FC910190F081E02DC80147
:109C10001995892B11F02196EECFCE01DF91CF91CE
:109C20001F910F91FF90EF9008956115710579F0E4
:109C3000FB0101900020E9F73197AF01461B570B5C
:109C4000DC01ED91FC910280F381E02D199480E01C
:109C500090E008954F925F926F927F92EF92FF9201
:109C60000F931F93CF93DF93CDB7DEB7A1970FB6B6
:109C7000F894DEBF0FBECDBF7C01FA01CB0119A263
:109C8000223008F42AE08E010F5D1F4F422E512C26
:109C9000612C712CBF01A30192010E94978CF901E4
:109CA000CA01015011096A3014F4605D01C0695C99
:109CB000D8016C93232B242B252B61F7B801C70106
:109CC000B4DFA1960FB6F894DEBF0FBECDBFDF9113
:109CD000CF911F910F91FF90EF907F906F905F90C9
:109CE0004F900895CF92DF92EF92FF920F931F93C0
:109CF000CF93DF93EC016A017B012115310579F4E3
:109D0000E881F9810190F081E02D642FDF91CF91FE
:109D10001F910F91FF90EF90DF90CF9019942A3010
:109D20003105D9F477FF18C06DE246DF8C01442776
:109D30005527BA014C195D096E097F092AE0CE0149
:109D400089DF800F911FDF91CF911F910F91FF90BD
:109D5000EF90DF90CF9008952AE0B701A601CE01E1
:109D6000DF91CF911F910F91FF90EF90DF90CF90F7
:109D700071CF9A01AB01770F660B770BB3CF6AED0A
:109D80007AE053CF0F931F93CF93DF93EC014DDF16
:109D90008C01CE01F4DF800F911FDF91CF911F91D5
:109DA0000F9108950F931F93CF93DF93EC010BDF77
:109DB0008C01CE01E4DF800F911FDF91CF911F91C5
:109DC0000F91089532CF1F920F920FB60F92112468
:109DD0000BB60F922F933F934F935F936F937F93A5
:109DE0008F939F93AF93BF93EF93FF9383EC9DE08B
:109DF00002DBFF91EF91BF91AF919F918F917F9186
:109E00006F915F914F913F912F910F900BBE0F90EB
:109E10000FBE0F901F9018951F920F920FB60F92C2
:109E200011240BB60F922F933F934F935F936F9331
:109E30007F938F939F93AF93BF93EF93FF9383ECA5
:109E40009DE068DAFF91EF91BF91AF919F918F9163
:109E50007F916F915F914F913F912F910F900BBE2A
:109E60000F900FBE0F901F9018951F920F920FB674
:109E70000F9211240BB60F922F933F934F935F9342
:109E80006F937F938F939F93AF93BF93EF93FF93C2
:109E900080E69EE0B0DAFF91EF91BF91AF919F9184
:109EA0008F917F916F915F914F913F912F910F9083
:109EB0000BBE0F900FBE0F901F9018951F920F9220
:109EC0000FB60F9211240BB60F922F933F934F931F
:109ED0005F936F937F938F939F93AF93BF93EF9312
:109EE000FF9380E69EE016DAFF91EF91BF91AF916C
:109EF0009F918F917F916F915F914F913F912F91A2
:109F00000F900BBE0F900FBE0F901F9018951F92D1
:109F10000F920FB60F9211240BB60F922F933F930F
:109F20004F935F936F937F938F939F93AF93BF9361
:109F3000EF93FF938DEF9EE05EDAFF91EF91BF917B
:109F4000AF919F918F917F916F915F914F913F91D1
:109F50002F910F900BBE0F900FBE0F901F90189572
:109F60001F920F920FB60F9211240BB60F922F93E0
:109F70003F934F935F936F937F938F939F93AF9391
:109F8000BF93EF93FF938DEF9EE0C4D9FF91EF91C4
:109F9000BF91AF919F918F917F916F915F914F9101
:109FA0003F912F910F900BBE0F900FBE0F901F90FF
:109FB0001895CF93DF93EC01E881F9810680F78152
:109FC000E02D1995EA89FB8980818F7E8083EA895B
:109FD000FB898081877F8083EA89FB8980818F77F5
:109FE0008083EA89FB8980818F7D80838A8D898F38
:109FF000DF91CF910895CF93DF93282F30E0F901BF
:10A00000E55EF44F8491F901EB52F54FD491F901DB
:10A01000E157F54FC491CC2389F08111A2DAEC2FDE
:10A02000F0E0EE0FFF1FEB58F54FA591B491EC91C6
:10A03000ED2381E090E021F480E002C080E090E038
:10A04000DF91CF910895862FD6CF1F93CF93DF93C3
:10A05000282F30E0F901E55EF44F8491F901EB52CD
:10A06000F54FD491F901E157F54FC491CC23C1F0DC
:10A07000162F811176DAEC2FF0E0EE0FFF1FE55A74
:10A08000F54FA591B4918FB7F894111105C09C912B
:10A09000ED2FE095E92302C0EC91ED2BEC938FBFFF
:10A0A000DF91CF911F910895CF93DF9390E0FC0152
:10A0B000EB52F54F2491FC01E157F54F8491882331
:10A0C00061F190E0880F991FFC01EF5BF54FC5919E
:10A0D000D491FC01E55AF54FA591B491611109C0E5
:10A0E0009FB7F8948881209582238883EC912E2352
:10A0F0000BC0623061F49FB7F8943881822F80954D
:10A1000083238883EC912E2B2C939FBF06C08FB79F
:10A11000F894E8812E2B28838FBFDF91CF9108958B
:10A12000863308F0865390917B00282F2870977F04
:10A13000922B90937B00877020915A0290E4299F84
:10A1400090011124822B80937C0080917A0080649E
:10A1500080937A0080917A0086FDFCCF8091780010
:10A160002091790090E0922B08953FB7F894809168
:10A170007E0C90917F0CA091800CB091810C26B543
:10A18000A89B05C02F3F19F00196A11DB11D3FBF2F
:10A19000BA2FA92F982F8827820F911DA11DB11DBD
:10A1A000BC01CD0142E0660F771F881F991F4A95B9
:10A1B000D1F708958F929F92AF92BF92CF92DF9284
:10A1C000EF92FF926B017C01D0DF4B015C01C11467
:10A1D000D104E104F104E9F0C8DFDC01CB01881906
:10A1E0009909AA09BB09883E9340A105B10578F3F6
:10A1F00021E0C21AD108E108F10888EE880E83E058
:10A20000981EA11CB11CC114D104E104F10421F772
:10A21000DECFFF90EF90DF90CF90BF90AF909F90F8
:10A220008F9008952FB7F89460917A0C70917B0C01
:10A2300080917C0C90917D0C2FBF08951F920F92FE
:10A240000FB60F9211242F933F938F939F93AF9349
:10A25000BF9380917A0C90917B0CA0917C0CB09173
:10A260007D0C3091790C23E0230F2D3720F40196DB
:10A27000A11DB11D05C026E8230F0296A11DB11D29
:10A280002093790C80937A0C90937B0CA0937C0C98
:10A29000B0937D0C80917E0C90917F0CA091800CEE
:10A2A000B091810C0196A11DB11D80937E0C9093FD
:10A2B0007F0CA093800CB093810CBF91AF919F91C4
:10A2C0008F913F912F910F900FBE0F901F90189577
:10A2D00096E0899FD0011124A35FBE4E90967C9397
:10A2E0006E935F9791E091969C93919790917911DD
:10A2F000E0917A11F0917B11992339F0309751F068
:10A30000811108C08091291104C0309719F05C9622
:10A310008C91199408953F924F925F926F927F9221
:10A320008F929F92AF92BF92CF92DF92EF92FF9265
:10A330000F931F93CF93DF93CDB7DEB728970FB658
:10A34000F894DEBF0FBECDBF0E9407666C01E12C02
:10A35000F12C1091A3101295110F110F107C1C5CA1
:10A3600087E70E94886164EF8AE99FE0D4D7612F74
:10A370008AE99FE0D0D70E9427618091A3108111C4
:10A3800005C065E070E080E090E012C0813029F403
:10A3900068E070E080E090E00BC0823029F46EE06D
:10A3A00070E080E090E004C06AE170E080E090E05E
:10A3B00001DF86EF0E94DA654C01A12CB12CBA2C8A
:10A3C000A92C982C882488EF0E94B765882A3090A1
:10A3D000A3108091B8109091B910A7019601281B85
:10A3E000390B41095109A091B610B091B7100E94E4
:10A3F000878C6B017C01AFE0F594E794D794C79408
:10A40000AA95D1F76091B0107091B110CB01770F80
:10A41000AA0BBB0BBC01CD01BBE0660F771F881FE9
:10A42000991FBA95D1F72091B2103091B3108901DC
:10A43000330F220B330BA90198012C0D3D1D4E1D2E
:10A440005F1D0E946B8CC20ED31EE41EF51E20EA17
:10A45000C21A2FE0D20AE108F108A7019601C7014C
:10A46000B6010E94E78F9B01AC011CE05595479512
:10A47000379527951A95D1F729833A834B835C83C7
:10A480000091A4101091A510A091A810B091A9104E
:10A49000A70196010E94918C2B013C018DE07594DF
:10A4A0006794579447948A95D1F7A091AA10B091D8
:10A4B000AB1029813A814B815C810E94918CBB2732
:10A4C00097FDB095AB2F840D951DA61DB71D029667
:10A4D000A11DB11D32E0B595A795979587953A9541
:10A4E000D1F79C01AD0130584F4F5F4FA091B41090
:10A4F000B091B5100E94878C2B013C014FE07694FF
:10A500006794579447944A95D1F788E090E083196F
:10A510009109A501940104C0569547953795279553
:10A520008A95D2F72D833E834F8358874801110FB8
:10A53000AA08BB0852E0880C991CAA1CBB1C5A959F
:10A54000D1F7A091AC10B091AD1029813A814B8127
:10A550005C810E94918C9B01AC016BE05595479505
:10A56000379527956A95D1F729833A834B835C8386
:10A57000A091A610B091A710A70196010E94918CFE
:10A58000DC01CB017BE0B595A795979587957A95EA
:10A59000D1F729813A814B815C81820F931FA41FDF
:10A5A000B51F880D991DAA1DBB1D032C04C0880F63
:10A5B000991FAA1FBB1F0A94D2F7BC01CD016E5F81
:10A5C0007F4F8F4F9F4F24E030E040E050E00E94EB
:10A5D0006B8C8D819E81AF81B885821B930BA40B00
:10A5E000B50B9C01AD0180E593ECA0E0B0E0BC01AF
:10A5F000CD0104C096958795779567953A94D2F7E3
:10A600000E94E78F97FD0BC0660F771F881F991F69
:10A61000A30192010E94978C69017A010AC0A301EB
:10A6200092010E94978C69017A01CC0CDD1CEE1C12
:10A63000FF1C9927F7FC9A958F2D7E2D6D2D9B0180
:10A64000AC010E94E78F9B01AC01AEEDBBE00E9424
:10A65000878C4C01BB2497FCB094AB2CA3E4B3EEE5
:10A66000A70196010E94938CBB2797FDB095AB2F55
:10A67000880D991DAA1DBB1D8153914FAF4FBF4F30
:10A6800044E0B595A795979587954A95D1F7BC0174
:10A69000CD016C0D7D1D8E1D9F1D28960FB6F89463
:10A6A000DEBF0FBECDBFDF91CF911F910F91FF9005
:10A6B000EF90DF90CF90BF90AF909F908F907F9062
:10A6C0006F905F904F903F900895CF92DF92EF92FE
:10A6D000FF920F931F930E940766AC0160E070E049
:10A6E000E3EAF0E1858996899A01AB01281B390BD1
:10A6F00041095109A389B4890E94878C6B017C01AF
:10A700008FE0F594E794D794C7948A95D1F765853F
:10A710007685CB01770FAA0BBB0BBC01CD012BE0DB
:10A72000660F771F881F991F2A95D1F727853089D3
:10A730008901330F220B330BA90198012C0D3D1D0C
:10A740004E1D5F1D0E946B8CD701C601820F931FA7
:10A75000A41FB51F0896A11DB11DBC01CD0134E099
:10A7600095958795779567953A95D1F70E943F8B98
:10A7700020E030E040E251E40E948F8D1F910F9164
:10A78000FF90EF90DF90CF9008958F929F92AF92BD
:10A79000BF92EF92FF920F931F93CF93DF93D82F27
:10A7A000C62F1092F3101092F4101092F510109220
:10A7B000F6101092F71061E077DC60E08D2F45DC39
:10A7C0006C2F70E080E090E0F5DC60E08D2F6CDCB9
:10A7D0008BE990E00197F1F700E911E08D2F0BDC98
:10A7E000892B31F401501109C9F78EEF9FEF4CC04E
:10A7F00000E911E08D2FFFDB019721F401501109D1
:10A80000C9F7F3CF18E2C0E800E020E9E22EFF2408
:10A81000F3948D2FF0DB892B29F481E0E81AF108FD
:10A82000C1F7E3CFA2DC4B015C0190E9E92EFF24E4
:10A83000F3948D2FE0DB019729F481E0E81AF10809
:10A84000C1F7D3CF92DCDC01CB0188199909AA09A1
:10A85000BB098997A105B10538F0E02FF0E0E5517B
:10A86000FF4E80858C2B80872C2F30E035952795E7
:10A870002115310511F0C22F02C00F5FC0E8115041
:10A8800009F0C3CF80E090E0DF91CF911F910F914D
:10A89000FF90EF90BF90AF909F908F900895EF92B0
:10A8A000FF920F931F93CF93DF93C82F8B017A01F1
:10A8B00083E50E9488616C2F8AE99FE02CD50E9475
:10A8C000276183E50E948861B80183E590E00E94DA
:10A8D000AE65E701CE018E199F093091770D209169
:10A8E000780D321729F08AE99FE0C5D48993F2CF19
:10A8F0008017910729F01092F91081E08093FA10E7
:10A90000DF91CF911F910F91FF90EF900C942761F1
:10A91000CF93DF93AC01990F660B770B2AE030E001
:10A920008DEF9EE0DFD9EC018DEF9EE028DA8C0FF1
:10A930009D1FDF91CF9108951F93CF93DF931F92B7
:10A94000CDB7DEB7162FAE014F5F5F4F61E070E00D
:10A95000A6DF898190E002C0959587951A95E2F768
:10A9600081700F90DF91CF911F910895CF93DF9366
:10A97000D82FC62F83E50E9488616D2F8AE99FE05A
:10A98000CAD46C2F8AE99FE0C6D4DF91CF910C9492
:10A990002761FF920F931F93CF93DF931F92CDB741
:10A9A000DEB7182F062FF42EAE014F5F5F4F61E028
:10A9B00070E075DF8981FF2049F041E050E001C07F
:10A9C000440F0A95EAF7482B498309C021E030E09B
:10A9D00001C0220F0A95EAF720952823298369816F
:10A9E000812FC4DF0F90DF91CF911F910F91FF90C6
:10A9F0000895CF93DF9342E00E94CE61EC018DEF8A
:10AA00009EE0BDD98C0F9D1FDF91CF910895AF922D
:10AA1000BF92CF92DF92EF92FF921F93CF93DF937B
:10AA2000CDB7DEB72A970FB6F894DEBF0FBECDBF05
:10AA3000182F47E051E166E070E082E39F832FDF4B
:10AA40002091081130E0322F222780910711282B06
:10AA50003A83298320910A1130E0322F22278091F6
:10AA60000911282B3C832B8320910C1130E0322FCD
:10AA7000222780910B11282B3E832D839E012F5F6F
:10AA80003F4F59015BEFC52E50E1D52EE12E9F813E
:10AA9000F92EF501619171915F01F60121913191DA
:10AAA000419151916F01072E000C880B990B2F8358
:10AAB000388749875A870E943F8B2F81388549857F
:10AAC0005A850E949E8BF7016193719381939193B4
:10AAD0007F01F7E0CF16F1E1DF06D9F62A960FB62F
:10AAE000F894DEBF0FBECDBFDF91CF911F91FF90D5
:10AAF000EF90DF90CF90BF90AF9008953F924F922C
:10AB00005F926F927F928F929F92AF92BF92CF92FD
:10AB1000DF92EF92FF920F931F93CF93DF9300D0BA
:10AB20001F921F92CDB7DEB7982E7CDB2B013C0124
:10AB300020ED420E27E0521E611C711C60E08091E6
:10AB40007C1183DA35E0832ECE0101966C01AA24B4
:10AB5000A394B12C55E0352E380EF601282D119214
:10AB60002A95E9F7860127E0E22EF12C80917D11EC
:10AB700042DA019731F456DB6415750586059705B1
:10AB8000A8F380917D1137DA892B31F44BDB641502
:10AB9000750586059705A8F380917E112CDA892B1F
:10ABA00051F0F8012081C5010E2C01C0880F0A94D4
:10ABB000EAF7822B8083F1E0EF1AF108B8F60F5F15
:10ABC0001F4F3012D0CF2EDB641575058605970513
:10ABD00048F061E080917C1138DA60E070E080EC50
:10ABE0009FE72BC089818911B8CF9B818A81980FFB
:10ABF000990D8C818913B1CF8D818D3009F0ADCF46
:10AC000061E080917C1121DA6A818B8170E0762F7E
:10AC10006627680F711D072E000C880B990B0E9488
:10AC20003F8B20E030E040E85DE30E949E8B23E311
:10AC300033E948E853E40E94C88C0F900F900F90BE
:10AC40000F900F90DF91CF911F910F91FF90EF9098
:10AC5000DF90CF90BF90AF909F908F907F906F903C
:10AC60005F904F903F900895AF92BF92CF92DF9246
:10AC7000EF92FF920F931F93CF93DF931F92CDB765
:10AC8000DEB75C01D62EE72EFC018585811105C05B
:10AC9000C5010E94C742811106C0F50113861586C1
:10ACA000148680E065C040E060EFC5010E945B4211
:10ACB00001E0F12CC12C11E0C5010E940842682F6F
:10ACC000C50169830E9408426981613019F48130AD
:10ACD000B9F433C04F2D50E068131BC0F5018385D4
:10ACE000181730F4E40FF51F8381802349F402C064
:10ACF000181731F060E0193058F4F501148708C0D6
:10AD0000F501EF0DF11D8381802B838361E009C084
:10AD1000C12EF501E40FF51F9381802F80958923C3
:10AD20008383C5010E942C421F5F000F11F4F3942E
:10AD300001E0F7E0FF1508F0BFCF113408F4ADCF04
:10AD4000F501C386C11002C081E08587F5018381CA
:10AD5000882309F4A2CFD5011396ED2DFE2D950180
:10AD6000255F3F4F8D918193A217B307D9F781E0FB
:10AD70000F90DF91CF911F910F91FF90EF90DF9097
:10AD8000CF90BF90AF9008959F92AF92BF92CF9215
:10AD9000DF92EF92FF920F931F93CF93DF93CDB784
:10ADA000DEB761970FB6F894DEBF0FBECDBF8C0142
:10ADB0008CE0F8018183C12CD12C2FE5E22E3FE7F6
:10ADC000B32E4FE1A42E5FE3952EF801848190E02D
:10ADD000C816D9060CF0A0C04C2DBE01665F7F4F8F
:10ADE000C8010E94CB41F8018181893038F0F82EEA
:10ADF000FCE0F81728F49CE0F92E02C089E0F82E58
:10AE00008A85803139F0BE01665F7F4FC8010E949C
:10AE1000D24301C08CE08F1509F47AC0AE014F5FB8
:10AE20005F4FBE01665F7F4FC8010E946943882360
:10AE300009F46EC08A85803109F46AC08BE0F81687
:10AE400051F0ECE0FE1629F0FAE0FF1206C09D82F8
:10AE500005C0BD8203C0ED8201C0AD82F8018681CC
:10AE600097810E94C742BE01665F7F4FF8018681CD
:10AE700097810E949C4240E06EE4F80186819781B0
:10AE80000E945B4240E06B81F801868197810E94BD
:10AE90005B4240E06C81F801868197810E945B42B1
:10AEA0008A85803139F040E06D81F8018681978193
:10AEB0000E945B42F801868197810E94C742BE01D1
:10AEC000665F7F4FF801868197810E949C42F8015E
:10AED000408168E4868197810E945B4264E170E072
:10AEE00080E090E067D9F8018081882329F06AE04A
:10AEF00070E080E090E05ED9F801868197810E9441
:10AF0000C742F8018181F81608F4F82EF801F182A1
:10AF1000FFEFCF1ADF0A59CF61960FB6F894DEBF64
:10AF20000FBECDBFDF91CF911F910F91FF90EF909A
:10AF3000DF90CF90BF90AF909F900895CF93DF9315
:10AF40000E94AD621092901180919411823018F09D
:10AF500098E09093901190919511992339F0813058
:10AF600029F48091901184608093901162E370E0E5
:10AF700080E090E01FD9609196118BE891E10E94EA
:10AF8000404568EE73E080E090E014D960E38BE820
:10AF900091E10E945B45CBE4D6E4CE010197F1F745
:10AFA00060E38BE891E10E945B452197F1F760E354
:10AFB0008BE891E10E945B4583E592E00197F1F710
:10AFC00060E28BE891E10E945B4580919011806284
:10AFD0000E94926184E0809391118CE00E949261C2
:10AFE00081E00E949261CBE3DFE1CE010197F1F7AE
:10AFF00082E08093921186E00E94926182E00E943A
:10B0000092612197F1F7DF91CF910895FC0144817E
:10B0100055818091A1109091A2108417950780F01E
:10B0200080919D1090919E10009751F060817181E8
:10B030006115710529F00E94819221E0892B09F0A8
:10B0400020E0822F0895FF920F931F93CF93DF93F9
:10B05000CDB7DEB72B970FB6F894DEBF0FBECDBFCE
:10B0600080E69EE00E94D94F40E855E260E070E043
:10B0700080E69EE00E94F67B64E670E080E090E06F
:10B0800099D88CED95E0A0E0B0E08093640E9093A9
:10B09000650EA093660EB093670E64E670E080E0E4
:10B0A00090E088D88FEF898381E08A8386E88B835C
:10B0B0001C821D821E821F82188689E7898780E68E
:10B0C0009EE00E94624A62E370E080E090E072D805
:10B0D00080E69EE00E94A34908974CF049E050E0CA
:10B0E000BE016F5F7F4F80E69EE00E945F4962E392
:10B0F00070E080E090E05ED880E69EE00E94D44957
:10B10000892B01F180E69EE00E94A349089784F410
:10B1100065E070E080E090E04DD800E010E0F12CB8
:10B1200080E69EE00E94D44902301105A4F50CC0CF
:10B1300049E050E0BE016F5F7F4F80E69EE00E94D5
:10B140005F49E6CFF12C27C080E69EE00E94D449FB
:10B15000892B99F465E070E080E090E02BD8023014
:10B160001105F1F69A8589819813DACF9B858B8139
:10B170009813D6CFFF24F394D3CF80E69EE00E94AD
:10B18000B249EAE0F0E0EC0FFD1FE00FF11F808311
:10B190000F5F1F4FDFCF62E370E080E090E00AD8DE
:10B1A00080E69EE00E94D94F8F2D2B960FB6F89423
:10B1B000DEBF0FBECDBFDF91CF911F910F91FF90EA
:10B1C00008950F931F93CF93DF93C82FD62F86E058
:10B1D000C89FF0011124E35FFE4E11A2878D90A15C
:10B1E00081309105E1F01CF4892B49F03FC0823099
:10B1F000910591F10397D1F560E070E031C06623CD
:10B20000A9F161E070E08C2F63D80CD860936511D0
:10B2100070936611809367119093681127C002D8CC
:10B22000009165111091661120916711309168119C
:10B23000AB01BC01401B510B620B730B809177116A
:10B2400090917811A0E0B0E084179507A607B707A2
:10B2500018F462E070E004C0D11108C063E070E04F
:10B260008C2FDF91CF911F910F9132C8DF91CF9139
:10B270001F910F9108959091780D8091770D9817F7
:10B2800050F4E92FF0E0E557F34F208130E09F5F65
:10B290009093780D02C02FEF3FEFC9010895809180
:10B2A000770D90E02091780D821B91090895089503
:10B2B00080E090E00895CF92DF92EF92FF920F939B
:10B2C0001F93CF93DF937C01262F972F8A018091C4
:10B2D000A00D882391F0C62FD72F6E01C40ED51E66
:10B2E000CC15DD0571F06991D701ED91FC910190CC
:10B2F000F081E02DC7011995F3CF642F822F0E94B2
:10B30000DD47C801DF91CF911F910F91FF90EF9022
:10B31000DF90CF900895CF93DF931F92CDB7DEB724
:10B3200069832091A00D2223D1F02091C20D2032FB
:10B3300040F021E030E0FC013383228380E090E0A4
:10B3400015C08091A10DE82FF0E0EE55F24F9981E4
:10B3500090838F5F8093A10D8093C20D05C061E043
:10B36000CE0101960E94DD4781E090E00F90DF91D1
:10B37000CF9108950C94F1900F931F93CF93C091A8
:10B38000840460E08C2F0E94255083E090E00197B8
:10B39000F1F761E08C2F0E94255083E290E0019745
:10B3A000F1F760E08C2F0E942550809182049091EB
:10B3B00083049927FC01EB52F54F6491FC01E1579E
:10B3C000F54FE491F0E0EE0FFF1FEB58F54F85913C
:10B3D000949100E412E42FE030E0462F0E945D7C5F
:10B3E000611571058105910549F0DC01CB010196DC
:10B3F000A11DB11DBC01CD019F7003C060E070E0D4
:10B40000CB010E943D8B20E030E048EC52E40E94EA
:10B410008F8D2091870C3091880C4091890C509130
:10B420008A0C0E949E8B20E030E44CE156E40E949E
:10B430008F8D20E030E040E05FE30E949E8BCF9153
:10B440001F910F9108950895CF92DF92EF92FF928E
:10B4500093DF6B017C0120E030E040E050E40E948B
:10B460007E8E18161CF488DF6B017C0120E030E032
:10B4700040E050E4C701B6010E947E8E18161CF40D
:10B480007BDF6B017C0120E030E040E050E4C7014D
:10B49000B6010E947E8E18161CF46EDF6B017C01D3
:10B4A00020E030E040E050E4C701B6010E947E8E0B
:10B4B00018162CF4FF90EF90DF90CF905DCFC7016E
:10B4C000B601FF90EF90DF90CF9008954F925F927A
:10B4D0006F927F928F929F92AF92BF92CF92DF92A4
:10B4E000EF92FF92CF93DF93CDB7DEB760970FB6A1
:10B4F000F894DEBF0FBECDBF61E0809184040E944E
:10B50000545060E0809182040E945450DED86093D1
:10B51000830C7093840C8093850C9093860C23E3AA
:10B5200033E948E853E40E948F8D20E030E040E8A2
:10B530005FE30E94C98C0E948D8F26E636EA45EAB9
:10B5400053E40E949E8B6093870C7093880C8093C9
:10B55000890C90938A0C78DFAB01BC0123E0CE010B
:10B5600001960E94324DBE016F5F7F4FCE0107965C
:10B570000E94C04D61E179E0CE0107960E94FC482F
:10B58000BC018FE790E10E94E94CCE0107960E9432
:10B59000FE4CCE0101960E94FE4C6FEA78E0CE018F
:10B5A00001960E94C84D6FE770E1CE0101960E949E
:10B5B0001349BC0185E890E10E94E94CCE01019657
:10B5C0000E94FE4C41DF9B01AC016D873E874F8797
:10B5D000588B0E94B5502B013C016EE170E080E079
:10B5E00090E00E94DA5030DF6B017C010E94B55080
:10B5F0004B015C0184189508A608B7082D853E8587
:10B600004F85588981ED881687E09806A104B1041A
:10B610000CF43FC0C701B6010E94C88C6B017C01CD
:10B6200020E030E0A9010E947E8E18165CF426EA24
:10B630003BE944EC5BE3C701B6010E94398B87FF0D
:10B640000BC027C026EA3BE944EC5BEBC701B6011F
:10B650000E947E8E1816ECF0C501B40128EE33E08E
:10B6600040E050E00E946B8CCA01B9010E943F8B00
:10B670004B015C0120E030E04AE754E4C701B60129
:10B680000E949E8BA50194010E948F8DAB01BC018D
:10B6900003C040E050E0BA0122E0CE0101960E94D2
:10B6A000324DBE016F5F7F4FCE0107960E94C04DA5
:10B6B00062EB78E0CE0107960E94FC48BC0189E766
:10B6C00090E10E94E94CCE0107960E94FE4CCE010B
:10B6D00001960E94FE4C6DED7AE0CE0101960E942B
:10B6E000C84D69E770E1CE0101960E941349BC0183
:10B6F00085E890E10E943249CE0101960E94FE4CFD
:10B7000064E07BE0CE0101960E94C84D69E770E1DC
:10B71000CE0101960E941349BC018FE790E10E947F
:10B720003249CE0101960E94FE4C66EB78E0CE01D4
:10B7300001960E94C84D4AE050E060E070E0CE0102
:10B7400001960E94ED6DCE0101960E94FE4C6FE7BE
:10B7500070E1CE0101960E94C04D45E050E06FEFD0
:10B760007FEFCE0101960E94BC6CCE0101960E9433
:10B77000FE4C61EE7AE085E890E10E94244960E0A9
:10B78000809184040E94545060960FB6F894DEBFF6
:10B790000FBECDBFDF91CF91FF90EF90DF90CF90A4
:10B7A000BF90AF909F908F907F906F905F904F90E1
:10B7B000089581E08093800480918104882341F082
:10B7C00088E08093961160E08BE891E10C9440450D
:10B7D00008958091810481110EC081E080938104DD
:10B7E0008093800480919111982F9460909391118F
:10B7F0008C6098D517C080918004882399F01092AE
:10B80000961160E08BE891E10E944045109280041F
:10B81000809191118B7F80939111886083D51092D4
:10B8200081040895C6CF2F923F924F925F926F92FC
:10B830007F928F929F92AF92BF92CF92DF92EF92C0
:10B84000FF920F931F93CF93DF93CDB7DEB764972B
:10B850000FB6F894DEBF0FBECDBF7C0180E69EE040
:10B860000E94D94F40E855E260E070E080E69EE03B
:10B870000E94F67B64E670E080E090E00E94DA507F
:10B880008CED95E0A0E0B0E08093640E9093650E9F
:10B89000A093660EB093670E64E670E080E090E0DF
:10B8A0000E94DA508FEF898381E08A8386E88B8358
:10B8B0001C821D821E821F82188689E78987C70124
:10B8C000880F991F9C8B8B8B212C312CC12CD12C58
:10B8D000812C912C5401CE14DF044CF080E69EE0C4
:10B8E0000E94D94FC114D104A1F1760132C08B89D5
:10B8F0009C892816390694F780E69EE00E94A349A9
:10B9000008974CF049E050E0BE016F5F7F4F80E642
:10B910009EE00E945F4965E070E080E090E00E9458
:10B92000DA5000E010E0412C512C320180E69EE01C
:10B930000E94D449892B31F484E0481651046104F3
:10B9400071041CF4023011057CF19FEF291A390AA9
:10B95000C2CFC501B4010E943F8B4B015C01B7010E
:10B96000FF0C880B990B0E943F8B9B01AC01C5011A
:10B97000B4010E948F8D64960FB6F894DEBF0FBE9F
:10B98000CDBFDF91CF911F910F91FF90EF90DF908E
:10B99000CF90BF90AF909F908F907F906F905F906F
:10B9A0004F903F902F90089580E69EE00E94D449EA
:10B9B000892B69F080E69EE00E94B249EAE0F0E05F
:10B9C000EC0FFD1FE00FF11F80830F5F1F4F65E03D
:10B9D00070E080E090E00E94DA5002301105D1F56D
:10B9E0009A858981981336C09B858B81981332C0C4
:10B9F00080E69EE00E94D449892B31F494E04916F8
:10BA00005104610471048CF40930110589F080E659
:10BA10009EE00E94B249EAE0F0E0EC0FFD1FE00F6B
:10BA2000F11F80830F5F1F4FE3CF043011057CF0BF
:10BA30002D858C8590E0982F8827820F911D092EE7
:10BA4000000CAA0BBB0B880E991EAA1EBB1E8FEF03
:10BA5000C81AD80A9FEF491A590A690A790A66CFA3
:10BA60002F923F924F925F927F928F929F92AF92CE
:10BA7000BF92CF92DF92EF92FF920F931F93CF93DB
:10BA8000DF9300D01F92CDB7DEB76C018CEE94E04F
:10BA90009C838B83E3E1F2E0FA83E98305EE1CE00B
:10BAA000EE24E394F12C9DE3292E312C2EE3422E3B
:10BAB000512C30E1A32EB12C41E1842E912C57E181
:10BAC000752E80911102909112028E159F050CF433
:10BAD000ECC0F1E0CF16D10431F4F80180819181FE
:10BAE000E981FA8109C0F2E0CF16D10439F4E98185
:10BAF000FA8180819181F80191838083E981FA81C3
:10BB000080819181009749F4EB81FC81828193814E
:10BB100090937F0480937E0428C08130910549F47E
:10BB2000EB81FC818281938190937D0480937C04DE
:10BB30001CC08230910549F4EB81FC8182819381A4
:10BB400090937B0480937A0410C0039771F4EB8187
:10BB5000FC818281938190937904809378046CEDC9
:10BB60007AE085EE90E10E94D44CE981FA818191DE
:10BB70009191FA83E9838430910549F4EB81FC814A
:10BB800022813381309377042093760430C085304E
:10BB9000910549F4EB81FC81228133813093750456
:10BBA0002093740424C08630910549F4EB81FC8114
:10BBB000228133813093C7042093C60424C0873088
:10BBC000910549F4EB81FC81228133813093730428
:10BBD0002093720424C08A30910549F4EB81FC81E2
:10BBE0002281338130937104209370043AC08531EF
:10BBF000910549F4EB81FC812281338130936F04FC
:10BC000020936E042EC08631910549F4EB81FC81AE
:10BC10002281338130936D0420936C0422C08731DC
:10BC20009105F9F4EB81FC8122813381A901475010
:10BC300051094230510540F4B0928504A092840429
:10BC4000909283048092820425503109223031057C
:10BC500040F43092850420928404509283044092F0
:10BC600082049C012B5031092A30310598F4EB8174
:10BC7000FC81228133813093790420937804789E6B
:10BC8000B001799E700D1124655A7D4F85EE90E1CB
:10BC90000E94D44CFFEFEF1AFF0A8B819C81029621
:10BCA0009C838B830E5F1F4F0CCF0F900F900F90D4
:10BCB0000F90DF91CF911F910F91FF90EF90DF9048
:10BCC000CF90BF90AF909F908F907F905F904F905C
:10BCD0003F902F900895FF920F931F93CF93DF9380
:10BCE000F82E0AE010E0C0E0D0E08F2D0E949050C6
:10BCF000C80FD91F65E070E080E090E00E94DA5044
:10BD00000150110991F7CE016AE070E00E94F68FB0
:10BD1000CB01DF91CF911F910F91FF9008952F924A
:10BD20003F924F925F926F927F928F929F92AF92CB
:10BD3000BF92CF92DF92EF92FF920F931F93CF9318
:10BD4000DF93CDB7DEB72B970FB6F894DEBF0FBEEB
:10BD5000CDBF7C018BEB8F838AEA888781E089875E
:10BD600084E68E9D90018F9D300D11243B872A879C
:10BD7000C12CD12C212C312C812C912C54012E142E
:10BD80003F048CF1C501B4010E943F8B20E030E0FC
:10BD900040E251E40E948F8D4B015C01B701FF0C22
:10BDA000880B990B0E943F8B9B01AC01C501B4012C
:10BDB0000E948F8D2B960FB6F894DEBF0FBECDBFBD
:10BDC000DF91CF911F910F91FF90EF90DF90CF9077
:10BDD000BF90AF909F908F907F906F905F904F90AB
:10BDE0003F902F9008952A853B85C216D30654F6BE
:10BDF000C6016AE070E00E940A90892B49F443E092
:10BE000050E0BE01695F7F4F80E69EE00E945F497F
:10BE100065E070E080E090E00E94DA503FEFC31AE6
:10BE2000D30A00E010E0412C512C320180E69EE064
:10BE30000E94D449892B39F424E04216510461044C
:10BE400071040CF09CCF063011050CF098CF80E601
:10BE50009EE00E94D449892B69F080E69EE00E9412
:10BE6000B249E1E0F0E0EC0FFD1FE00FF11F80832D
:10BE70000F5F1F4F65E070E080E090E00E94DA50B5
:10BE80000630110501F599818F8198131CC09A81A4
:10BE90008885981318C09B818985981314C02C81BC
:10BEA0008D8190E0A0E0B0E0BA2FA92F982F8827CD
:10BEB000820F911DA11DB11D880E991EAA1EBB1EC9
:10BEC0008FEF281A380A9FEF491A590A690A790A26
:10BED000ADCF1F93CF93DF93182FC7E2DDE0812F03
:10BEE0000E949050899399936CE370E080E090E019
:10BEF0000E94DA508DE0C737D80789F754D320E085
:10BF000030E040EA50E40E949E8B20E030E040E8C0
:10BF10005AE30E949E8BDF91CF911F910895CF929B
:10BF2000DF92EF92FF920F931F93CF93DF93CDB7E2
:10BF3000DEB72C970FB6F894DEBF0FBECDBF809151
:10BF4000820C811102C00E94586C80E69EE00E9423
:10BF5000D94F64E670E080E090E00E94DA506BE731
:10BF60007BE08FE790E10E9438496FE770E1CE01F6
:10BF700001960E94C04D44E150E060E070E0CE01C7
:10BF800001960E94ED6DCE0101960E94FE4C6CE67A
:10BF90007BE08FE790E10E9438496FE770E1CE01C6
:10BFA00001960E94C04D44E150E06FEF7FEFCE015B
:10BFB00001960E94BC6CCE0101960E94FE4C8CE45E
:10BFC0000E947E556B017C0104E010E0A701960100
:10BFD000C701B6010E94CE8F882309F47EC00150AC
:10BFE000110961F064E670E080E090E00E94DA50B0
:10BFF0008CE40E947E556B017C01E8CF61E67BE01A
:10C000008FE790E10E9438496FE770E1CE01019619
:10C010000E94C04D4AE050E060E070E0CE01019621
:10C020000E94ED6DCE0101960E94FE4C64EF7AE015
:10C03000CE0101960E94C84D6FE770E1CE010196D6
:10C040000E941349BC0185E890E10E94E94CCE01B1
:10C0500001960E94FE4C80914C0C90914D0C0397E0
:10C0600051F510924D0C10924C0C25C06CED7AE0FD
:10C070008BE890E10E94D44C6BE870E1CE01019610
:10C080000E94C04D64E07BE0CE0101960E94FC4816
:10C0900065E870E10E941349BC0185E890E10E94C7
:10C0A000E94CCE0101960E94FE4C83E090E0909313
:10C0B0004D0C80934C0C64E670E080E090E00E94B0
:10C0C000DA508091820C882309F4B2C060E273E0F8
:10C0D00080E090E00E94DA50ABC021E0B701A601F9
:10C0E000CE0107960E94324D66E07BE0CE010196BC
:10C0F0000E94C84DBE01695F7F4FCE0101960E942C
:10C100001349BC0185E890E10E94E94CCE010196FB
:10C110000E94FE4CCE0107960E94FE4C65E870E13D
:10C12000CE0101960E94C04D42E350E06FEF7FEFD9
:10C13000CE0101960E94BC6CCE0101960E94FE4C7D
:10C140000E949A6C6FE07BE085E890E10E942449B0
:10C1500086E60E947E556B017C0104E010E0A70199
:10C160009601C701B6010E94CE8F882381F001504D
:10C17000110909F47BCF68EC70E080E090E00E9448
:10C18000DA5086E60E947E556B017C01E8CF21E003
:10C19000B701A601CE0107960E94324D61EE78E00C
:10C1A000CE0101960E94C84DBE01695F7F4FCE014E
:10C1B00001960E941349BC018BE890E10E94E94C72
:10C1C000CE0101960E94FE4CCE0107960E94FE4CC5
:10C1D00064E07BE0CE0101960E94C84D6BE870E1FF
:10C1E000CE0101960E941349BC018FE790E10E94A5
:10C1F000E94CCE0101960E94FE4C6FE770E1CE0142
:10C2000001960E94C04D4AE050E060E070E0CE012F
:10C2100001960E943B6DCE0101960E94FE4C0E9449
:10C220009A6C6FE07BE08BE890E10E94244924CF78
:10C230002C960FB6F894DEBF0FBECDBFDF91CF9125
:10C240001F910F91FF90EF90DF90CF900895209174
:10C25000C20D90919711213208F04AC080919F0D34
:10C260008111FCCF32E030939F0D31E030939E0D71
:10C270003FEF30939D0D10929C0D20939B0DA2EAF1
:10C28000BDE04BE75DE0FA013E2F341B321718F496
:10C290003D913193F9CF10927A0D20917A0D990F3B
:10C2A000922B90937A0D9091790D913061F41092C8
:10C2B000790D90917A0D9093BB009091BC0093FD05
:10C2C000F8CF95EC01C095EE9093BC0090919F0D36
:10C2D0009230E1F390919D0D9F3F79F080919D0DFB
:10C2E000803241F080919D0D803331F084E005C0B3
:10C2F00081E003C082E001C083E01092A10D1092A2
:10C30000C20D1092A00D0895682F8AE99FE003C81E
:10C3100091E09093A00D809397111092A10D10922F
:10C32000C20D0895CF93C82F682F607F8BE891E1ED
:10C330000E945B4580E1C89FB00111248BE891E128
:10C34000CF910C945B45CF93DF93CDB7DEB72897A1
:10C350000FB6F894DEBF0FBECDBF98E0EEEFF4E06D
:10C36000DE01119601900D929A95E1F7909194114A
:10C37000961710F46FEF690FFE013196E60FF11D6D
:10C38000E60FF11D9081890F806828960FB6F8940A
:10C39000DEBF0FBECDBFDF91CF91C4CF4F925F9272
:10C3A0006F927F928F929F92AF92BF92CF92DF92C5
:10C3B000EF92FF926B017C01B42E9B01AC010E94B5
:10C3C000CE8F882319F060E27BE027C02601370179
:10C3D000E89477F82FEF3FEF4FE75FE7C301B20133
:10C3E0000E94CE8F81110DC02FEF3FEF4FE75FE727
:10C3F000C301B2010E94398B18161CF464E27BE081
:10C400000CC02FEF3FEF4FE75FE4C701B6010E947A
:10C410007E8E181694F468E27BE08DEF9EE0FF902C
:10C42000EF90DF90CF90BF90AF909F908F907F90D4
:10C430006F905F904F900C94154E2FEF3FEF4FE7AA
:10C440005FECC701B6010E94398B87FDE4CF20E085
:10C4500030E0A901C701B6010E94398B87FF0BC0EC
:10C460006DE28DEF9EE00E94DC4D4C01F7FAF094F6
:10C47000F7F8F09402C0812C912CA12C60E070E0C0
:10C4800080E09FE3AB1441F020E030E040E251E473
:10C490000E948F8DA394F6CF9B01AC01C701B6011A
:10C4A0000E94C98C2B013C010E942D8E6B017C01E6
:10C4B0000E943D8B9B01AC01C301B2010E94C88C5C
:10C4C0002B013C012AE0B701A6018DEF9EE00E94FE
:10C4D0002A4E7C01E80CF91CBB2039F06EE28DEF8E
:10C4E0009EE00E94DC4DE80EF91EDB2CDD2031F1D0
:10C4F00020E030E040E251E4C301B2010E949E8B93
:10C500002B013C010E942D8E4B01A12CB12C2AE065
:10C51000B501A4018DEF9EE00E942A4EE80EF91E9F
:10C52000C501B4010E943D8B9B01AC01C301B20166
:10C530000E94C88C2B013C01DA94D8CFC701FF9030
:10C54000EF90DF90CF90BF90AF909F908F907F90B3
:10C550006F905F904F90089521CF1092780D1092B8
:10C56000770D1092A10D1092C20D10929F0D81E0D7
:10C5700080939E0D1092790D61E084E10E94255018
:10C5800061E085E10E942550E9EBF0E080818E7F3B
:10C59000808380818D7F808388E48093B80085E4E8
:10C5A0008093BC0008952F923F924F925F926F92BA
:10C5B0007F928F929F92AF92BF92CF92DF92EF9233
:10C5C000FF920F931F93CF93DF93CDB7DEB72897DA
:10C5D0000FB6F894DEBF0FBECDBF4091270D50912E
:10C5E000280DC090290DD0902A0D4C155D052CF01A
:10C5F0003C2D2D2D6A01432F522FEBE2FDE060E030
:10C6000070E0CB01019111910417150754F44A0110
:10C61000550FAA08BB08680D791D8A1D9B1DA8012E
:10C6200015C0C016D10654F40D2C000CEE08FF08FE
:10C630006C0D7D1D8E1D9F1D680108C0012E000C14
:10C64000220B330B600F711F821F931F2DE0E73702
:10C65000F207C1F60E943F8B20E030E048E152E44F
:10C660000E948F8D6B017C0107E21DE0812C912CD3
:10C670005401D8016D917D918D01072E000C880B1E
:10C68000990B0E943F8BA70196010E94C88C9B01C9
:10C69000AC010E949E8B9B01AC01C501B4010E94BC
:10C6A000C98C4B015C01BDE007371B0711F720E087
:10C6B00030E04CE152E40E948F8D0E948D8F4B013F
:10C6C0005C0120E030E040E85FE30E947E8E1816B7
:10C6D0000CF06EC007E21DE0212C312C19821A8269
:10C6E0001B821C82F801819191918F019C01990F0D
:10C6F000440B550B2D833E834F835887CA01B901E4
:10C700000E943F8BA70196010E94C88C2B013C011F
:10C7100020E030E0A9010E947E8E181624F077FAFE
:10C72000709477F87094A5019401C301B2010E943E
:10C73000398B87FF13C089819A81AB81BC812D81A0
:10C740003E814F815885820F931FA41FB51F898397
:10C750009A83AB83BC833FEF231A330A4DE007373C
:10C76000140709F0BFCF20E030E040EC5FE3C501E3
:10C77000B4010E949E8B4B015C0155E025163104EB
:10C780000CF4A8CF69817A818B819C810E943F8BB8
:10C790006B017C01B101330C880B990B0E943F8B1C
:10C7A0009B01AC01C701B6010E948F8D6B017C011A
:10C7B000C701B60128960FB6F894DEBF0FBECDBFF5
:10C7C000DF91CF911F910F91FF90EF90DF90CF906D
:10C7D000BF90AF909F908F907F906F905F904F90A1
:10C7E0003F902F9008954F925F926F927F928F9219
:10C7F0009F92AF92BF92CF92DF92EF92FF920F93F0
:10C800001F93CF93DF9300D01F92CDB7DEB76B019C
:10C810007C0111E0A12EB12C4501880C991C880CDB
:10C82000991CF401E256FB4F408051806280738076
:10C83000A3019201C701B6010E947E8E181614F45E
:10C840001F5FE8CFA3019201C701B6010E94398B97
:10C8500084010A571B4F811106C0D8016D917D914B
:10C860008D919C9142C0C5018150904C880F991FB9
:10C87000880F991FFC01E256FB4F208131814281D4
:10C88000538129833A834B835C83FC01EA57FB4F36
:10C8900080809180A280B380C701B6010E94C88CBD
:10C8A0006B017C01A5019401D8016D917D918D9161
:10C8B0009C910E94C88C9B01AC01C701B6010E94EB
:10C8C0009E8B6B017C0129813A814B815C81C30184
:10C8D000B2010E94C88C9B01AC01C701B6010E9445
:10C8E0008F8DA50194010E94C98C0F900F900F901D
:10C8F0000F90DF91CF911F910F91FF90EF90DF90FC
:10C90000CF90BF90AF909F908F907F906F905F90EF
:10C910004F900895DF92EF92FF920F931F93CF9362
:10C92000DF937C018B01EA014617570720F4812F22
:10C930008A01C62FD82F6CED7AE0C7010E94C84D3E
:10C940008091A1109091A21008171907E0F48C179C
:10C950009D0708F4EC01E0919D10F0919E10EC0F02
:10C96000FD1FD080108260919D1070919E10600F0D
:10C97000711FC7010E94D44CE0919D10F0919E1050
:10C98000EC0FFD1FD082C701DF91CF911F910F9156
:10C99000FF90EF90DF900895CF93DF93EC014091EB
:10C9A000A1105091A210B6DFCE01DF91CF91089572
:10C9B0000F931F930E9412516093680E7093690E3B
:10C9C00080936A0E90936B0EE091600EF091610E71
:10C9D0000284F385E02D80E69EE0199597FF1FC045
:10C9E0000E9412510091680E1091690E20916A0EFA
:10C9F00030916B0EDC01CB01801B910BA20BB30BB2
:10CA00000091640E1091650E2091660E3091670EB4
:10CA100080179107A207B307B8F28FEF9FEF1F911E
:10CA20000F910895CF93DF931F92CDB7DEB760913A
:10CA3000250D8EED93E069830E94558C69816817FE
:10CA400021F08EED93E00E945D8C6091260D8FEDBC
:10CA500093E069830E94558C6981681721F08FEDFE
:10CA600093E00E945D8C85E29DE00F90DF91CF9175
:10CA70000895CF92DF92EF92FF920F931F93CF937F
:10CA8000DF931F92CDB7DEB76C010BEA1CE07C018F
:10CA90008AE7E80EF11CF80161918F01C6016983F4
:10CAA0000E94558C6981681719F0C6010E945D8C3F
:10CAB000FFEFCF1ADF0ACE14DF0469F78BEA9CE0A0
:10CAC0000F90DF91CF911F910F91FF90EF90DF902A
:10CAD000CF90089590919F0D9111FCCF91E090938C
:10CAE0009F0D90939E0D2FEF20939D0D10929C0D06
:10CAF000260F20939B0D90937A0D90917A0D880FBD
:10CB0000892B80937A0D8091790D813061F4109298
:10CB1000790D80917A0D8093BB008091BC0083FDDC
:10CB2000F8CF85EC01C085EE8093BC0080919F0D0D
:10CB30008130E1F380919C0D861710F460919C0D7B
:10CB4000ABE7BDE02BE83CE0F9018E2F821B861796
:10CB500018F48D918193F9CF862F0895613208F0F2
:10CB600060E2B8DF1092780D8093770D08951F93DF
:10CB7000CF93DF931F92CDB7DEB7682F87E7698326
:10CB8000C7DB69818AE99FE00E948B5960DB87E7F8
:10CB9000BFDB61E070E087E790E0E0DF8AE99FE0DB
:10CBA0000E943B59182F53DB812F0F90DF91CF91BB
:10CBB0001F9108950F931F93CF93DF931F92CDB7CB
:10CBC000DEB7682F87E76983A3DB69818AE99FE085
:10CBD0000E948B593CDB87E79BDB62E070E087E7D4
:10CBE00090E0BCDF8AE99FE00E943B5900E010E042
:10CBF000182F8AE99FE00E943B59082B192B27DB4D
:10CC0000C8010F90DF91CF911F910F91089587E791
:10CC10007FDB64EF8AE99FE00E948B596EE28AE92C
:10CC20009FE00E948B5913DB65E070E080E090E0AC
:10CC30000E94DA5086EFBECF8F929F92AF92BF9242
:10CC4000CF92DF92EF92FF920F931F93CF93DF93D8
:10CC50007C01862F9BE0E916F10409F070C09091E9
:10CC6000F810992309F0F89462E10E94C553EC0191
:10CC70008091F810882309F07894209709F074C007
:10CC8000D090F310C090F4106D2D70E080E090E033
:10CC90000E943F8B4B015C016C2D70E080E090E0C6
:10CCA0000E943F8B2DEC3CEC4CEC5DE30E949E8B94
:10CCB0009B01AC01C501B4010E94C98C6093EB10CB
:10CCC0007093EC108093ED109093EE101091F5108E
:10CCD0000091F610612F6F7770E080E090E00E9485
:10CCE0003F8B4B015C01602F70E080E090E00E9480
:10CCF0003F8B2DEC3CEC4CEC5DE30E949E8B9B014A
:10CD0000AC01C501B4010E94C98C17FD09C0609334
:10CD1000EF107093F0108093F1109093F2100BC00D
:10CD2000DC01CB01B0588093EF109093F010A093EA
:10CD3000F110B093F210DC0C1D0D100F6FC096E1D6
:10CD4000E916F10409F071C09091F810992309F0E7
:10CD5000F89461E00E94C553EC018091F81088239B
:10CD600009F078942097A9F080E090ECA9E7B4EC62
:10CD70008093EB109093EC10A093ED10B093EE1015
:10CD80008093EF109093F010A093F110B093F210F5
:10CD90004FC00091F410D090F310602F70E07D2907
:10CDA00080E090E00E943D8B2DEC3CEC4CEC5DE390
:10CDB0000E949E8B6093EB107093EC108093ED10AB
:10CDC0009093EE10C090F6101091F510812F8F7790
:10CDD0006C2D70E0782B80E090E00E943D8B2DEC74
:10CDE0003CEC4CEC5DE30E949E8B17FD09C0609308
:10CDF000EF107093F0108093F1109093F2100BC02D
:10CE0000DC01CB01B0588093EF109093F010A09309
:10CE1000F110B093F2100D0DC00E1C0D8091F710A3
:10CE2000811731F0CFEFDFEF03C0CFEFDFEF48C066
:10CE3000CF3F9FEFD90709F410C1209709F01CC11B
:10CE40008090EB109090EC10A090ED10B090EE1050
:10CE500020E030E048EC52E4C501B4010E947E8E2F
:10CE600018160CF006C1CBEFDFEF20E030E0A9018F
:10CE7000C501B4010E94398B87FF02C0CAEFDFEF02
:10CE80008090EF109090F010A090F110B090F21000
:10CE900020E030E048EC52ECC501B4010E94398B2F
:10CEA00087FF02C0C9EFDFEF20E030E040EF52E43F
:10CEB000C501B4010E947E8E181614F4C8EFDFEF8E
:10CEC0008CE0E816F10409F0DFC08CE521DA80E09F
:10CED00090E01ADABCD965E08CE5FCDD1092780DA3
:10CEE0008093770DC82FD0E02097B1F0C530D105E1
:10CEF00084F000E010E08AE99FE00E943B59F801CD
:10CF0000E856FE4E80870F5F1F4F0C171D079CF3DE
:10CF100006C0CDEFDFEFB8C0CEEFDFEFB5C0C091F8
:10CF2000A0110091A1116C2F70E080E090E00E94B0
:10CF30003F8B6B017C01602F70E080E090E00E94ED
:10CF40003F8B2DEC3CEC4CEC5DE30E949E8B9B01F7
:10CF5000AC01C701B6010E94C98C6093981170930F
:10CF6000991180939A1190939B11D091A2111091D5
:10CF7000A3116D2F6F7770E080E090E00E943F8BEF
:10CF80006B017C01612F70E080E090E00E943F8B9C
:10CF90002DEC3CEC4CEC5DE30E949E8B9B01AC01C4
:10CFA000C701B6010E94C98CD7FF5AC0DC01CB0172
:10CFB000B05880939C1190939D11A0939E11B093B3
:10CFC0009F11802F8C0FC82FCD0FC10F8091A411FE
:10CFD0008C1343C0C0909811D0909911E0909A1191
:10CFE000F0909B1120E030E048EC52E4C701B6011C
:10CFF0000E947E8E18161CF4CBEFDFEF02C0C0E05B
:10D00000D0E020E030E0A901C701B6010E94398BD1
:10D0100087FF02C0CAEFDFEFC0909C11D0909D1136
:10D02000E0909E11F0909F1120E030E048EC52EC2F
:10D03000C701B6010E94398B87FF02C0C9EFDFEF3D
:10D0400020E030E040EF52E4C701B6010E947E8E3E
:10D050001816D4F4C8EFDFEF17C0CFEFDFEF14C01E
:10D0600060939C1170939D1180939E1190939F11DA
:10D07000A8CFC0E0D0E0F9CE229619F0CCEFDFEFD8
:10D080001FCFCEEFDFEF1CCFCE01DF91CF911F91ED
:10D090000F91FF90EF90DF90CF90BF90AF909F9057
:10D0A0008F9008958F929F92AF92BF92CF92DF920E
:10D0B000EF92FF92CF93DF93CDB7DEB72C970FB6E9
:10D0C000F894DEBF0FBECDBF64E77CE0CE010196D1
:10D0D0000E94B84D4CE251E06FEF7FEFCE01019618
:10D0E0004BD4CE0101960E94FE4C60917C0470915D
:10D0F0007D0480912302909124029EDD84E1882E9C
:10D10000912CA12CB12CE12CF12C8FEFE81AF80A0C
:10D11000C501B4010E94DA5060917C0470917D04D5
:10D12000809123029091240287DD23E0E216F1042E
:10D1300034F424E1820E911CA11CB11CE6CF2AE03C
:10D14000E216F1041CF4892BA1F703C0892B09F026
:10D150006FC180912302909124028B309105C9F414
:10D160008091EF109091F010A091F110B091F21019
:10D170008093A9119093AA11A093AB11B093AC1115
:10D180008091EB109091EC10A091ED10B091EE1009
:10D190001DC08631910521F30C9701F580919C11FA
:10D1A00090919D11A0919E11B0919F118093A91112
:10D1B0009093AA11A093AB11B093AC1180919811E8
:10D1C00090919911A0919A11B0919B118093A51102
:10D1D0009093A611A093A711B093A8114091A91103
:10D1E0005091AA116091AB117091AC1121E0CE0168
:10D1F00007960E94324D61EE78E0CE0101960E94C2
:10D20000C84DBE01695F7F4FCE0101960E94134950
:10D21000BC0185E890E10E94E94CCE0101960E9494
:10D22000FE4CCE0107960E94FE4C4091A5115091F4
:10D23000A6116091A7117091A81121E0CE01079667
:10D240000E94324D6DE879E0CE0101960E94C84DF2
:10D25000BE01695F7F4FCE0101960E941349BC0158
:10D2600085E890E10E943249CE0101960E94FE4C71
:10D27000CE0107960E94FE4C66E279E085E890E1D7
:10D280000E9424496CED7AE0CE0101960E94C84DBF
:10D2900044E150E060E070E0CE0101969ED4CE0102
:10D2A00001960E94FE4C6091A9117091AA11809183
:10D2B000AB119091AC110E94288E4AE0CE010196EC
:10D2C0000E948D4DBE016F5F7F4F8FE790E10E94FE
:10D2D000434CCE0101960E94FE4C60E086E033D8BC
:10D2E0006FE770E18BE891E10E94E34D6FED8BE811
:10D2F00091E10E94DC4D63E979E08BE891E10E94C5
:10D30000E24E6091A5117091A6118091A7119091A4
:10D31000A8110E94288E4AE050E08BE891E10E941B
:10D32000B94E66E279E08BE891E10E94E24E64E654
:10D3300070E080E090E00E94DA50C090A911D09097
:10D34000AA11E090AB11F090AC1120E030E040EF7A
:10D3500051E4C701B6010E947E8E87FD03C065E6D9
:10D360007CE052C020E030E040ED51E4C701B6015E
:10D370000E947E8E87FD1EC065E57CE0CE01019691
:10D380000E94B84D4AE050E06FEF7FEFCE0101966A
:10D39000F3D2CE0101960E94FE4C8091490288236F
:10D3A00031F06CED75E080E090E00E94DA5065E4C9
:10D3B0007CE02AC020E030E040EB51E4C701B60138
:10D3C0000E947E8E87FD03C067E37CE01DC068E29B
:10D3D0007CE0CE0101960E94B84D4AE050E06FEF2C
:10D3E0007FEFCE010196C8D2CE0101960E94FE4C7D
:10D3F00080914902882331F06CED75E080E090E087
:10D400000E94DA506AE17CE0CE0101960E94B84D9C
:10D410004AE050E06FEF7FEFCE010196ADD2CE0132
:10D4200001960E94FE4C62E370E080E090E0C5C08F
:10D430003FD26EE170E080E090E00E94DA500E94FE
:10D4400065536B017C0164E670E080E090E00E942F
:10D45000DA5061EE78E085E890E10E94D44C21E05A
:10D46000B701A601CE0101960E94324DBE016F5F49
:10D470007F4F85E890E10E943249CE0101960E94DB
:10D48000FE4C65E870E1CE0101960E94C04D4AE075
:10D4900050E060E070E0CE0101969FD3CE0101968E
:10D4A0000E94FE4C47D26FE07BE085E890E10E944D
:10D4B0002449C092A911D092AA11E092AB11F09226
:10D4C000AC1120E030E040EF51E4C701B6010E940A
:10D4D0007E8E87FD03C06AE07CE052C020E030E031
:10D4E00040ED51E4C701B6010E947E8E87FD1EC04B
:10D4F0006AEF7BE0CE0101960E94B84D4AE050E011
:10D500006FEF7FEFCE01019637D2CE0101960E94D8
:10D51000FE4C80914902882331F06CED75E080E08B
:10D5200090E00E94DA506AEE7BE02AC020E030E012
:10D5300040EB51E4C701B6010E947E8E87FD03C017
:10D540006CED7BE01DC06DEC7BE0CE0101960E948E
:10D55000B84D4AE050E06FEF7FEFCE0101960CD25C
:10D56000CE0101960E94FE4C80914902882331F041
:10D570006CED75E080E090E00E94DA506FEB7BE0AC
:10D58000CE0101960E94B84D4AE050E06FEF7FEF68
:10D59000CE010196F1D1CE0101960E94FE4C6CE2C3
:10D5A00071E080E090E00E94DA5080914902882387
:10D5B00031F068EE73E080E090E00E94DA502C9643
:10D5C0000FB6F894DEBF0FBECDBFDF91CF91FF90B5
:10D5D000EF90DF90CF90BF90AF909F908F90089585
:10D5E000CF93DF93FC0124813581232B69F0EC017B
:10D5F000BC018DEF9EE00E94D24EBE0183EC9DE007
:10D60000DF91CF910C94D24EDF91CF910895CF92BC
:10D61000DF92EF92FF920F931F93CF93DF93CDB7DB
:10D62000DEB728970FB6F894DEBF0FBECDBF8234A9
:10D6300009F441C0CCF4803309F45DC07CF483323A
:10D6400009F450C08A3209F076C067E875E08DE9C8
:10D6500090E10E94D44C8FEF9FEF6AC0813309F4B0
:10D6600059C08134E9F067C08136D1F02CF483349D
:10D6700069F1843439F05FC0833641F1E4F08436D7
:10D6800009F059C08091951090919610892B09F45A
:10D69000F8C081E990E10E94654897FF74C0F1C02D
:10D6A0006EE775E08DE990E10E94D44C80914A0CC0
:10D6B00090914B0C3DC06BE775E08DE990E10E94C5
:10D6C000D44C1092820C8CEF9FEF32C061E875E071
:10D6D0008DE990E10E94D44C81E08093820C8DEF23
:10D6E0009FEF26C064E875E08DE990E10E94D44C7C
:10D6F0008EEF9FEF1DC065E775E081E990E10E9424
:10D70000D44C65E775E08DE990E10E94D44C80E04F
:10D7100090E00EC068E875E081E990E10E94D44C89
:10D7200068E875E08DE990E10E94D44C81E090E0DA
:10D730000E94221FAEC01A8219821C821B821E8286
:10D740001D828F831886BE01695F7F4FCE010196CF
:10D750000E94D44CBE016F5F7F4F81E990E10E942F
:10D76000434CCE0101960E94FE4C81E990E10E945B
:10D770006548CB010E94221F64E670E080E090E0E3
:10D780000E94DA5086C080914E0C882361F068EBCD
:10D790007BE08DEF9EE00E94F14D61E970E18DEF3D
:10D7A0009EE00E94D24E81E990E10E9465480AEF16
:10D7B0001FEF2FEF3FEF68017901C61AD70AE80A79
:10D7C000F90AB701A6012AE0CE0101960E94614D37
:10D7D000BE016F5F7F4F81E990E10E94434CCE0113
:10D7E00001960E94FE4C81E990E147C08FEFE81A54
:10D7F000F80A89EEE81683E0F80609F448C06EE1FD
:10D8000070E080E090E00E94DA500E94377A182F92
:10D81000112361F31033DCF16AE270E0611B7109DE
:10D8200017FD73954AE0CE0101960E948D4DBE0111
:10D830006F5F7F4F8DE990E10E94434CCE010196CE
:10D840000E94FE4C6DE970E181E990E10E94E94C93
:10D8500080914E0C882379F061EB7BE08DEF9EE0A8
:10D860000E94F14D612F8DEF9EE00E94DC4D8DEF07
:10D870009EE00E94BF4E8DE990E10E946548CB0179
:10D8800057CF0E94377A182FE12CF12CC1CF1451B9
:10D89000C3CF28960FB6F894DEBF0FBECDBFDF9181
:10D8A000CF911F910F91FF90EF90DF90CF9008954F
:10D8B000809181048823F9F0809180048823D9F035
:10D8C00081E00E9492618BE39FE10197F1F760E0B4
:10D8D00080E00E94A36166ED7CE08BE891E10E940C
:10D8E000F14D61E080E00E94A36166EC7CE08BE892
:10D8F00091E10C94F14D0895CF93DF932091810431
:10D900002223A9F020918004222389F0EC016FEDFD
:10D910008BE891E10E94DC4D8C819D81892B39F04F
:10D92000BE018BE891E1DF91CF910C94E34DDF9143
:10D93000CF91089580918104882379F080918004AB
:10D94000882359F06FED8BE891E10E94DC4D60E196
:10D950007BE08BE891E10C94E24E08958091810484
:10D96000882349F080918004882329F060E08BE8C7
:10D9700091E10C94714508958F929F92AF92BF925E
:10D98000EF92FF920F931F93CF93DF937C01EB01F4
:10D990008A0180918104882309F462C08091800407
:10D9A000882309F45DC077FF18C0C095D09561E069
:10D9B0008C2F0E94A361B7018BE891E10E94E34D97
:10D9C00065EB7CE08BE891E10E94F14DF7018481E9
:10D9D00061E08C0F0E94A36133C00E9412518090BD
:10D9E000D40B9090D50BA090D60BB090D70B24E61B
:10D9F000820E911CA11CB11C86169706A806B906BA
:10DA000078F561E08C2F0E94A361B7018BE891E16A
:10DA10000E94E34D64EA7CE08BE891E10E94F14DC5
:10DA2000F701848161E08C0F0E94A3610E94125172
:10DA30006093D40B7093D50B8093D60B9093D70B38
:10DA4000B801110F880B990BDF91CF911F910F91A6
:10DA5000FF90EF90BF90AF909F908F900C94DA5012
:10DA6000DF91CF911F910F91FF90EF90BF90AF90FA
:10DA70009F908F900895AF92BF92CF92DF92EF92D6
:10DA8000FF920F931F93CF93DF93CDB7DEB76297CB
:10DA90000FB6F894DEBF0FBECDBF209181042223C4
:10DAA00009F48AC020918004222309F485C06A0108
:10DAB0007B015C010E9412510091AD111091AE11D9
:10DAC0002091AF113091B0110C591F4F2F4F3F4F84
:10DAD000061717072807390708F06EC0F7FE08C0B9
:10DAE00087010095109560E0802F0E94A36143C0DC
:10DAF00060E080E00E94A3610E94125128EE33E0B2
:10DB000040E050E00E946B8CBA01A9012AE0CE01EE
:10DB100001960E94614DBE016F5F7F4FCE01079657
:10DB20000E94C04D6CE776E0CE0107960E94FC484B
:10DB3000BC01CE010D960E94C04DCE0107960E94F9
:10DB4000FE4CCE0101960E94FE4CBE01635F7F4FEA
:10DB50008BE891E10E94E34D09891A89E114F104EF
:10DB600031F00E0D1F1D60E0802F0E94A361CE01D9
:10DB70000D960E94FE4CB5018BE891E10E94E34DA9
:10DB800063E97CE08BE891E10E94F14DF50184812D
:10DB900060E0800F0E94A3610E9412516093AD115A
:10DBA0007093AE118093AF119093B011B601DD0C5C
:10DBB000880B990B0E94DA5062960FB6F894DEBF7C
:10DBC0000FBECDBFDF91CF911F910F91FF90EF90CE
:10DBD000DF90CF90BF90AF900895BF92CF92DF9229
:10DBE000EF92FF920F931F93CF93DF93CDB7DEB7E2
:10DBF00062970FB6F894DEBF0FBECDBF6C018B01EC
:10DC00007A0180918104882309F475C08091800491
:10DC1000882309F470C077FF07C00095109560E075
:10DC2000802F0E94A36146C060E080E00E94A36153
:10DC30000E94125128EE33E040E050E00E946B8CCD
:10DC4000BA01A9012AE0CE0101960E94614DBE01F0
:10DC50006F5F7F4FCE0107960E94C04D6CE776E064
:10DC6000CE0107960E94FC48BC01CE010D960E9491
:10DC7000C04DCE0107960E94FE4CCE0101960E9437
:10DC8000FE4CBE01635F7F4F8BE891E10E94E34D44
:10DC9000B98860E08B2D0E94A3610115110511F474
:10DCA0000B2D04C060E0802F0E94A361CE010D9671
:10DCB0000E94FE4CB6018BE891E10E94E34D62E8C0
:10DCC0007CE08BE891E10E94F14DF601848160E0F7
:10DCD000800F0E94A3610E9412516093AD11709356
:10DCE000AE118093AF119093B011B701FF0C880B68
:10DCF000990B0E94DA5062960FB6F894DEBF0FBE01
:10DD0000CDBFDF91CF911F910F91FF90EF90DF90EA
:10DD1000CF90BF900895CF93DF93CDB7DEB72C9708
:10DD20000FB6F894DEBF0FBECDBF8091210D90914C
:10DD3000220D892B01F561E17AE0CE0101960E9466
:10DD4000C84D65E871E1CE0101960E941349BC01FE
:10DD5000CE0107960E94C04D48EC50E06FEF7FEF78
:10DD6000CE0107963ADFCE0107960E94FE4CCE0107
:10DD700001960E94FE4C8091210D9091220D0197F9
:10DD800001F56DEF79E0CE0101960E94C84D65E87E
:10DD900071E1CE0101960E941349BC01CE010796A4
:10DDA0000E94C04D48EC50E06FEF7FEFCE01079628
:10DDB00014DFCE0107960E94FE4CCE0101960E9410
:10DDC000FE4C65E17AE0CE0101960E94C84D6FE7F6
:10DDD00071E1CE0101960E941349BC01CE01079664
:10DDE0000E94C04D40ED57E06FEF7FEFCE010796E8
:10DDF000C3DDCE0107960E94FE4CCE0101960E9423
:10DE0000FE4C80914C0C90914D0C019719F462E4FA
:10DE10007EE002C064E37EE0CE0101960E94B84D30
:10DE200048EC50E06FEF7FEFCE01019624DECE018B
:10DE300001960E94FE4C64E27EE0CE0101960E94B3
:10DE4000B84D40ED57E06FEF7FEFCE01019694DDC6
:10DE5000CE0101960E94FE4C64E17EE0CE01019667
:10DE60000E94B84D48EC50E06FEF7FEFCE01019675
:10DE700002DECE0101960E94FE4C67E07EE0CE01FC
:10DE800001960E94B84D40ED57E06FEF7FEFCE0155
:10DE9000019672DDCE0101960E94FE4C6AEF7DE094
:10DEA000CE0101960E94B84D48EC50E06FEF7FEF35
:10DEB000CE010196E0DDCE0101960E94FE4C6FEE90
:10DEC0007DE0CE0101960E94B84D40ED57E06FEF26
:10DED0007FEFCE01019650DDCE0101960E94FE4CEF
:10DEE00063EE7DE0CE0101960E94B84D48EC50E013
:10DEF0006FEF7FEFCE010196BEDDCE0101960E944D
:10DF0000FE4C62ED7DE0CE0101960E94B84D40EDE1
:10DF100057E06FEF7FEFCE0101962EDDCE01019627
:10DF20000E94FE4C80914C0C90914D0C039719F47B
:10DF300067EC7DE002C06DEB7DE0CE0101960E94B2
:10DF4000B84D48EC50E06FEF7FEFCE01019693DDC6
:10DF5000CE0101960E94FE4C62EB7DE0CE0101965F
:10DF60000E94B84D40ED57E06FEF7FEFCE01019674
:10DF700003DDCE0101960E94FE4C65EA7DE0CE01F4
:10DF800001960E94B84D48EC50E06FEF7FEFCE0154
:10DF9000019671DDCE0101960E94FE4C66E97DE09E
:10DFA000CE0101960E94B84D40ED57E06FEF7FEF34
:10DFB000CE010196E1DCCE0101960E94FE4C6BE899
:10DFC0007DE0CE0101960E94B84D48EC50E06FEF25
:10DFD0007FEFCE0101964FDDCE0101960E94FE4CEF
:10DFE0006EE77DE0CE0101960E94B84D40ED57E00E
:10DFF0006FEF7FEFCE010196BFDCCE0101960E944C
:10E00000FE4C80914C0C90914D0C029719F46DE6EA
:10E010007DE002C06DE57DE0CE0101960E94B84D25
:10E0200048EC50E06FEF7FEFCE01019624DDCE018A
:10E0300001960E94FE4C60E57DE0CE0101960E94B3
:10E04000B84D40ED57E06FEF7FEFCE01019694DCC5
:10E05000CE0101960E94FE4C64E47DE0CE01019663
:10E060000E94B84D48EC50E06FEF7FEFCE01019673
:10E0700002DDCE0101960E94FE4C64E37DE0CE01FC
:10E0800001960E94B84D40ED57E06FEF7FEFCE0153
:10E09000019672DCCE0101960E94FE4C69E27DE0A1
:10E0A000CE0101960E94B84D48EC50E06FEF7FEF33
:10E0B000CE010196E0DCCE0101960E94FE4C6FE19C
:10E0C0007DE0CE0101960E94B84D40ED57E06FEF24
:10E0D0007FEFCE01019650DCCE0101960E94FE4CEE
:10E0E0006FE07DE0CE0101960E94B84D48EC50E013
:10E0F0006FEF7FEFCE010196BEDCCE0101960E944C
:10E10000FE4C62E07DE0CE0101960E94B84D40EDEC
:10E1100057E06FEF7FEFCE0101962EDCCE01019626
:10E120000E94FE4C66EF7CE0CE0101960E94B84D45
:10E1300048EC50E06FEF7FEFCE0101969CDCCE0102
:10E1400001960E94FE4C66EE7CE0CE0101960E9494
:10E15000B84D40ED57E06FEF7FEFCE0101960CDC3C
:10E16000CE0101960E94FE4C2C960FB6F894DEBFAD
:10E170000FBECDBFDF91CF9108950F931F93CF9323
:10E18000DF9300D000D0CDB7DEB720914E0C222314
:10E19000A9F08C016EE97AE0CE0101960E94C84D8B
:10E1A000B801CE0101960E941349BC018DEF9EE09B
:10E1B0000E94D24ECE0101960E94FE4C26960FB6CA
:10E1C000F894DEBF0FBECDBFDF91CF911F910F91AD
:10E1D00008954F925F926F927F928F929F92AF922B
:10E1E000BF92CF92DF92EF92FF920F931F93CF9344
:10E1F000DF93CDB7DEB7C654D1090FB6F894DEBFB2
:10E200000FBECDBF8C016CED7AE0CE018B960E94E3
:10E21000C84D6CED7AE0CE0185960E94C84DBE01D6
:10E220006F5F7F4F8AEB90E10E94544B8D889E88F0
:10E23000AF88B88C498C5A8C6B8C7C8C8D8D9E8D64
:10E24000AF8DB8A127968CAF9DAFAEAFBFAF27976C
:10E25000C8010197039708F0C0C1A3019201C5014D
:10E26000B40190580E943C8D2BED3FE049EC5FE3F8
:10E270000E94C98C20914102309142024091430298
:10E28000509144020E94C98C6B017C0120E030E077
:10E29000A9010E94398B87FD09C0C092B911D092A3
:10E2A000BA11E092BB11F092BC1110C02BED3FE00F
:10E2B00049EC50E4C701B6010E94C98C6093B911C2
:10E2C0007093BA118093BB119093BC11C090B91197
:10E2D000D090BA11E090BB11F090BC112BED3FE053
:10E2E00049EC50E4C701B6010E947E8E181684F4F2
:10E2F0002BED3FE049EC50E4C701B6010E94C88C09
:10E300006093B9117093BA118093BB119093BC11B3
:10E3100020E030E044E353E46091B9117091BA1108
:10E320008091BB119091BC110E949E8B2BED3FE020
:10E3300049E450E40E948F8D6093B5117093B6113B
:10E340008093B7119093B8110E94288E4AE0CE01B5
:10E35000C7960E948D4D6CE27BE0CE01C1960E9473
:10E36000C84DBE01695C7F4FCE01C1960E94134922
:10E3700066E37BE00E94FC48BC018BE890E10E94D0
:10E38000E94CCE01C1960E94FE4CCE01C7960E9478
:10E39000FE4CC090B511D090B611E090B711F0903E
:10E3A000B81120E030E044EB52E4C701B6010E940E
:10E3B000398B181694F020E030E040E05FE3C701AD
:10E3C000B6010E94C98C0E94288E4AE0CE01C796F1
:10E3D0000E948D4D6DE37BE023C020E030E044E3FC
:10E3E00053E4C701B6010E94398B1816A4F1A701A6
:10E3F000960160E070E884E393E40E94C88C609327
:10E40000B5117093B6118093B7119093B8110E9413
:10E41000288E4AE0CE01C7960E948D4D60E47BE0D5
:10E42000CE01C1960E94C84DBE01695C7F4FCE01EE
:10E43000C1960E941349BC01CE018B960E94E94C03
:10E44000CE01C1960E94FE4CCE01C7960E94FE4CA2
:10E4500066E777E063C020E030E047E853E4C701B7
:10E46000B6010E94398B181604F120E030E044E335
:10E4700053E4C701B6010E94C88C20E030E040E0C0
:10E480005FE30E94C98C6093B5117093B6118093BD
:10E49000B7119093B8110E94288E4AE0CE01C7961A
:10E4A0000E948D4D60E47BE01FC0A701960160E0F3
:10E4B00070E084EB93E40E94C88C20E030E040E000
:10E4C0005FE30E94C98C6093B5117093B61180937D
:10E4D000B7119093B8110E94288E4AE0CE01C796DA
:10E4E0000E948D4D6DE37BE0CE01C1960E94C84D28
:10E4F000BE01695C7F4FCE01C1960E941349BC01E9
:10E50000CE018B960E94E94CCE01C1960E94FE4C32
:10E51000CE01C7960E94FE4C63E47BE0CE01859657
:10E520000E94D44CBE01655D7F4FCE01C1960E9412
:10E53000C04D4AE050E060E070E0CE01C1964DDB96
:10E54000CE01C1960E94FE4C0E941251C090AD11A6
:10E55000D090AE11E090AF11F090B011A4E6CA0EC9
:10E56000D11CE11CF11CC616D706E806F90608F412
:10E5700023C20E9412510E943D8B6B017C0160916D
:10E58000AD117091AE118091AF119091B0110E94B8
:10E590003F8B20E030E048EC51E40E94C98C9B01A5
:10E5A000AC01C701B6010E94398B87FD05C264E04A
:10E5B0007BE0CE01C1960E94C84DBE016B5D7F4FCE
:10E5C000CE01C1960E941349BC01CE018B960E94D8
:10E5D0003249CE01C1960E94FE4CC80102970297B3
:10E5E00008F0C4C120E030E040E251E4C501B401CC
:10E5F0000E949E8B6B017C0120E030E040E251E400
:10E60000C301B2010E949E8B4B015C0120E030E00F
:10E6100040E251E427966CAD7DAD8EAD9FAD27975E
:10E620000E949E8B2B013C010E9412512091D80B1D
:10E630003091D90B4091DA0B5091DB0B621B730BBD
:10E64000840B950B0E943D8B20E030E04AE754E4B8
:10E650000E948F8DAB01BC0123E0CE01C7960E94C2
:10E66000324D69E57BE0CE01C1960E94C84DBE01E6
:10E67000695C7F4FCE01C1960E9413496CE776E03A
:10E680000E94FC48BC0189E790E10E94E94CCE0160
:10E69000C1960E94FE4CCE01C7960E94FE4C69E7CF
:10E6A00070E1CE01C1960E94C04D6BE870E1CE01D1
:10E6B000C1960E941349BE01655D7F4F0E941349B8
:10E6C000BC01CE018B960E94E94CCE01C1960E94FE
:10E6D000FE4C65E47BE085E890E10E94D44C21E0AB
:10E6E000B701A601CE01C1960E94324DBE016F5CFA
:10E6F0007F4F85E890E10E943249CE01C1960E9489
:10E70000FE4C21E0B301A201CE01CD960E94324D14
:10E7100021E0B501A401CE01C7960E94324D64E00C
:10E720007BE0CE01C1960E94C84DBE01695C7F4F5F
:10E73000CE01C1960E94134964E07BE00E94FC4830
:10E74000BE01635C7F4F0E94134960E57BE00E943D
:10E75000FC48BC0185E890E10E943249CE01C19697
:10E760000E94FE4CCE01C7960E94FE4CCE01CD9673
:10E770000E94FE4CA7019601C701B6010E949E8B24
:10E780006B017C01A5019401C501B4010E949E8B1F
:10E790009B01AC01C701B6010E94C98C6B017C01D1
:10E7A000A3019201C301B2010E949E8B9B01AC01A7
:10E7B000C701B6010E94C98C0E948D8F6B017C013C
:10E7C0006093B1117093B2118093B3119093B4110F
:10E7D00064E57BE085E890E10E94244921E0B701EF
:10E7E000A601CE01C1960E94324DBE016F5C7F4FE3
:10E7F000CE01C7960E94C04D65E67BE0CE01C7966C
:10E800000E94FC48BC018BE890E10E94E94CCE01DB
:10E81000C7960E94FE4CCE01C1960E94FE4C6BE84A
:10E8200070E185E890E10E943249C090B111D0902A
:10E83000B211E090B311F090B41120E030E04AE75B
:10E8400054E4C701B6010E947E8E87FD29C020E0F6
:10E8500030E04AE754E4C701B6010E948F8DAB0156
:10E86000BC0123E0CE01C1960E94034DBE016F5C46
:10E870007F4FCE01C7960E94C04D66E67BE0CE0179
:10E88000C7960E94FC48BC018BE890E10E94E94CCD
:10E89000CE01C7960E94FE4CCE01C1960E94FE4C4E
:10E8A00020E030E64AE656E46091B1117091B21171
:10E8B0008091B3119091B4110E94398BBE01655DB6
:10E8C0007F4F87FF4FC0CE01C1960E94C04D68E5C3
:10E8D0007BE0CE01C1960E94FC4865E870E10E9491
:10E8E0001349BC0185E890E10E94E94CCE01C19634
:10E8F0000E94FE4C03301105A1F465E870E1CE01E1
:10E90000C1960E94C04DCE01C1960E94F06ACE0110
:10E91000C1960E94FE4C6CED7AE085E890E10E9481
:10E92000D44C6BE57BE0CE01C1960E94C84D6BE8EC
:10E9300070E1CE01C1960E941349BC01CE01C79679
:10E940000E94C04D4AE050E06FEF7FEFCE01C796C6
:10E9500013D8CE01C7960E94FE4CCE01C1960E94EC
:10E96000FE4C04C085E890E10E94E94C6AE070E04A
:10E9700080E090E00E94DA50CE0185960E94FE4C25
:10E98000CE018B960E94FE4CCA5BDF4F0FB6F89407
:10E99000DEBF0FBECDBFDF91CF911F910F91FF90D2
:10E9A000EF90DF90CF90BF90AF909F908F907F902F
:10E9B0006F905F904F9008956CED7AE0CE01C19614
:10E9C0000E94C84DCE01C1960E947C6CCE01C196BA
:10E9D0000E94FE4CBE016B5D7F4F8BE891E10E946F
:10E9E000E34DE5CD1F93CF93DF93CDB7DEB7A89767
:10E9F0000FB6F894DEBF0FBECDBF182F0E94AD62D8
:10EA00008EE10E94886162E08AE99FE00E948B5952
:10EA100060E08AE99FE00E948B590E9427618EE1A5
:10EA20000E94886161E08AE99FE00E948B5960E260
:10EA30008AE99FE00E948B590E94276180E290E062
:10EA40009093BE108093BD1080E090E8A9E8B4E4F4
:10EA50008093560290935702A0935802B0935902A4
:10EA600080E090E0A5E7B4E48093520290935302D3
:10EA7000A0935402B0935502BE016F5F7F4F8AEBA3
:10EA800090E10E94074B112309F49CC080914E0C29
:10EA9000882309F497C067ED7EE08DEF9EE00E9429
:10EAA000F14D8DEF9EE00E94BF4E67EC7EE08DEF52
:10EAB0009EE00E94F14DBE016F5F7F4F8DEF9EE0A3
:10EAC0000E94C24E67EB7EE08DEF9EE00E94F14D0A
:10EAD0004D855E856F8578892AE030E08DEF9EE078
:10EAE0000E94724E8DEF9EE00E94BF4E67EA7EE06C
:10EAF0008DEF9EE00E94F14D49895A896B897C898E
:10EB00002AE030E08DEF9EE00E94724E8DEF9EE095
:10EB10000E94BF4E67E97EE08DEF9EE00E94F14DBE
:10EB200020E030E040E251E4698D7A8D8B8D9C8D40
:10EB30000E949E8B42E050E00E94AC6264E67BE063
:10EB40008DEF9EE00E94C24E67E87EE08DEF9EE072
:10EB50000E94F14D20E030E040E251E46D8D7E8D69
:10EB60008F8D98A10E949E8B42E050E00E94AC6283
:10EB700064E67BE08DEF9EE00E94C24E67E77EE098
:10EB80008DEF9EE00E94F14D20E030E040E251E444
:10EB900069A17AA18BA19CA10E949E8B42E050E0CA
:10EBA0000E94AC6264E67BE08DEF9EE00E94C24E64
:10EBB00061E57EE08DEF9EE00E94F14D8DEF9EE0DD
:10EBC0000E94BF4E64EF71E080E090E00E94DA5056
:10EBD000A8960FB6F894DEBF0FBECDBFDF91CF91E0
:10EBE0001F9108952F923F924F925F926F927F9262
:10EBF0008F929F92AF92BF92CF92DF92EF92FF924D
:10EC00000F931F93CF93DF93CDB7DEB7C954D109CC
:10EC10000FB6F894DEBF0FBECDBF2B013C01279687
:10EC20002FAF279728963FAF289729964FAF299760
:10EC30002A965FAF2A970E94125122966CAF7DAF41
:10EC40008EAF9FAF229727962FAD279728963FAD7F
:10EC5000289729964FAD29972A965FAD2A9780E984
:10EC6000481681E058066104710434F060E9462ECC
:10EC700055245394612C712C203197E239074105BA
:10EC800051052CF42DA73EA74FA758AB0AC090E121
:10EC9000C92E97E2D92EE12CF12CCDA6DEA6EFA647
:10ECA000F8AA8091820C882321F02DA73EA74FA7B8
:10ECB00058AB22966CAD7DAD8EAD9FAD229728EE00
:10ECC00033E040E050E00E946B8C26962CAF3DAFC5
:10ECD0004EAF5FAF269721E02DAB19A61AA61BA653
:10ECE0001CA68E01035F1F4FCC24DD247601C418BF
:10ECF000D508E608F708C9AADAAAEBAAFCAAC9A4AB
:10ED0000DAA4EBA4FCA42DA53EA54FA558A9C216D4
:10ED1000D306E406F5060CF033C369A57AA58BA5E6
:10ED20009CA50E943F8B20E030E04AE754E40E941B
:10ED30008F8DAB01BC0123E0C8010E94324DB801A8
:10ED40008FE790E10E94434CC8010E94FE4C2DA524
:10ED50003EA54FA558A92A3031054105510594F427
:10ED60002AE026964CAD5DAD6EAD7FAD2697C8010D
:10ED70000E94614DB8018FE790E10E94434CC801A9
:10ED80000E94FE4CCE0101960E94075568E67BE08A
:10ED900085E890E10E94D44CAE014F5F5F4F1A01AD
:10EDA000C12CD12C7601D1018D909D90AD90BD905C
:10EDB0001D01A5019401C501B4010E949E8B9B0118
:10EDC000AC01C701B6010E94C98C6B017C0123E034
:10EDD000B501A401C8010E94034DB801CE014396BC
:10EDE0000E94C04D64E07BE0CE0143960E94FC4847
:10EDF000BC0185E890E10E943249CE0143960E9411
:10EE0000FE4CC8010E94FE4C2016310661F6C70177
:10EE1000B6010E948D8F6B017C01BDE24B16B1E003
:10EE20005B066104710434F00E94586C60E080E07D
:10EE30000E94A36123E0B701A601CE0143960E9480
:10EE4000324D68E57BE0C8010E94C84D6FE770E174
:10EE5000C8010E94134965E77BE00E94FC48BE019F
:10EE60006D5E7F4F0E9413496AE77BE00E94FC4879
:10EE7000BC0185E890E10E943249C8010E94FE4C25
:10EE8000CE0143960E94FE4C2DEC3CEC4CE45FE33B
:10EE9000C701B6010E947E8E29813A814B815C8137
:10EEA0002DA33EA34FA358A718160CF0ACC12AE916
:10EEB00039E949E95FE3C701B6010E94398B87FF51
:10EEC000A2C1CDA8CC2009F49EC189849A84AB84C8
:10EED000BC8420E030E0A901C501B4010E94398B57
:10EEE000CD80DE80EF80F884882309F12DA13EA13A
:10EEF0004FA158A5CA01B9010E949E8B6EAB7FAB92
:10EF000088AF99AFA7019601C701B6010E949E8BF9
:10EF10009B01AC016EA97FA988AD99AD0E94C98CF7
:10EF20000E948D8FA50194010E943C8D04C06BED61
:10EF30007FE089EC9FE320EE3EE245E652E40E944A
:10EF40009E8B6EAB7FAB88AF99AF20E030E0A9011C
:10EF5000C701B6010E94398B882309F12DA13EA17A
:10EF60004FA158A5CA01B9010E949E8B6AAF7BAF21
:10EF70008CAF9DAFA5019401C501B4010E949E8B89
:10EF80009B01AC016AAD7BAD8CAD9DAD0E94C98C7F
:10EF90000E948D8FA70196010E943C8D04C06BEDED
:10EFA0007FE089EC9FE320EE3EE245E652E40E94DA
:10EFB0009E8B6AAF7BAF8CAF9DAF20E030E0A901A4
:10EFC0006DA17EA18FA198A50E94398B8823F9F0AD
:10EFD000A5019401C501B4010E949E8B4B015C0107
:10EFE000A7019601C701B6010E949E8B9B01AC014F
:10EFF000C501B4010E94C98C0E948D8F2DA13EA134
:10F000004FA158A50E943C8D6B017C0108C08BED7F
:10F01000C82E8FE0D82E89ECE82E8FE3F82E69E514
:10F020007BE0C8010E94C84D6FE770E1C8010E94F3
:10F0300013496DE77BE00E94FC48BC0185E890E144
:10F040000E94E94CC8010E94FE4C69E57BE0C801C2
:10F050000E94C84D6FE770E1C8010E94134967E93B
:10F060007BE00E94FC48BC018FE790E10E94E94CE4
:10F07000C8010E94FE4C21E04EA95FA968AD79ADA0
:10F08000CE014F960E94324D21E04AAD5BAD6CAD92
:10F090007DADCE0149960E94324D20EE3EE245E61E
:10F0A00052E4C701B6010E949E8BAB01BC0121E076
:10F0B000C8010E94324DB801CE0143960E94C04D56
:10F0C00064E07BE0CE0143960E94FC48BE01675E8F
:10F0D0007F4F0E94134964E07BE00E94FC48BE0120
:10F0E000615E7F4F0E941349BC0189E790E10E9455
:10F0F000E94CCE0143960E94FE4CC8010E94FE4C92
:10F10000CE0149960E94FE4CCE014F960E94FE4CC5
:10F110002DE2421621E052066104710474F469A5DF
:10F120007AA58BA59CA525E030E040E050E00E9448
:10F130006B8C672B682B692BC1F56FE770E1C801F9
:10F140000E94C04D45E050E06FEF7FEFC8010E9484
:10F150003B6DC8010E94FE4C60EA7BE0C8010E9442
:10F16000C84D45E050E061EF7FEFC8010E94ED6DB2
:10F17000C8010E94FE4C6CED7AE0C8010E94C84DA7
:10F18000C8010E947C6CC8010E94FE4C69E770E1D6
:10F19000C8010E94C04D45E050E060E070E0C80149
:10F1A0000E94BC6CC8010E94FE4C69E770E185E8D2
:10F1B00090E10E9432493FE1431651046104710419
:10F1C00034F4C9A4DAA4EBA4FCA4F7FC11C065E8EC
:10F1D00070E1C8010E94C04DC8010E94F06AC801D8
:10F1E0000E94FE4C6CED7AE085E890E10E94D44CE0
:10F1F000B201C30177FE04C069A97AA98BA99CA9B1
:10F200000E94DA50AAC023E04DA15EA16FA178A5AB
:10F21000CE0143960E94324D69E57BE0C8010E9411
:10F22000C84D6FE770E1C8010E94134962EA7BE0B4
:10F230000E94FC48BE016D5E7F4F0E9413496BE740
:10F240007BE00E94FC48BC018FE790E10E94E94C02
:10F25000C8010E94FE4CCE0143960E94FE4C498597
:10F260005A856B857C8523E0CE0149960E94034D2B
:10F270004D815E816F81788523E0C8010E94034D36
:10F28000B801CE0143960E94C04D67EA7BE0CE01F3
:10F2900043960E94FC48BE01675E7F4F0E9413495F
:10F2A0006BE77BE00E94FC48BC0189E790E10E948B
:10F2B000E94CCE0143960E94FE4CC8010E94FE4CD0
:10F2C000CE0149960E94FE4C2DE2421621E05206E4
:10F2D0006104710474F469A57AA58BA59CA525E049
:10F2E00030E040E050E00E946B8C672B682B692B6C
:10F2F000F1F46FE770E1C8010E94C04D4AE050E0B0
:10F300006FEF7FEFC8010E943B6DC8010E94FE4C69
:10F3100069E770E1C8010E94C04D4AE050E060E03A
:10F3200070E0C8010E94BC6CC8010E94FE4C65E8F8
:10F3300070E1C8010E94C04DC8010E94F06AC80176
:10F340000E94FE4C6CED7AE085E890E10E94D44C7E
:10F35000C301B2010E94DA501DAA0E9412516B0132
:10F360007C0122962CAD3DAD4EAD5FAD2297C21A09
:10F37000D30AE40AF50AC9A6DAA6EBA6FCA6BFCC16
:10F380006FE770E1CE010D960E94C04D4AE050E05B
:10F390006FEF7FEFCE010D960E94ED6DCE010D96C1
:10F3A0000E94FE4CCDA8CC20B1F160EA7BE0CE01FA
:10F3B0000D960E94C84D45E050E061EF7FEFCE0111
:10F3C0000D960E94ED6DCE010D960E94FE4C80912F
:10F3D000820C882391F062E07FE0CE010D960E94BE
:10F3E000B84D45E050E060E070E0CE010D960E941F
:10F3F000ED6DCE010D960E94FE4C6CED7AE0CE01D3
:10F400000D960E94C84DCE010D960E947C6CCE01D7
:10F410000D960E94FE4C69E770E1CE010D960E94A8
:10F42000C04D4AE050E06FEF7FEFCE010D960E9495
:10F43000BC6CCE010D960E94FE4CC75BDF4F0FB631
:10F44000F894DEBF0FBECDBFDF91CF911F910F911A
:10F45000FF90EF90DF90CF90BF90AF909F908F90F4
:10F460007F906F905F904F903F902F9008956F9294
:10F470007F928F929F92AF92BF92CF92DF92EF9244
:10F48000FF920F931F93CF93DF9381E080937911C5
:10F490000E9412510091691110916A1120916B1113
:10F4A00030916C11AB01BC01401B510B620B730B13
:10F4B0008091751190917611A0E0B0E084179507C6
:10F4C000A607B70708F00BC1C0E080917311C817F9
:10F4D00060F4E0916F11F0917011EC0FF11D62E09A
:10F4E00080810E945450CF5FF0CF712C812C912CE1
:10F4F0005401839480917411781608F05FC0072D31
:10F5000010E0E0917111F0917211E00FF11F61E0D4
:10F5100080810E945450E0917111F0917211E00FBE
:10F52000F11F60E080810E942550D501C401072CA5
:10F5300004C0880F991FAA1FBB1F0A94D2F76C0141
:10F540007C01E094F094612C809173116816F8F4BA
:10F55000C62DD0E0E0916F11F0917011EC0FFD1FFE
:10F5600080810E94FB4F2496CC0FDD1FC35FDE4ECF
:10F57000892B29F4888199818C299D2904C088814F
:10F5800099818E219F21998388836394DDCFE091B7
:10F590007111F0917211E00FF11F61E080810E9402
:10F5A00025508091711190917211FC01E00FF11FB3
:10F5B00060E080810E94545073949CCFE9E2F1E1B5
:10F5C0008FEF9FEF23813481232B21F410829283CC
:10F5D00081831582369621E1E536F20799F710E02E
:10F5E00096E0F92E80917311181708F052C000E0D0
:10F5F000C12FD0E0CC0FDD1FCB5EDE4E2091741109
:10F60000021708F044C068817981002E02C0769507
:10F6100067950A94E2F761707727129F9001112491
:10F62000200F311DE0916D11F0916E11E20FF31F6B
:10F630004081EDE0F1E180E0A58DB68DA217B30722
:10F6400011F461701AC08F5F36968A30A9F7672B64
:10F65000E1F0E9E2F1E180E090E05081511110C069
:10F66000F89EF001F99EF00D1124E35FFE4E448FE9
:10F67000368F258F10A2178E61E00E94E15805C0D9
:10F68000019636968A30910541F70F5FB7CF1F5F1D
:10F69000A9CF80E090E0C0E0FC01E35FFE4E21A135
:10F6A0002111C1E006968C339105B1F70E941251E9
:10F6B0006093691170936A1180936B1190936C1130
:10F6C000CC2369F080912E11882349F080912C1170
:10F6D00090912D11019719F48091291103C0109276
:10F6E000791180E0DF91CF911F910F91FF90EF9002
:10F6F000DF90CF90BF90AF909F908F907F906F9052
:10F7000008958F929F92AF92BF92CF92DF92EF9225
:10F71000FF920F931F93CF93DF93DB01CD91DC9189
:10F72000DC011C96ED91FC911D97CE17DF070CF0C4
:10F730004AC0FE01EE0FFF1F1A968D919C911B97F8
:10F74000E80FF91F80809180C170DD27B1E0CB27E1
:10F75000209719F404E610E002C00CE91FEF7901CC
:10F760005A016B01020F131FB801C4010E944446E5
:10F77000892B99F40E0D1F1DB801C4010E94444647
:10F78000892B71F4B8016E0D7F1DC4010E9444469F
:10F79000892BE1F023E030E005C021E030E002C039
:10F7A00022E030E0F5018081918101968217930774
:10F7B00034F011821082F60180819181019691834B
:10F7C0008083CE0105C081E090E002C08FEF9FEF03
:10F7D000DF91CF911F910F91FF90EF90DF90CF902D
:10F7E000BF90AF909F908F9008950895CF92DF9231
:10F7F000EF92FF920F931F93CF93DF93EC016A0177
:10F800007B01E889F98982E080834115514E6105C9
:10F810007105B1F060E079E08DE390E0A701960119
:10F820000E94978C89019A0101501109210931091F
:10F830003695279517950795980101151041A8F061
:10F84000E889F989108260E874E88EE190E0A70108
:10F8500096010E94978CDA01C9010197A109B109AB
:10F86000B695A795979587959C01EC85FD85308386
:10F87000EE85FF852083188EEC89FD8986E08083E4
:10F88000EA89FB89808180618083EA89FB898081A4
:10F8900088608083EA89FB89808180688083EA8927
:10F8A000FB8980818F7D8083DF91CF911F910F91A4
:10F8B000FF90EF90DF90CF900895CF92DF92EF927C
:10F8C000FF920F931F93E82FF92F05C001501109E4
:10F8D0002109310961F1908196239417B9F305C08C
:10F8E000015011092109310911F1908196239413D6
:10F8F000F7CFC12CD12CE12CF12C0AC08FEFC81A04
:10F90000D80AE80AF80A0C151D052E053F0579F0FE
:10F9100080818623841791F36C2D7D2D8E2D9F2D54
:10F920001F910F91FF90EF90DF90CF90089560E0CE
:10F9300070E080E090E01F910F91FF90EF90DF90DA
:10F94000CF900895CF93DF93CDB7DEB72C970FB646
:10F95000F894DEBF0FBECDBF789484B5826084BDBD
:10F9600084B5816084BD85B5826085BD85B58160C3
:10F9700085BD80916E00816080936E001092810041
:10F9800080918100826080938100809181008160FC
:10F9900080938100809180008160809380008091BD
:10F9A000B10084608093B1008091B0008160809349
:10F9B000B0008091910082608093910080919100CD
:10F9C000816080939100809190008160809390008D
:10F9D0008091A10082608093A1008091A10081604C
:10F9E0008093A1008091A00081608093A00080910D
:10F9F00021018260809321018091210181608093A7
:10FA000021018091200181608093200180917A0002
:10FA1000846080937A0080917A00826080937A007B
:10FA200080917A00816080937A0080917A0080686A
:10FA300080937A001092C10061E089E10E945450E5
:10FA400061E089E10E9425500E94AD6261E27AE0A6
:10FA50008DEF9EE00E94C24E67E2C62ED12CE12CB3
:10FA6000F12C00E010E08C2D0E9488610E9427613B
:10FA7000811127C06DE27AE08DEF9EE00E94E24E98
:10FA800020E1B701A6018DEF9EE00E942A4E8DEF86
:10FA90009EE00E94BF4EC0928F1169E47AE08DEF24
:10FAA0009EE00E94E24E20E1B701A6018DEF9EE0AC
:10FAB0000E942A4E8DEF9EE00E94BF4E0F5F1F4FA7
:10FAC00013C0843089F463E67AE08DEF9EE00E94F3
:10FAD000E24E20E1B701A6018DEF9EE00E942A4E82
:10FAE0008DEF9EE00E94BF4E8FEFC81AD80AE80A39
:10FAF000F80AE0E4CE16D104E104F10409F0B3CF32
:10FB0000012B19F46EE77AE002C064E97AE08DEF28
:10FB10009EE00E94C24E0E949E5780E40E94926125
:10FB20000AE412E0F80161918F018BE891E10E94F3
:10FB30007145F2E002351F07A9F70E94586C0E9438
:10FB4000D95B8EED93E09093780C8093770C0E94B4
:10FB5000558C8093250D8FED93E00E94558C8093FA
:10FB6000260D8091250D9091260D1816190654F436
:10FB700010924902019731F41092260D1092250D32
:10FB80000E94126560E37AE0CE0101960E94B84DB2
:10FB90004AE050E06FEF7FEFCE0101960E94ED6DDD
:10FBA000CE0101960E94FE4C40E052EC61E070E014
:10FBB0008DEF9EE01BDE80914902882331F068EED4
:10FBC00073E080E090E00E94DA508DEF9EE00E94AA
:10FBD000B249F82E82E7F81609F44EC11092780C5B
:10FBE0001092770C5BEAC52E5CE0D52E00E010E0A9
:10FBF000C8010E94558CF60181936F010F5F1F4F62
:10FC00000A371105A9F78091AB0C9091AC0CA0912B
:10FC1000AD0CB091AE0C85369105A105B1050CF483
:10FC20002BC18093450290934602A0934702B09364
:10FC300048028091AF0C9091B00CA091B10CB091A2
:10FC4000B20C8093410290934202A0934302B0937E
:10FC500044028091B30C9091B40CA091B50CB0917A
:10FC6000B60C80933D0290933E02A0933F02B09366
:10FC7000400267EC7CE0CE0101960E94C84DBE01B7
:10FC80006F5F7F4F85E891E10E94434CCE01019662
:10FC90000E94FE4C8091B70C9091B80CA091B90CC9
:10FCA000B091BA0C8093390290933A02A0933B0230
:10FCB000B0933C028091BB0C9091BC0CA091BD0C08
:10FCC000B091BE0C8093350290933602A093370218
:10FCD000B09338028091BF0C9091C00CA091C10CE0
:10FCE000B091C20C8093310290933202A093330200
:10FCF000B09334028091C30C9091C40CA091C50CB8
:10FD0000B091C60C80932D0290932E02A0932F02E7
:10FD1000B09330028091CF0C9091D00CA091D10C77
:10FD2000B091D20C8093C2049093C304A093C404F6
:10FD3000B093C5048091D30C9091D40CA091D50CB4
:10FD4000B091D60C8093BE049093BF04A093C004DE
:10FD5000B093C1048091D70C9091D80CA091D90C8C
:10FD6000B091DA0C8093BA049093BB04A093BC04C6
:10FD7000B093BD048091DB0C9091DC0CA091DD0C64
:10FD8000B091DE0C8093B6049093B704A093B804AE
:10FD9000B093B9048091DF0C9091E00CA091E10C3C
:10FDA000B091E20C8093290290932A02A0932B0237
:10FDB000B0932C028090F50C9090F60CA090F70C6C
:10FDC000B090F80CA5019401C501B4010E94CE8F3A
:10FDD000811108C08092250290922602A0922702EB
:10FDE000B09228026091210D7091220D072E000C17
:10FDF000880B990B0E943F8B9B01AC010E94CE8F18
:10FE0000882321F01092220D1092210D0091230DD4
:10FE10001091240DB801012E000C880B990B0E9443
:10FE20003F8B9B01AC010E94CE8F811104C01093C7
:10FE300024020093230200E010E0F801E750F34FA2
:10FE400080809180A280B380A5019401C501B40196
:10FE50000E94CE8F811107C0F801E15BF34F8082D1
:10FE60009182A282B3820C5F1F4F0832110529F7DD
:10FE700081E090E00E94305D4EE8E42EEF0CF1E06E
:10FE8000FE1570F48091AB0C9091AC0CA091AD0C70
:10FE9000B091AE0C85369105A105B1050CF05EC19F
:10FEA0008091450290914602A0914702B09148028C
:10FEB0008093AB0C9093AC0CA093AD0CB093AE0CB4
:10FEC0008091410290914202A0914302B09144027C
:10FED0008093AF0C9093B00CA093B10CB093B20C84
:10FEE00080913D0290913E02A0913F02B09140026C
:10FEF0008093B30C9093B40CA093B50CB093B60C54
:10FF000082E7F81220C087EC9CE0892BE1F0009199
:10FF1000891110918A110115110519F41092C70C5D
:10FF200012C00730110510F007E010E06091851154
:10FF300070918611A80187EC9CE00E948F92F801D5
:10FF4000E953F34F10828091390290913A02A091C7
:10FF50003B02B0913C028093B70C9093B80CA093F5
:10FF6000B90CB093BA0C8091350290913602A091F1
:10FF70003702B09138028093BB0C9093BC0CA093D5
:10FF8000BD0CB093BE0C8091310290913202A091D1
:10FF90003302B09134028093BF0C9093C00CA093B5
:10FFA000C10CB093C20C80912D0290912E02A091B1
:10FFB0002F02B09130028093C30C9093C40CA09395
:10FFC000C50CB093C60C8091C2049091C304A0915B
:10FFD000C404B091C5048093CF0C9093D00CA0932F
:10FFE000D10CB093D20C8091BE049091BF04A0912B
:10FFF000C004B091C1048093D30C9093D40CA0930F
:020000021000EC
:10000000D50CB093D60C8091BA049091BB04A0910A
:10001000BC04B091BD048093D70C9093D80CA093EE
:10002000D90CB093DA0C8091B6049091B704A091EA
:10003000B804B091B9048093DB0C9093DC0CA093CE
:10004000DD0CB093DE0C8091290290912A02A091E0
:100050002B02B0912C028093DF0C9093E00CA093C4
:10006000E10CB093E20C8091250290912602A091C0
:100070002702B09128028093F50C9093F60CA09380
:10008000F70CB093F80C8091230290912402909386
:10009000240D8093230DEFE4FCE0A9EFBCE0419137
:1000A0005191619171914D935D936D937D938CE02E
:1000B000E737F807A1F76AE17AE0CE0101960E94DE
:1000C000B84DCE0101960E94BD70CE0101960E94EE
:1000D000FE4C21E1C22E22E0D22E33EEA32E3CE0D4
:1000E000B32E00E010E0809111029091120280176F
:1000F00091074CF1F60180819181F50181939193F3
:100100005F0180914E0C8823C1F06EE97AE08DEF9B
:100110009EE00E94E24E4AE050E0B8018DEF9EE082
:100120000E94B94E6BE97AE08DEF9EE00E94E24EAC
:10013000F601808191810E9488540F5F1F4FF2E089
:10014000CF0ED11CD0CF81E08E1540F01092780CEC
:100150001092770C80E090E00E9439658091210D2B
:100160009091220D892B39F440E855E260E070E06F
:1001700083EC9DE03BDB8091210D9091220D019756
:1001800039F440E052EC61E070E083EC9DE02EDB5E
:1001900064E670E080E090E00E94DA5064E670E08F
:1001A00080E090E00E94DA50F89482E08093B00002
:1001B0008093B10094E69093B3001092B2008093C4
:1001C000700078948093A60F1092AA0F8091A70FC9
:1001D00060E00E94545060EA7AE0CE0101960E94ED
:1001E000C84D4AE050E06FEF7FEFCE0101960E94CC
:1001F000ED6DCE0101960E94FE4C8091210D9091F3
:10020000220D892B09F561E17AE0CE0107960E9463
:10021000C84D65E871E1CE0107960E941349BC0103
:10022000CE0101960E94C04D4AE050E06FEF7FEF93
:10023000CE0101960E94BC6CCE0101960E94FE4C3C
:10024000CE0107960E94FE4C8091210D9091220DC7
:10025000019709F56DEF79E0CE0107960E94C84D30
:1002600065E871E1CE0107960E941349BC01CE01F9
:1002700001960E94C04D4AE050E06FEF7FEFCE0143
:1002800001960E94BC6CCE0101960E94FE4CCE01EC
:1002900007960E94FE4C6EE97AE0CE0107960E9416
:1002A000C84D65E871E1CE0107960E94134960EBE5
:1002B0007AE00E94FC48BC01CE0101960E94C04D2C
:1002C000CE0101960E94F06ACE0101960E94FE4C7A
:1002D000CE0107960E94FE4C64E670E080E090E05C
:1002E0000E94DA500E94AD6264E670E080E090E027
:1002F0000E94DA5083E20E94886181E090E00E94CF
:1003000084610E94276183E090E090934D0C80937C
:100310004C0C8CE40E947E554B015C0162E370E062
:1003200080E090E00E94DA50A5019401C501B4017B
:100330000E94CE8F882309F478C086E60E947E55FD
:100340004B015C0162E370E080E090E00E94DA50D3
:10035000A5019401C501B4010E94CE8F882309F440
:1003600064C081E090E090934D0C80934C0C40E091
:1003700052EC61E070E080E69EE038DA64E670E01E
:1003800080E090E00E94DA5080E69EE00E94D94F23
:1003900040E052EC61E070E080E69EE027DA8CED10
:1003A00095E0A0E0B0E08093640E9093650EA0937A
:1003B000660EB093670E64E670E080E090E00E9405
:1003C000DA5092E0C92ED12CE12C65E070E080E09B
:1003D00090E00E94DA5000E010E0812C912C540152
:1003E000E11056C180E69EE00E94D449892B39F481
:1003F000F5E18F169104A104B1040CF049C103305A
:1004000011050CF48AC144C1EE2009F44FC161E02A
:100410007AE0CE0101960E94B84DCE0101960E946D
:10042000BD70CE0101960E94FE4C80914C0C9091C3
:100430004D0C039771F462ED79E0CE0101960E94B4
:10044000B84DCE0101960E94BD70CE0101960E946A
:10045000FE4C83E08093A3100E94AD6280ED0E9469
:10046000B765853509F084C18AEA0E94DA65909300
:10047000A5108093A4108CEA0E94DA659093A710CF
:100480008093A6108EEA0E94DA659093A91080935B
:10049000A81080EB0E94DA659093B5108093B41099
:1004A00082EB0E94DA659093B7108093B61084EBCC
:1004B0000E94DA659093B9108093B81086EB0E9481
:1004C000DA659093AB108093AA1088EB0E94DA65EE
:1004D0009093AD108093AC108AEB0E94DA659093F4
:1004E000AF108093AE108CEB0E94DA659093B11040
:1004F0008093B0108EEB0E94DA659093B3108093D6
:10050000B21069E979E085E890E10E9438490E94DB
:100510008B510E943F8B0E94288E0E943F8B20E0CF
:1005200030E048EC52E40E948F8DAB01BC0122E028
:10053000CE0107960E94324DBE01695F7F4FCE010A
:1005400001960E94C04D6BE077E0CE0101960E94BB
:10055000FC48BC0185E890E10E943249CE01019639
:100560000E94FE4CCE0107960E94FE4C65E870E1A9
:10057000CE0101960E94C04DCE0101960E94BD7031
:10058000CE0101960E94FE4C63E879E085E890E197
:100590000E9438496091450270914602809147025D
:1005A000909148020E943F8B20E030E048EC52E4FA
:1005B0000E948F8DAB01BC0122E0CE0107960E9404
:1005C000324DBE01695F7F4FCE0101960E94C04D42
:1005D0006BE077E0CE0101960E94FC48BC0185E803
:1005E00090E10E943249CE0101960E94FE4CCE015C
:1005F00007960E94FE4C65E870E1CE0101960E94CC
:10060000C04DCE0101960E94BD70CE0101960E94A0
:10061000FE4C81E6F81205C081E00E94D13B81E0EA
:1006200011C08DEF9EE00E94B249182F64E670E081
:1006300080E090E00E94DA50113671F380E00E9471
:10064000D13B80E00E94F27464E670E080E090E0CC
:100650000E94DA5010914902112331F068EE73E0E4
:1006600080E090E00E94DA5065E875E081E990E171
:100670000E94D44C82E090E090934B0C80934A0C03
:1006800011110E9452680E94B9070E94834AFBCF51
:1006900064E670E080E090E00E94DA50CA94CD28D1
:1006A00009F4B2CECC24C394D12C8FCE10924D0C31
:1006B00010924C0C80E69EE00E94D94F64E670E0F8
:1006C00080E090E00E94DA5040E855E260E070E09F
:1006D00080E69EE08BD880E69EE00E94D449892B7C
:1006E00009F4A3CE67EE79E0CE0101960E94B84DE1
:1006F000CE0101960E94BD70CE0101960E94FE4C73
:1007000082E090E090934D0C80934C0C64E670E096
:1007100080E090E00E94DA5088CE80E69EE00E9461
:10072000D449892B69F080E69EE00E94B249E1E05D
:10073000F0E0EC0FFD1FE00FF11F80830F5F1F4FF4
:1007400065E070E080E090E00E94DA500230110530
:100750004CF089818B3B31F4EE24E3948A818A3A10
:1007600009F0E12CEFEF8E1A9E0AAE0ABE0A38CECF
:100770006CEA79E0CE0101960E94B84DCE01019657
:100780000E94F06ACE0101960E94FE4C1092100267
:100790005BCF89E790E10E94FE4C8FE790E10E94D9
:1007A000FE4C85E890E10E94FE4C8BE890E10E94AF
:1007B000FE4C81E990E10E94FE4C87E990E10E94A5
:1007C000FE4C8DE990E10E94FE4C85EE90E10E9486
:1007D000FE4C8FE791E10E94FE4C85E891E10C947C
:1007E000FE4CCF92DF92EF92FF921F93CF93DF9355
:1007F000182FCAE0D0E0C12CD12C7601812F0E94A5
:100800009050BC01990F880B990B39D79B01AC0113
:10081000C701B6010E94C98C6B017C0162E370E0E4
:1008200080E090E00E94DA50219741F720E030E02C
:1008300040E251E4C701B6010E948F8D20E030E014
:1008400040EA50E47BD720E030E040E85AE376D736
:10085000DF91CF911F91FF90EF90DF90CF9008959F
:100860008F929F92AF92BF92CF92DF92EF92FF92C0
:100870001092C60D1092C50D88EE93E0A0E0B0E096
:100880008093C70D9093C80DA093C90DB093CA0D66
:100890002AE035E03093C40D2093C30D45E351E0C9
:1008A0005093D00D4093CF0D44E351E05093D20DBF
:1008B0004093D10D40E351E05093D40D4093D30DBC
:1008C00041E351E05093D60D4093D50D42E351E002
:1008D0005093D80D4093D70D46E351E05093DA0D75
:1008E0004093D90D1092DC0D1092DD0D1092DE0DAB
:1008F0001092DF0D1092630E1092620E8093640EC0
:100900009093650EA093660EB093670E3093610EC0
:100910002093600E45ED50E050936D0E40936C0EA9
:1009200044ED50E050936F0E40936E0E40ED50E05A
:100930005093710E4093700E41ED50E05093730E42
:100940004093720E42ED50E05093750E4093740E3A
:1009500046ED50E05093770E4093760E1092790E4C
:1009600010927A0E10927B0E10927C0E1092000F55
:100970001092FF0E8093010F9093020FA093030F2C
:10098000B093040F3093FE0E2093FD0E25EC30E063
:1009900030930A0F2093090F24EC30E030930C0FB2
:1009A00020930B0F20EC30E030930E0F20930D0FAF
:1009B00021EC30E03093100F20930F0F22EC30E049
:1009C0003093120F2093110F26EC30E03093140F68
:1009D0002093130F1092160F1092170F1092180FEA
:1009E0001092190F10929D0F10929C0F80939E0FE2
:1009F00090939F0FA093A00FB093A10F8CE195E06F
:100A000090939B0F80939A0F10928E1110928D11DC
:100A100088E395E090938C1180938B1110928F1145
:100A200084E18093931184E0809394111092951146
:100A300088E08093961162E17BE085E891E10E9475
:100A4000C84D68E17BE08FE791E10E94C84D88E1E5
:100A500080937C1181E180937D1180E180937E11F0
:100A600061E088E10E94545061E080917C110E9415
:100A7000255060E080917D110E94545060E080918B
:100A80007E110E94545061E080917D110E9425509A
:100A900061E080917E110E94255061E080917C117F
:100AA0000E94255010920F111092131110921211E2
:100AB000109214118EE295E090930E1180930D1117
:100AC00080E090E0FC01E35FFE4E148E10A2178ED2
:100AD00011A206968C339105A9F78CEC94E09093C3
:100AE000701180936F1188EC94E090937211809351
:100AF000711184E0809373118093741180ED94E000
:100B000090936E1180936D118AE090E0909376112E
:100B10008093751184EF91E0909378118093771111
:100B200010927B1110927A111092691110926A1131
:100B300010926B1110926C111092791181E08093D8
:100B4000F9101092FA1083EC9BEAA6E7BBE38093BE
:100B5000FB109093FC10A093FD10B093FE1088ED55
:100B60009BE6A6E7BBE38093FF1090930011A09350
:100B70000111B093021182EF94EEA4E6BBE38093DF
:100B8000031190930411A0930511B09306111092D4
:100B9000F8106CED7AE085EE90E10E94C84D8091EE
:100BA000C6049091C7049093E4108093E310809062
:100BB000C2049090C304A090C404B090C5042091D6
:100BC000BE043091BF044091C0045091C104C501DE
:100BD000B401DED66B017C016093DF107093E010EE
:100BE0008093E1109093E2106091BA047091BB047D
:100BF0008091BC049091BD046093D3107093D41085
:100C00008093D5109093D6108092D7109092D810E0
:100C1000A092D910B092DA102091B6043091B704A6
:100C20004091B8045091B904B3D69B01AC01C701FF
:100C3000B60175D76093DB107093DC108093DD10E4
:100C40009093DE108EE595E09093BB108093BA10E0
:100C50008FEF9FEFDC018093CF109093D010A09383
:100C6000D110B093D2106CED7AE08DE990E10E9442
:100C7000C84D6CED7AE087E990E10E94C84D6CEDBB
:100C80007AE081E990E10E94C84D6CED7AE08BE852
:100C900090E10E94C84D6CED7AE085E890E10E94F9
:100CA000C84D6CED7AE08FE790E10E94C84D6CED85
:100CB0007AE089E790E10E94C84D87E08093A70F12
:100CC0001092A90FFF90EF90DF90CF90BF90AF9060
:100CD0009F908F900895EF920F931F93CF93DF9380
:100CE000E80147FD02C034E001C034E1E42F440FC5
:100CF000FF0BF7FF03C0F195E195F109E32E022FF9
:100D00002E2FAE01BBD0CE01DF91CF911F910F915D
:100D1000EF900895662777273EC21F93FC0199271D
:100D20008827BC01E89411911032E9F3193010F0D2
:100D30001E30C8F31B3249F01D3241F4689405C0DF
:100D40004ED0610F711D811D911D119110531A30EC
:100D5000B8F33EF490958095709561957F4F8F4FD5
:100D60009F4F1F910895FB01DC0105900D9200201B
:100D7000E1F70895FC0105900020E9F78095909532
:100D80008E0F9F1F08954532510518F4423008F028
:100D900004C0FB011082CB010895BB274A3031F417
:100DA000992322F4BDE2909581959F4F4FC0253243
:100DB000310518F4223008F004C0FA011082CA018B
:100DC0000895BB272A3051F4992342F4BDE290954F
:100DD0008095709561957F4F8F4F9F4F16C0592F0B
:100DE000482F372F262F660F771F881F991F660FF2
:100DF000771F881F991F620F731F841F951F660F2F
:100E0000771F881F991F0895BB27FA01A62F621725
:100E1000710581059105330B30FB66F0AA27660F3B
:100E2000771F881F991FAA1FA21710F0A21B639596
:100E30003850A9F7A05DAA3308F0A95DA19336F751
:100E4000B111B1931082CA0104C4BB27FB0155271D
:100E5000AA27880F991FAA1FA41710F0A41B839517
:100E60005051B9F7A05DAA3308F0A95DA19300978E
:100E700079F7B111B1931192CB01EBC34F925F920D
:100E80006F927F929F92AF92BF92CF92DF92EF923A
:100E9000FF920F931F93CF93DF93CDB7DEB72997C0
:100EA0000FB6F894DEBF0FBECDBF6A01122FB02E71
:100EB0002BE3201720F0FF24F394F00E02C0BCE3D4
:100EC000FB2E0F2D27E0AE014F5F5F4FCAD2AC0162
:100ED0008981982F9970913031F0E1FC06C0E0FED5
:100EE00006C090E205C09DE203C09BE201C090E015
:100EF000EE2DE07183FF3CC0911102C083E001C080
:100F000084E0811718F4212F281B01C020E0E11193
:100F10000BC0F601822F30E2882319F03193815003
:100F2000FBCFC20ED11C20E0992329F0D6019C935F
:100F3000F60131966F01C6010396E2FE0AC03EE457
:100F4000D6013C9341E411964C93119712963C9331
:100F500006C03EE6F601308341E641833283FC0160
:100F6000322F40E2332309F442C041933150FACF8B
:100F700082FF44C0911102C083E001C084E0811768
:100F800018F4212F281B01C020E0E1110BC0F6014D
:100F9000822F30E2882319F031938150FBCFC20EAB
:100FA000D11C20E0992329F0D6019C93F6013196BB
:100FB0006F01C6010396E2FE0BC039E4D6013C93F3
:100FC0003EE411963C93119736E412963C9307C089
:100FD00039E6F60130833EE6318336E63283FC01A2
:100FE000322F40E2332319F041933150FBCFFC0103
:100FF000E20FF11D10828EEF9FEFB7C0F1E091116B
:1010000001C0F0E06F2F70E01416150624F49A0169
:101010002F5F3F4F02C021E030E0260F371FBB207B
:1010200029F06B2D70E06F5F7F4F02C060E070E0D1
:10103000260F371F612F70E0261737071CF4121B8D
:10104000212F01C020E03E2D387159F4D601322FF6
:1010500060E2332319F06D933150FBCFC20ED11CE7
:1010600020E0FF2331F0D6019C93B6016F5F7F4FE4
:101070006B01E1110BC0F601922F30E3992319F0B7
:1010800031939150FBCFC20ED11C20E09F2D940FC5
:101090003A81782F7071A72E84FF03C0313309F491
:1010A0009150191624F4993018F098E001C091E09D
:1010B000E42F852F57FF02C0E0E080E06E2F782FED
:1010C000E0E0F0E0AEE29A2E3A01691A71082A01D6
:1010D000461A570A0B2D10E01195019511096F3F23
:1010E0008FEF780729F4D6019C92C60101966C0116
:1010F0004617570784F0661677066CF47F01E40CF8
:10110000F51CA1E0B0E0AC0FBD1FEA0EFB1ED7013D
:101110001196BC9002C090E3B92E615071093196CE
:10112000C60101967C016017710724F0D601BC92BC
:101130006C01D5CF6417750741F4363320F435338D
:1011400021F4A11002C081E3B82EF601B082F701AC
:10115000822F90E2882319F091938150FBCFF70101
:10116000E20FF11D108280E090E029960FB6F8940E
:10117000DEBF0FBECDBFDF91CF911F910F91FF90CA
:10118000EF90DF90CF90BF90AF909F907F906F9047
:101190005F904F9008956F927F928F929F92AF923F
:1011A000BF92CF92DF92EF92FF920F931F93CF9354
:1011B000DF93EC017B016115710519F0DB018D9363
:1011C0009C938E010F5F1F4F7880872D90E021D276
:1011D000892B11F0E801F5CFBDE27B1205C00F5F4E
:1011E0001F4F7980C1E008C0EBE27E1204C08E017F
:1011F0000E5F1F4F7980C0E06801F1E0CF1AD1087F
:1012000043E050E06AE272E0C6010BD2892BE9F4B8
:10121000680122E0C20ED11C45E050E065E272E0B8
:10122000C601FFD1892B21F4680187E0C80ED11CCB
:10123000E114F10419F0D701CD92DC92C111F9C08B
:1012400060E070E080E89FE7FDC043E050E062E2CC
:1012500072E0C601E6D1892B51F4E114F10409F4DE
:10126000EDC00E5F1F4FF70111830083E7C06801D7
:1012700060E070E0CB0100E010E0F601D0EDD70DAA
:10128000DA3050F52C2F2260622E2C2F2870C2FFEE
:1012900005C0211127C00F5F1F4F24C0222311F06A
:1012A00001501109A5E0B0E09B01AC0130D34B0126
:1012B0005C01880C991CAA1CBB1CC501B4016D0FF4
:1012C000711D811D911D6839A9E97A078A07A9E175
:1012D0009A0740F0C66005C0DE3F51F4C3FD44C02C
:1012E000C8606C2EBFEFCB1ADB0A7080C62DC5CF4D
:1012F0002D2F2F7D2531C1F540814D3211F4C06174
:1013000006C04B3221F0319621E030E006C0329623
:10131000D60111964C9122E030E0A0EDA40FAA3046
:1013200018F0E21BF30B20C040E050E04038BCE076
:101330005B075CF49A01220F331F220F331F420F09
:10134000531F440F551F4A0F511D3196DF0111974E
:101350002C91A0EDA20FAA3048F3C4FF03C0519511
:1013600041955109040F151FC1FF07C0E114F10495
:1013700021F03197D701ED93FC937FD1C370C33037
:1013800019F06B017C0106C06B017C01F7FAF09447
:10139000F7F8F09420E030E0A901C701B60169D167
:1013A000882309F443C017FF06C011950195110960
:1013B000C1E4D2E002C0C9E5D2E05E01B8E1AB1AF7
:1013C000B1084601BE2DAF2D90E2E92EF12C0E158D
:1013D0001F057CF0FE012591359145915491B40192
:1013E0008B2F9A2FABD14B01B82FA92F0E191F09A4
:1013F000EECF2497F594E794CA15DB0541F7640115
:10140000EB2EFA2E8E2D880F8F2D881F8F3F41F0E7
:1014100020E030E0A901C701B6012BD1811106C03F
:1014200082E290E09093BE118093BD11C701B60196
:1014300009C060E070E080E89FEF04C060E070E009
:1014400080EC9FE7DF91CF911F910F91FF90EF907C
:10145000DF90CF90BF90AF909F908F907F906F90D4
:101460000895283008F027E03327DA01990F311D5D
:1014700087FD916000966105710539F432602E5F39
:101480003D9330E32A95E1F708959F3F30F080388F
:101490007105610509F03C5F3C5F3D93913008F0B8
:1014A0008068911DDF93CF931F930F93FF92EF926C
:1014B000192F987F9695E92F96959695E90FFF2716
:1014C000E954FD4F99273327EE24FF24A701E701B4
:1014D00005900894079428F4360FE71EF81E491F5C
:1014E000511D660F771F881F991F0694A1F705905D
:1014F000079428F4E70EF81E491F561FC11D770FE9
:10150000881F991F661F0694A1F70590079428F479
:10151000F80E491F561FC71FD11D880F991F661F40
:10152000771F0694A1F70590079420F4490F561FE2
:10153000C71FD81F990F661F771F881F0694A9F72A
:1015400084911095177041F0D695C795579547959A
:10155000F794E7941A95C1F7EDE5F2E068941590D9
:10156000159135916591959105907FE27395E118FC
:10157000F10A430B560BC90BD009C0F7E10CF11E61
:10158000431F561FC91FD01D7EF4703311F48A9576
:10159000E6CFE894015030F0080F0AF40027021754
:1015A00008F4202F2395022F7A3328F079E37D93D6
:1015B0002A95E9F710C07D932A9589F606949795A8
:1015C0006795379517951794E118F10A430B560B59
:1015D000C90BD00998F023957E9173957A3308F062
:1015E00070E37C932013B8F77E9170617D9330F0A7
:1015F000839571E37D9370E32A95E1F71124EF90D1
:10160000FF900F911F91CF91DF91992787FD9095C2
:1016100008959111F6C0803219F089508550D0F7A5
:101620000895FB01DC014150504088F08D918134D8
:101630001CF08B350CF4805E659161341CF06B35C9
:101640000CF4605E861B611171F3990B0895881B81
:10165000FCCFDC01FC01672F71917723E1F7329712
:1016600004C07C916D9370836291AE17BF07C8F37D
:10167000089540D008F481E00895E89409C097FBEC
:101680003EF490958095709561957F4F8F4F9F4F59
:101690009923A9F0F92F96E9BB279395F69587959D
:1016A00077956795B795F111F8CFFAF4BB0F11F460
:1016B00060FF1BC06F5F7F4F8F4F9F4F16C0882307
:1016C00011F096E911C0772321F09EE8872F762F3D
:1016D00005C0662371F096E8862F70E060E02AF07E
:1016E0009A95660F771F881FDAF7880F969587956A
:1016F00097F90895990F0008550FAA0BE0E8FEEF3F
:1017000016161706E807F907C0F012161306E407C5
:10171000F50798F0621B730B840B950B39F40A26BE
:1017200061F0232B242B252B21F408950A2609F49C
:10173000A140A6958FEF811D811D08950BD07BC020
:101740006CD028F071D018F0952309F05DC062C00C
:101750001124A5C081D0A0F3959FD1F3950F50E03F
:10176000551F629FF001729FBB27F00DB11D639F53
:10177000AA27F00DB11DAA1F649F6627B00DA11DF9
:10178000661F829F2227B00DA11D621F739FB00D9F
:10179000A11D621F839FA00D611D221F749F33270F
:1017A000A00D611D231F849F600D211D822F762FA8
:1017B0006A2F11249F5750408AF0E1F088234AF0A5
:1017C000EE0FFF1FBB1F661F771F881F91505040F1
:1017D000A9F79E3F510570F017C061C05F3FECF361
:1017E000983EDCF3869577956795B795F795E795DD
:1017F0009F5FC1F7FE2B880F911D9695879597F9EE
:10180000089599278827089597F99F6780E870E0E1
:1018100060E008959FEF80EC089500240A94161666
:10182000170618060906089500240A9412161306CE
:10183000140605060895092E0394000C11F488235C
:1018400052F0BB0F40F4BF2B11F460FF04C06F5F78
:101850007F4F8F4F9F4F089557FD9058440F551F4E
:1018600059F05F3F71F04795880F97FB991F61F022
:101870009F3F79F087950895121613061406551F99
:10188000F2CF4695F1DF08C0161617061806991F05
:10189000F1CF86957105610508940895E894BB27FA
:1018A00066277727CB0197F90895F999FECF92BD66
:1018B00081BDF89A992780B50895262FF999FECF12
:1018C0001FBA92BD81BD20BD0FB6F894FA9AF99A5D
:1018D0000FBE01960895052E97FB16F400940FD0C5
:1018E00057FD05D024D007FC02D046F408C050951F
:1018F0004095309521953F4F4F4F5F4F08959095FC
:101900008095709561957F4F8F4F9F4F089531D08F
:10191000A59F900DB49F900DA49F800D911D112443
:101920000895B7FFF4CFF3DF821B930B0895A1E274
:101930001A2EAA1BBB1BFD010DC0AA1FBB1FEE1F49
:10194000FF1FA217B307E407F50720F0A21BB30B94
:10195000E40BF50B661F771F881F991F1A9469F710
:1019600060957095809590959B01AC01BD01CF016C
:101970000895A29FB001B39FC001A39F700D811D68
:101980001124911DB29F700D811D1124911D089588
:101990005058BB27AA270ED04ECF3FDF30F044DF90
:1019A00020F031F49F3F11F41EF434CF0EF4E09593
:1019B000E7FB2ACFE92F50DF80F3BA1762077307DE
:1019C0008407950718F071F49EF568CF0EF4E09542
:1019D0000B2EBA2FA02D0B01B90190010C01CA01E9
:1019E000A0011124FF27591B99F0593F50F4503E94
:1019F00068F11A16F040A22F232F342F4427585F86
:101A0000F3CF469537952795A795F0405395C9F79D
:101A10007EF41F16BA0B620B730B840BBAF0915055
:101A2000A1F0FF0FBB1F661F771F881FC2F70EC0F4
:101A3000BA0F621F731F841F48F4879577956795C7
:101A4000B795F7959E3F08F0B3CF9395880F08F0B0
:101A50009927EE0F979587950895DFDE58F080E877
:101A600091E009F49EEFE0DE28F040E851E059F4FF
:101A70005EEF09C0CFCE12CFE92FE078EDDE68F33C
:101A8000092E052AC1F3261737074807590738F0EA
:101A90000E2E07F8E02569F0E025E0640AC0EF6348
:101AA00007F8009407FADB01B9019D01DC01CA01C6
:101AB000AD01EF9343D0BFDE0AD05F91552331F0E3
:101AC0002BED3FE049E450FD49EC63CF0895DF93EF
:101AD000DD27B92FBF7740E85FE3161617064807E2
:101AE0005B0710F4D92F0ED19F938F937F936F9341
:101AF00052D2E2E7F1E0DDD09EDE2F913F914F918F
:101B00005F9128DEDD2349F09058A2EA2AED3FE0FC
:101B100049EC5FE3D0785D274DDFDF918CCE0CD0B0
:101B20008ACE82DE40F079DE30F021F45F3F19F09A
:101B30006BCE5111B4CE6ECE8FDE98F39923C9F3DC
:101B40005523B1F3951B550BBB27AA2762177307C3
:101B5000840738F09F5F5F4F220F331F441FAA1F77
:101B6000A9F333D00E2E3AF0E0E830D09150504037
:101B7000E695001CCAF729D0FE2F27D0660F771FE5
:101B8000881FBB1F261737074807AB07B0E809F0C7
:101B9000BB0B802DBF01FF2793585F4F2AF09E3F5C
:101BA000510568F031CE7BCE5F3FECF3983EDCF31D
:101BB000869577956795B795F7959F5FC9F7880FD5
:101BC000911D9695879597F90895E1E0660F771F27
:101BD000881FBB1F621773078407BA0720F0621BB8
:101BE000730B840BBA0BEE1F88F7E095089519F478
:101BF0000EF00ACE53CE0ECE37DEC8F39638C0F7BD
:101C000007F80F92E8942BE33AEA48EB5FE7A4DD8C
